:020000040000FA
:1000000008480400010000003CCC00003CCC00008B
:100010003CCC00003CCC00003CCC00003CCC0000C0
:100020003CCC00003CCC00003CCC00003CCC0000B0
:100030003CCC00009A0900003CCC00003CCC000005
:100040003CCC0000C0090000E60900003CCC0000E8
:100050003CCC00003CCC00003CCC00008EA1000059
:100060003CCC00003CCC00003CCC000082100000E6
:100070003CCC0000B6070000220900003CCC000088
:100080003CCC0000DC0700003CCC00003CCC000075
:100090003CCC00001A0A0000400A0000620900007F
:1000A0003CCC00003CCC00003CCC00003CCC000030
:1000B0003CCC00003CCC00003CCC00003CCC000020
:1000C0003CCC00003CCC00003CCC00003CCC000010
:1000D0003CCC00003CCC00003CCC00003CCC000000
:1000E0003CCC00003CCC00003CCC00003CCC0000F0
:1000F0001C1100003CCC00003CCC0000900700002C
:10010000501200003CCC00003CCC00003CCC000075
:100110003CCC00003CCC00003CCC00003CCC0000BF
:100120003CCC00003CCC00003CCC00003CCC0000AF
:100130003CCC00003CCC00003CCC00003CCC00009F
:100140003CCC00003CCC00007C0700003CCC000014
:100150003CCC00003CCC00003CCC00003CCC00007F
:100160003CCC00003CCC00003CCC00003CCC00006F
:100170003CCC00003CCC00003CCC0000B6110000A0
:10018000740A00003CCC00003CCC00003CCC0000D9
:100190003CCC00003CCC00003CCC000054080000EB
:1001A0003CCC00003CCC00003CCC00003CCC00002F
:1001B0003CCC00003CCC00003CCC00003CCC00001F
:1001C0003CCC00003CCC00003CCC00003CCC00000F
:1001D0003CCC00003CCC00003CCC00003CCC0000FF
:1001E0003CCC00003CCC00003CCC00003CCC0000EF
:1001F0003CCC00003CCC00003CCC00003CCC0000DF
:1002000000000000000000003CCC00003CCC0000DE
:100210003CCC00003CCC00003CCC00003CCC0000BE
:100220003CCC00003CCC00003CCC00003CCC0000AE
:100230003CCC00009A0900003CCC00003CCC000003
:100240003CCC0000C0090000E60900003CCC0000E6
:100250003CCC00003CCC00003CCC00008EA1000057
:100260003CCC00003CCC00003CCC000082100000E4
:100270003CCC0000B6070000220900003CCC000086
:100280003CCC0000DC0700003CCC00003CCC000073
:100290003CCC00001A0A0000400A0000620900007D
:1002A0003CCC00003CCC00003CCC00003CCC00002E
:1002B0003CCC00003CCC00003CCC00003CCC00001E
:1002C0003CCC00003CCC00003CCC00003CCC00000E
:1002D0003CCC00003CCC00003CCC00003CCC0000FE
:1002E0003CCC00003CCC00003CCC00003CCC0000EE
:1002F0001C1100003CCC00003CCC0000900700002A
:10030000501200003CCC00003CCC00003CCC000073
:100310003CCC00003CCC00003CCC00003CCC0000BD
:100320003CCC00003CCC00003CCC00003CCC0000AD
:100330003CCC00003CCC00003CCC00003CCC00009D
:100340003CCC00003CCC00007C0700003CCC000012
:100350003CCC00003CCC00003CCC00003CCC00007D
:100360003CCC00003CCC00003CCC00003CCC00006D
:100370003CCC00003CCC00003CCC0000B61100009E
:100380009E4801003CCC00003CCC00003CCC00006E
:100390003CCC00003CCC00003CCC000054080000E9
:1003A0003CCC00003CCC00003CCC00003CCC00002D
:1003B0003CCC00003CCC00003CCC00003CCC00001D
:1003C0003CCC00003CCC00003CCC00003CCC00000D
:1003D0003CCC00003CCC00003CCC00003CCC0000FD
:1003E0003CCC00003CCC00003CCC00003CCC0000ED
:1003F0003CCC00003CCC00003CCC00003CCC0000DD
:1004000000480400010000000F122300807D24003A
:1004100000018800000000000B000700007D29009B
:100420000100200010000700000020000000E00094
:1004300002003200000002000000000030B502009F
:10044000000000000000FE004440A90020502100F0
:100450000000E0000300320000002000A00188003E
:100460004440A80000000600F8FF2000591C2100AD
:1004700091018800800078000000EB001A0037002E
:100480008180E80032A0B4009101BA00E28040000F
:1004900032A0B4009102BA00E280400032A0B40061
:1004A0000002EB00472BDE00F507B200602CE100F4
:1004B00009003A00330007000700E00002003200A4
:1004C0000059EB00010037000201E8008301E90058
:1004D000F8FF3E00040037006128E100010032000F
:1004E0000082EB00040007001101BA000200E000E6
:1004F000E3FF3A0000000600220007000700E000CA
:10050000020032003159BA00020037008100E800D1
:100510000201E8008301E90017003200190007001A
:100520000700E000020032002159BA000200370043
:100530008100E9000201E8008301E9000D003200BA
:100540000400E00003003A00E280400032A0B40062
:10055000E9FF37000B0007000700E000020032004F
:1005600011D9BA00010037000201E8008301E90057
:10057000F5FF3A008100E800E180400032A0B400BD
:10058000000006000810E600020037000910E6002F
:10059000020037008083EB00000006008003EB00C0
:1005A0000000060091018800800078000000EB0048
:1005B00015003700E280400032A0B4009101BA007B
:1005C000E280400032A0B4009102BA00E280400014
:1005D00032A0B4000002EB00472BDE00F507B200AA
:1005E000602CE10004003A000059EB008301E900AF
:1005F000FDFF3E00040037006128E10001003200E9
:100600000082EB00040007001101BA000200E000C4
:10061000E8FF3A00000006003159BA008301E90002
:100620000C0032002159BA008301E90008003200B1
:100630000400E00003003A00E280400032A0B40071
:10064000F5FF370011D9BA008301E900FAFF3A003B
:100650008100E800E180400032A0B4000000060004
:10066000AE9D0400000000009E9B040000000000FE
:10067000A29B040000000000D29B040000000000C8
:10068000FA9C0400000000000E7504000000000049
:1006900040750400000000007075040000000000B8
:1006A000B275040000000000F475040000000000B2
:1006B00036760400000000007C7604000000000094
:1006C000E076040000000000247704000000000031
:1006D0006877040000000000D677040000000000E6
:1006E0004E78040000000000A07804000000000024
:1006F000BA78040000000000447904000000000003
:100700008E79040000000000C87904000000000099
:10071000027A040000000000967A04000000000045
:10072000CA7B040000000000AE930400000000003B
:10073000589404000000000026940400000000000B
:100740008A94040000000000BC9404000000000033
:10075000F094040000000000709504000000000008
:10076000CC950400000000009E95040000000000ED
:100770007697040000000000FA95040000000000D5
:100780004C96040000000000EA96040000000000FF
:1007900018970400000000003097040000000000DB
:1007A0004897040000000000A0970400000000002B
:1007B00012B504000000000094A104000000000035
:1007C0003EB404000000000024B404000000000057
:1007D0004CB404000000000058B404000000000005
:1007E000B0BF0400000000001CB8040000000000BE
:1007F0006AC60400000000007CA90400000000009C
:10080000487C040000000000607E0400000000003E
:1008100030CC04000000000078AC040000000000B0
:10082000020AB900001BB9000200B80081004200B2
:1008300081004300000006008001780011000900DB
:100840008280D8008001FD00110009004288D80094
:1008500083007800000006006022B8000602200035
:100860000000D0008180D2000482D2008582D200B4
:100870000000A0000202520083825A0003003100EF
:100880000202420083824A000000A1000603E90040
:10089000F3FF3A0000000600839F68000100E000BB
:1008A00002003D0060001000E08018000300E0003E
:1008B00002003D0060011100E0811900E6FF070021
:1008C0004F00E00002003B0060001000E0801800D4
:1008D00000000600889FBE008A9FBE008C1F780023
:1008E0000205BE000004BE000006EB00E00F500051
:1008F000E08F5800E00F5900E08F590007003D00DD
:100900006000B8006011B8000804500089845800E5
:100910000A0559008B8559001C002000E00F520089
:10092000E08F5A00E00F5B00E08F5B0002003D00AB
:100930000F0007000C00A2000800BE000A01BE0064
:100940001D0107000203BE000002BE000C00E00013
:1009500001003200060007000400BE000601BE00D0
:100960004F0678004F05BE004F04BE000000060091
:100970006000B8006011B800040250008582580081
:10098000060359008783590000000600881F78007D
:10099000000478005001BE004000BE00040040008A
:1009A000858048000601490087814900009CBE00FF
:1009B0000294BE000400E1000588E1000690E10019
:1009C0000798E10002003100680044001008E800C8
:1009D0004F04780000000600F4874700889FBE009F
:1009E0008A9FBE008C9FBE008E1F78000205BE004D
:1009F0000004BE00D4B79F00E5B79F00F6B79F0084
:100A000087BF9F000000EB00C0B79F00B0B79F00FA
:100A1000A0B79F0090B79F0080B79F000D042000F3
:100A2000BFB097004FB09700000140000000E00009
:100A30000F003D004F08DE0000007100C0B79F00AE
:100A40009E00070001003D0012002000A1000700E9
:100A500001003D0012002000A6000700B1000700C1
:100A6000B60007000F004000C8FF07002200370053
:100A70004F08DE0000067100CCB79F008F00070012
:100A800001003D00120020009200070001003D001F
:100A90001200200097000700A20007000FB2970085
:100AA0009FB297002FB39700BFB39700A90007002C
:100AB0000000520081805A0002015B0083815B00CC
:100AC00080B79F0091B79F00A2B79F00B3B79F0068
:100AD0000007EB009F0007000020E10001A8E100F3
:100AE00002B0E10003B8E100010031001E00200067
:100AF0000E005600C0B79F004FB297000400E00000
:100B00000700350010002000010020006011B8002F
:100B100008047000898470000A0571008B857100DB
:100B20008D06E900BEFF3A000400E00003003D002E
:100B3000820007000F00400094FF07004FA89700B5
:100B40000000E00004003A000FB497009FB4970043
:100B50002FB59700BFB59700940007004F077800A6
:100B60004F06BE004F05BE004F04BE004F01B1004E
:100B700000000600881F780018002000881F7800F9
:100B800095FF07008F87E9004F04780000000600FA
:100B9000801FEB0090FF07008F87E9000000060030
:100BA000889FBE008A9FBE008C1F78006E000700E1
:100BB00007003D0073000700E00F5B00E08F5B0063
:100BC00007003D00320007000006EB00040037007C
:100BD0003400070002003D002A0007001C0020002E
:100BE00072000700E3FF07000203BE000002BE0020
:100BF0000C00E00001003200220007000400BE00EB
:100C00000601BE004F0678004F05BE004F04BE002F
:100C100000000600889FBE008A9FBE008C1F7800DF
:100C20005100070005003D0056000700E00F5B0083
:100C3000E08F5B0006003D0004003700190007004C
:100C400003003D006000B8006011B800100007000C
:100C500056000700CEFF07000203BE000002BE00E0
:100C60000C00E00001003200060007000400BE0096
:100C70000601BE004F0678004F05BE004F04BE00BF
:100C8000000006006000B8006011B80000003700E6
:100C900004025000858258000603590087835900DA
:100CA000000006000006EB00E00F5200E08F5A0043
:100CB000E00F5B00E08F5B00000006000180400059
:100CC00090B79F000001EB008FB097000100E0009B
:100CD000000006000200700090B79F0001804000F5
:100CE00080B79F000001EB00FFA897000100E00023
:100CF000000006000200700080B79F0001804000E5
:100D00006FAA9700CF20DE0001007000F0AF9F00B7
:100D100004024200250007004F18DE0000027200A6
:100D200000000600E4AF9F000804440089844C00E2
:100D30000A054D008B854D00000006003FB297006C
:100D4000CFB297005FB39700EFB3970000FE2F007C
:100D5000000006003FB09700CFB097005FB197004A
:100D6000EFB19700000006000205BE000004BE00BF
:100D7000E00F5000E08F5800E00F5900E08F59005D
:100D8000000006006000B8006011B80008045000C0
:100D9000898458000A0559008B8559001C002000E1
:100DA000E00F5200E08F5A00000006000800BE006D
:100DB0000A01BE0000000600889FBE008A9FBE0098
:100DC0008C9FBE000404B8000506B80089044600E4
:100DD00060854E000606B8000A054600E0854E0014
:100DE0000706B8008B054600040EB80089044600CB
:100DF0000A854E00E0854D00050EB8000A05460044
:100E00008B854E00060EB8008B0546000416B80010
:100E10000A0546008B854E000516B8008B05460076
:100E2000041EB8008B0546000800BE000A01BE0083
:100E30004F06BE004F05BE004F04BE000000060076
:100E40000400FA00E0BF9F00E48157008129780088
:100E50000002EB000F0037006FB897009040780059
:100E60007FB89700104078000402E80080CF50005F
:100E7000040032008180FB000080FB0000805000F5
:100E8000070037006FB897000000E800E0BF9F0040
:100E90009309E800820F5200EFFF3A000000EB00D8
:100EA0000080FA00000006008001EB00020037001D
:100EB000817178008301E800828F5100FCFF3A00C5
:100EC00000000600800078003004E000FEFF3A00D9
:100ED000010050000000E900000006008001EB0066
:100EE0000200370061F079008301E800828F510031
:100EF000FCFF3A00000006003400F800881F78006C
:100F000008002000A80188004F0478008D00A90087
:100F10009D00A9008AA0A8003400F9000040060046
:100F20003600F800809FBE00829FBE00849FBE00F6
:100F3000869FBE003400F80000002000A001880059
:100F40008AA0A9009AA0A9000000EB00B5560700EE
:100F50003400F9004F03BE004F02BE004F01BE0037
:100F60004F00BE003600F900004006003600F800D1
:100F7000809FBE00829FBE00849FBE00869FBE00F1
:100F80003400F80000002000A00188008660A9005D
:100F9000DA42E20001003D00E35B07003400F900A3
:100FA0004F03BE004F02BE004F01BE004F00BE0007
:100FB0003600F900004006003600F800809FBE00B1
:100FC000829FBE00849FBE00869FBE003400F80052
:100FD00000002000A001880086E0A900E30B80004B
:100FE00078C1BF0081CFB3000140600078E1B70055
:100FF000F0E2A80035C6A90022FA8000C9C2BF00ED
:101000000058A3000B003A00007122000018B8003D
:1010100009FE070022C521000001510093002000B5
:10102000110009000301D80080017800CDA2A900B9
:101030000E0037000200E0000B0032006F10B80015
:1010400003004000E080480068004000E080480065
:101050004C09DD004400DE0000007100C408DE0021
:1010600020FA88000100370023FA8800EC62A9000A
:1010700031FA80000100E000020032000300780035
:1010800001000100F0C2A900C9A2A9003400F900C2
:101090004F03BE004F02BE004F01BE004F00BE0016
:1010A0003600F900004006003600F800809FBE00C0
:1010B000829FBE00849FBE00869FBE003400F80061
:1010C00000002000A00188008FA0A90011F6800078
:1010D000C01EE2000E003A001000200000F688005A
:1010E000200C8000F0F5880000002800E0F5880062
:1010F000E0002000D0F588006011B8000100780001
:10110000C831070010F680009B3407004600370006
:101110006011B80001007800C231070080C1BF0033
:101120000048A3003D00320037003700210C80004A
:10113000F0F5800000815000F1F58800F0232A00CE
:101140000000410021D22200810F50000C003E001F
:10115000E1F58000D2F580008201E8001000200057
:101160000300DD00008060000000D100808070007E
:10117000E1F588000201E900D2F58800240037007B
:10118000B051270000004100C1782300810F5000BA
:101190000C003E00E2F58000D1F580000100E8007F
:1011A000130020000018DD000000610013003A0069
:1011B0000118DD0000007100E0F588000100E90081
:1011C0000F00370020272C00800F51000E00360042
:1011D000E2F58000D1F580000100E8001300200056
:1011E0000018DD0000006100070032000100E90086
:1011F0000018DD0000007100E0F588000180E900C2
:10120000D0F5880002003700825E07000600370034
:10121000BA1EE20001003C007E5E070080C1BF00F4
:101220000038A300C1FF3A003400F9004F03BE00AC
:101230004F02BE004F01BE004F00BE003600F90055
:10124000004006003600F800809FBE00829FBE006E
:10125000849FBE00869FBE003400F800000020007E
:10126000A00188008680A90082B48000A1B480001B
:10127000F0072000808F50000400360060692100D4
:101280000200E00004003A00060037000200E0001F
:101290000400320060712100020001000000E00043
:1012A00001003A00055C07003400F9004F03BE005E
:1012B0004F02BE004F01BE004F00BE003600F900D5
:1012C000004006003600F800809FBE00829FBE00EE
:1012D000849FBE00869FBE003400F80000002000FE
:1012E000A001880087A0A90091B48000F007200029
:1012F000808F50000400360060792100005C0700F8
:10130000607921000300370060812100FC5B070049
:10131000608121005C5007003400F9004F03BE00DB
:101320004F02BE004F01BE004F00BE003600F90064
:10133000004006003600F800809FBE00829FBE007D
:10134000849FBE00869FBE003400F800000020008D
:10135000A00188000000EB0031F1800001000100D5
:101360008460A9003400F9004F03BE004F02BE00A4
:101370004F01BE004F00BE003600F90000400600DD
:101380003600F800809FBE00829FBE00849FBE0092
:10139000869FBE003400F80000002000A0018800F5
:1013A00084E0A9001000200051F18000010001003C
:1013B0003400F9004F03BE004F02BE004F01BE00D3
:1013C0004F00BE003600F900004006003600F8006D
:1013D000809FBE00829FBE00849FBE00869FBE008D
:1013E0003400F80000002000A00188008500A9005A
:1013F00060F1800066006000E60F500003003A00D4
:101400009000200051F180000200370020002000F1
:1014100071F18000010001003400F9004F03BE00AB
:101420004F02BE004F01BE004F00BE003600F90063
:10143000004006003600F800809FBE00829FBE007C
:10144000849FBE00869FBE003400F800000020008C
:10145000A00188008760A9003000200091F1800081
:10146000010001003400F9004F03BE004F02BE002E
:101470004F01BE004F00BE003600F90000400600DC
:101480003600F800809FBE00829FBE00849FBE0091
:10149000869FBE003400F80000002000A0018800F4
:1014A0008780A900A0F1800066006000E60F500070
:1014B00003003A00A000200091F1800002003700F4
:1014C00040002000B1F18000010001003400F9006B
:1014D0004F03BE004F02BE004F01BE004F00BE00D2
:1014E0003600F900004006003600F800809FBE007C
:1014F000829FBE00849FBE00869FBE00889FBE0064
:101500008A1F78003400F80000002000A001880045
:101510000200FA0000828000E10F500008003A004B
:1015200094C4BF000068A30005003A008AA4EF003D
:101530008C04A8008C84A800200020000082880071
:101540008AC4BF000028A3000C00320082C4BF0080
:101550000048A30009003200080120000824880088
:101560008430EF000001EB008000EB00400720001A
:10157000F05E07008284A9000824880088C4BF00A8
:101580000018A300D4023A008AC4BF000008A300D8
:10159000090032008CC4BF000008A300060032001E
:1015A000FF1007009EC0A8004000200000828800B5
:1015B00010002000502488008AC4BF000048A30007
:1015C0000D0032008CC4BF000048A3000A003200A6
:1015D0008284A80008012000582488001000200000
:1015E000208488000001EB008000EB005007200001
:1015F000D05E0700582488008AC4BF000028A300DA
:101600000F0032008CC4BF000028A3000400320089
:10161000120020008000EB0030072000C55E0700AC
:1016200040002000502488008650E2000100320073
:101630008670ED008650E20001003A001F1107009D
:101640008A44E20014003D008C44E20012003D0098
:10165000AAC4BF000018A3000D003200328280002F
:101660009240900000C8B30080CF500007003A00BD
:10167000808280009040900040C8B30080CF50002E
:1016800002003A006840400010419800AA24A900D6
:1016900000082000502488008AC4BF000018A3005E
:1016A0000A0032008CC4BF000018A30007003200FB
:1016B000120020008000EB00F0FF27009D5E070075
:1016C0008EA4EF00200020005024880000828000BB
:1016D000E30F5000800236008CC4BF000038A30026
:1016E0007D0232000045EB008AC4BF000038A30031
:1016F00079023200902480006CF0B7006CD0BF00FB
:101700000080FB004400DE006AF0B700800020008B
:10171000502488006CD0BF000038A30004003A00B9
:101720006AD0BF000080FB002107210003003700C2
:101730006AD0BF000080FB00E106210001004000EC
:1017400010417800E14061000104A2001004A100F2
:1017500010C870006A50E20058023A00D0C2B300CC
:1017600086F0B7006CD0BF0080017800B30FB200E4
:1017700015023A006CD0BF00C00FB200010021007A
:101780000101400032828800428288004850AA004D
:1017900012409000C043B20041C3B300814F5000DB
:1017A0009A013A00820078000203210011009000A3
:1017B00010F17900110090000000E80090009800FE
:1017C0008301E800E88F5100F8FF3A00920098008A
:1017D0005670EF007630EF007C30EF007E30EF0087
:1017E0008030EF005870EF0081828000114090003F
:1017F0000074A100904098005050AA00818280009F
:10180000114090000074A100904098005050AA0030
:1018100041828000114090000074A1009040980027
:101820005C70EF005E30EF006270EF0063D0BF00CD
:101830006370EF0064D0BF006470EF0030D0BF0071
:101840000046B20040013A0031D0BF000080FB00EA
:1018500001002000EB0F5000E08F58003A013E00DD
:10186000006001005D003700890037003601370055
:1018700087003700340137000600370008003700C2
:101880002D013700530037003300370018013700AF
:10189000210137005CF0A8008000200045003700DF
:1018A000010321009140780000C8B30080CF5000B0
:1018B00025013A0000CCB3005CF0B70033D0BF0084
:1018C000E24F500008003200E34F50001300320096
:1018D000E14F50001E003A0000122100D082880023
:1018E000200120001800370032D0BF000080FB002C
:1018F00000004000E11B210060807800D082880059
:10190000D0828000204090005EF0B700D08280003E
:10191000304090005FF0B7000B01370032D0BF00BD
:10192000E24F50000A003E0032D0BF000080FB00B2
:1019300000004000011C210060807800D0828800F7
:10194000D08280001080FB00F0828800FE0037000B
:101950005C70EF00FC0037005CF0A800AC24EF00E6
:10196000AE24EF000000EB0001002100010178002F
:101970000019EB000019EB000000E800EC0F50002C
:10198000FBFF3A009424A8004470EF009424A900BF
:101990008000210080828800318288004182880096
:1019A00032D0BF0042F0B7004250E20003003A00DC
:1019B0000001200000828800E300370012002000B0
:1019C0002104210010002000DA5D07000002200041
:1019D000F8FF370020042100C90037003870EF00FD
:1019E0003970EF0030D0BF007F006000E10F500081
:1019F0000B003200E20F50000B0032000000E0004C
:101A00001B003A005CF0A8003810A8001084800089
:101A1000E10F500016003A003830A80014003700DB
:101A20005CF0A800120037005CF0A8003450E2001F
:101A30000500350034D0BF006F006000000040009A
:101A4000A10421000400370034D0BF006F00600003
:101A500000004000010521006080780010409000E7
:101A60000028A3000200320010C0B30038F0B70015
:101A70005C50E200B4003D0080032100D082880069
:101A80005C10A80020C0B3005EF0B700AE003700C5
:101A900032D0BF00E14F50000B003A0030D0BF0001
:101AA0007F40600008003A005CF0A80031D0BF0021
:101AB000E34F500003003A0010002000108488001B
:101AC000010037008230EF003250E2009E003A0001
:101AD00030D0BF007F406000E24F50009A003A00D3
:101AE00034D0BF006F4060009700320034D0BF0098
:101AF0006F006000E20F500093003C000182800004
:101B000000022000808F50008F003A005CF0A80097
:101B10003450E2000A00350034D0BF006F0060008E
:101B200000004000A104210060807800F0BF9F0009
:101B300034D0BF006F00600021072100090037008A
:101B400034D0BF006F00600000004000010521009C
:101B500060807800F0BF9F0034D0BF006F0060004D
:101B6000E106210060C478000808A30004003A00E0
:101B70006FF997000224A100E2FF9F0003003700E5
:101B80006FF897000024A000E0FF9F003450E200AF
:101B90000500350034D0BF006F0060000000400039
:101BA000A10421000400370034D0BF006F006000A2
:101BB00000004000010521007FB9970002B07800C5
:101BC00031D0BF00E34F500014003A007FB89700B7
:101BD0001000E0000B003D003450E200040035002E
:101BE00034D0BF006F0060002107210003003700E0
:101BF00034D0BF006F006000E1062100010040000A
:101C00001014A0007FB897009040900042C8B30025
:101C100082C07000114098004B0037008F84E900AB
:101C20006FF897000024A200E0FF9F00FFB8970024
:101C3000114090001100E0000B003D000074A10075
:101C400090409800FFB89700114090000064A000F9
:101C50009040980022002000FFB89700500020001C
:101C6000345D0700020037000064A0009040980037
:101C70001924A2000818A30006003A007FB99700B3
:101C8000004028001200600001002800810F500071
:101C900013003A003450E2000400350034D0BF0095
:101CA0006F006000210721000300370034D0BF001F
:101CB0006F006000E1062100010040001014A10047
:101CC000FFB8970011409000B043B20090409800D8
:101CD00022002000FFB897005000200019003700B4
:101CE00012409000B043B200104198001600370037
:101CF00034D0BF000080FB004104210001004000FF
:101D0000D08288005C10A80010C0B3005EF0B7005D
:101D10005CF0A8000C0037005CF0A80034D0BF00D5
:101D20000080FB00410421002203210012417800C1
:101D300002F07800040037000001EB008000EB00A7
:101D400020002000FB5C07000001EB008000EB009E
:101D500030002000F75C070094A4A9005C50E2006A
:101D6000130035006250E20008003D0020C0B300BF
:101D700058F0B7007E10E20001003A00A20F070001
:101D80007A30EF007830EF00D000370081C0B30028
:101D900040828000014878004182800000032100D9
:101DA00090009800C0C8B30090409800A40037008D
:101DB0003050E20006003D0010C0B30058F0B700FC
:101DC0007C10E2000C003A008F0F07000A00370079
:101DD00020C0B30058F0B70081C0B300408280003B
:101DE00001487800418280000003210090009800A3
:101DF00040C8B300904098007A30EF007830EF0090
:101E00007610E200B1003A005E00370058D0BF0003
:101E1000E24F50005D003A001242780063D0BF00EC
:101E20000080FB004106210091407800C808DD00D9
:101E3000808070000480FB00810F50000400360099
:101E400063D0BF0041062100914078000042780035
:101E500031062100914078008180FB0064D0BF00F2
:101E60004800DD00010070008480FB00010050008C
:101E7000310621009140780063F0B7004800DE0091
:101E8000410621009140780064F0B70085032100ED
:101E90001000370001062100914078008180FB008E
:101EA00061D0BF004800DD00010070008280FB00AF
:101EB00061D87A00010621009140780060F0B700F7
:101EC0004800DE00110621009140780061F0B70063
:101ED0008301E8000341780084CF5100EDFF390011
:101EE0004282800031062100914078008180FB0011
:101EF00064D0BF004800DD00010070000A0032001D
:101F000080C0B30000497800418280008003210036
:101F10009000980030828000104090000068A3007C
:101F20004E0032004F00370080C0B30000497800F7
:101F300041828000000321009000980040C8B30057
:101F40009040980051062100914078008180FB006C
:101F500066D0BF004800DD000100700007003200BD
:101F600051062100914078008180FB0066D0BF00BF
:101F70004800DD00010070000000010062F0A900CF
:101F80009FFF3700CD0E0700500037008001FD0095
:101F900058F0B7008001FD008010E20008003A0010
:101FA00081C0B300408280000148780041828000F7
:101FB0000003210090009800C0C8B3002A00370039
:101FC00003848800410037006CD0BF00B00FB2001E
:101FD000E80F50003D003A008082800010409000E1
:101FE0004600DE00610460005050AA0000828000BC
:101FF000E80F500008003A0032D0BF000080FB001C
:10200000B0248800000120009604E20001003A009C
:10201000400020000082880058D0BF00E14F5000EF
:1020200013003A0080032100818280009000980014
:10203000C70E070056D0BF00E24F500004003A0020
:1020400041C8B30080828000114098001F00370013
:10205000818280000804E00002003A0080CCB300D6
:102060000100370080C8B300904098001700370087
:102070006250E2000F003D005106210091407800BF
:102080008180FB0066D0BF004800DD0001007000C9
:102090000700320051062100914078008180FB004A
:1020A00066D0BF004800DD000100700000000100A4
:1020B00062F0A9005870EF00040037000001EB0047
:1020C000C1062100200720001A5C07000A45E8002D
:1020D000E44F550084FD3A008EC0A9000080FA004C
:1020E0003400F9004F0578004F04BE004F03BE00D6
:1020F0004F02BE004F01BE004F00BE003600F90087
:10210000004006003600F800809FBE00829FBE009F
:10211000849FBE00869FBE003400F80000002000AF
:10212000A00188000400FA008620A90030F3800096
:10213000E10F500003003A000110800040F38000DE
:102140000148780093202000934178008381FB00B0
:1021500022F38000C719DE008F80E9000000EB0049
:1021600014F380000400010080007800E0BF9F00AD
:10217000E40F50001900320006003C00E20F50004E
:102180001000320013003C00E10F50001C003A0028
:1021900008003700E60F500015003200110035002E
:1021A000E70F500014003200E80F500014003A000E
:1021B000190037007FB8970040F388000662A80036
:1021C000140037007FB897001080FB0010108800C3
:1021D000100037000622A8000E00370006A2A90052
:1021E0000100370006A2A8000682A80009003700F7
:1021F0000642A80007003700623EEF0005003700E6
:10220000E481570042A02000F10F200060BE2A00A8
:10221000955D070031F388000080FA003400F90072
:102220004F03BE004F02BE004F01BE004F00BE0074
:102230003600F900004006003600F800809FBE001E
:10224000829FBE00849FBE00869FBE003400F800BF
:1022500000002000A00188000400FA008A40A900C4
:1022600070F38000E10F500003003A0081108000FD
:1022700080F380000148780093212000934178008A
:102280008381FB0062F38000C719DE008F80E900C4
:102290001000200054F3800004000100800078004A
:1022A000E0BF9F00E40F50001900320006003C0020
:1022B000E20F50001000320013003C00E10F50000C
:1022C0001C003A0008003700E60F500015003200ED
:1022D00011003500E70F500014003200E80F5000E5
:1022E00014003A00190037007FB8970080F3880087
:1022F0001662A800140037007FB897001080FB001A
:1023000090108800100037001622A8000E00370039
:1023100016A2A9000100370016A2A8001682A80084
:10232000090037001642A800070037006A3EEF0098
:1023300005003700E481570042A02000E11320008F
:1023400060BE2A00485D070071F388000080FA0033
:102350003400F9004F03BE004F02BE004F01BE0023
:102360004F00BE003600F900004006003600F800BD
:10237000809FBE00829FBE00849FBE00869FBE00DD
:102380003400F80000002000A00188000400FA00DA
:102390008EA0A900B0F38000E10F500003003A00C6
:1023A00081138000C0F3800001487800932720004B
:1023B000934178008381FB00A2F38000C719DE00FF
:1023C0008F80E9002000200094F3800004000100C9
:1023D00080007800E0BF9F00E40F50001900320039
:1023E00006003C00E20F50001000320013003C00D9
:1023F000E10F50001C003A0008003700E60F5000C3
:102400001500320011003500E70F500014003200B3
:10241000E80F500014003A00190037007FB8970009
:10242000C0F388007662A800140037007FB89700D8
:102430001080FB0090138800100037007622A8005F
:102440000E00370076A2A9000100370076A2A8008E
:102450007682A800090037007642A80007003700FE
:10246000723EEF0005003700E481570042A02000D3
:10247000D117200060BE2A00FB5C0700B1F3880082
:102480000080FA003400F9004F03BE004F02BE0086
:102490004F01BE004F00BE003600F90000400600AC
:1024A0003600F800809FBE00829FBE00849FBE0061
:1024B000869FBE00889FBE008A1F78003400F80007
:1024C00000002000A00188008AC0A900D47EAB00D3
:1024D0001F003200D35EE2000D003200D2DEEC00BD
:1024E000D2FEB700FF4F50000200340000CEB30010
:1024F000D2FEB700D2DEBF000000FB0001003B00AF
:102500000000EA0080407800E0C0B3008546070084
:102510008040EB00D35EE20004003A0011C0B3003B
:1025200010002000E45EE200010032000000EB0039
:102530008000FD00E4FEB7008000FD000004E00024
:10254000030032008040EB00E0C0B3007546070096
:10255000D4BEAB00D800320084C4BF006844600021
:102560003B003200D05EE2000B003A008040EB00FE
:1025700050C0B3006B4607008040EB0060C0B30062
:10258000684607008040EB0070C0B3006546070056
:1025900010C0B300D0FEB70011ED210091407800CB
:1025A000100020000104E000040032000100FB00E4
:1025B00072C0B300EA0F500007003C002200200068
:1025C000811F7800110009000200D8000001780086
:1025D000CF0078000241E80082C04000010078008E
:1025E000D1FEB70040C6B30080CF500012003400C7
:1025F000CF5EEC0080407800CFFEB70010C0B30083
:10260000D1FEB700E3CF500001003A00CF7EEF00CB
:10261000F8EC2100184478000804E00006003A00B5
:102620008840780070C0B3003E46070088407800BC
:1026300060C0B3003B46070011ED210091407800D7
:10264000CFDEBF0065404000364607009A003700E5
:10265000209380006212B400823E20000280B90004
:10266000A2F82000809FBE00110009004288D80017
:10267000800478004F00BE00D05EE20021003200EE
:1026800008007800D0FEB70050182000808F54005A
:102690000800360001C2B30050C0B3002146070055
:1026A00001C2B30060C0B3001E46070001C2B30000
:1026B0001200370080162000808F5400050036007D
:1026C00001C2B30050C0B3001646070001C2B300F8
:1026D0000700370040152000808F540009003600A5
:1026E00001C2B30050C0B3000E4607008840780016
:1026F00060C0B3000B4607008840780070C0B3008C
:10270000084607008040EB0050182000808F5400DE
:102710000400360011C0B30010002000E35EE200A8
:10272000010032000000EB008000FD00E3FEB70076
:102730008000FD000004E0000900320001C2B30087
:1027400050C0B300F745070001C2B30060C0B3003A
:10275000F445070001C2B30070C0B300F1450700A3
:102760008040EB0070E92F0000804400F70F50001C
:1027700004003E0011C0B30010002000E25EE20041
:10278000010032000000EB008000FD00E2FEB70017
:102790008000FD000004E0000900320001C2B30027
:1027A00050C0B300DF45070001C2B30060C0B300F2
:1027B000DC4507008040EB0070C0B300D94507003E
:1027C0008040EB00B0EA2F0000804400EE0F500084
:1027D00004003E0011C0B30010002000E15EE200E2
:1027E000010032000000EB008000FD00E1FEB700B8
:1027F0008000FD000004E0000900320001C2B300C7
:1028000050C0B300C74507008040EB0060C0B30074
:10281000C44507008040EB0070C0B300C14507000D
:102820008040EB0040152000808F540004003E00E3
:1028300011C0B30010002000E05EE2000100320091
:102840000000EB008000FD00E0FEB7008000FD000E
:102850000004E000060032008040EB0060C0B300DE
:10286000B04507008040EB0070C0B300AD450700E5
:1028700040152000808F54000F003E00D15EEC0018
:10288000D1FEB700E34F500003003A0001C2B3008D
:1028900050C0B300A345070010ED210051C0B300A4
:1028A00090CF1000040034008040EB0050C0B30013
:1028B0009C450700D17EEF00D43EAB008A00320079
:1028C000F3FA2000A1EC210044FB20001304E000F7
:1028D00008003200114178006340410080487800D0
:1028E00002C2B300824F50000300360082487800D5
:1028F000010037008048EB008301E8008100E80018
:10290000848F5100F1FF3A00CC5EE2000A003200F1
:1029100008022000C1EC21009140780008407800B6
:10292000804507000804E80040022000800F5400A2
:1029300019003200F7FF3700A1EC21009140780028
:102940000104E0000200320010C2B3007545070028
:10295000B1EC2100914078000104E0000200320057
:1029600020C2B3006F450700D1EC210091407800F0
:102970000104E0000200320000C2B3006945070014
:10298000E1EC2100914078000104E00002003200F7
:1029900030C2B30063450700CA5EE20003003A009C
:1029A00010002000CC5EE200010032000000EB00CD
:1029B000804078000004E000030032001000200096
:1029C000DF5EE200010032000000EB008000FD004D
:1029D000DFFEB7008000FD000004E00003003200CD
:1029E0008040EB0010C2B3004E450700CB5EE20012
:1029F00003003A0010002000CC5EE200010032002B
:102A00000000EB00804078000004E000030032008A
:102A100010002000DE5EE200010032000000EB004A
:102A20008000FD00DEFEB7008000FD000004E00035
:102A3000030032008040EB0020C2B300394507009C
:102A4000CD5EE20003003A0010002000CC5EE20000
:102A5000010032000000EB00804078000004E0003C
:102A60000300320010002000DD5EE20001003200B1
:102A70000000EB008000FD00DDFEB7008000FD00DF
:102A80000004E000030032008040EB0000C2B3000D
:102A900024450700CE5EE20003003A00100020004B
:102AA000CC5EE200010032000000EB0080407800C4
:102AB0000004E0000300320010002000DC5EE200B1
:102AC000010032000000EB008000FD00DCFEB700DA
:102AD0008000FD000004E000030032008040EB00B5
:102AE00030C2B3000F450700D41EAB003C003200DB
:102AF000AFCFBF000400320010C0B30011002000AF
:102B0000DB5EE200010032008000EB00DBFEB7007C
:102B10000104E0000200320020002000F151070013
:102B2000B0CFBF000400320010C0B300110020007D
:102B3000DA5EE200010032008000EB00DAFEB7004E
:102B40000104E0000200320020002000E5510700EF
:102B5000B1CFBF000400320010C0B300110020004C
:102B6000D95EE200010032008000EB00D9FEB70020
:102B70000104E0000200320030002000D9510700BB
:102B8000B2CFBF000400320010C0B300110020001B
:102B9000D85EE200010032008000EB00D8FEB700F2
:102BA0000104E0000200320020002000CD510700A7
:102BB000B3CFBF000400320010C0B30011002000EA
:102BC000D75EE200010032008000EB00D7FEB700C4
:102BD0000104E0000200320020002000C151070083
:102BE000D45EAB005300320041E1210043242100B8
:102BF00022E0210024E2210013007800910F100050
:102C000001003D00800878000000E0000300320071
:102C1000920F100001003400000978008180E80064
:102C20008381E8000281E800848F5000F2FF3A00BF
:102C3000A225210063E2210012007800910F10000C
:102C400001003D00800878008180E8000281E800F2
:102C5000838F5000F8FF3A008004EB0009057800EC
:102C600020E02100EA007800402421006A0078007A
:102C70000101500040E121006A007800810150000C
:102C80000200E00001003D000001EB000002200016
:102C90000090B900809FBE00110009004308D800D1
:102CA000000478004F00BE0080DF210069407800FA
:102CB000884078009B440700E28F540003003A00EC
:102CC000FA5DEC0088407800964407008904E8002B
:102CD0000A85E800E78F5400E1FF3A00A8252100AB
:102CE00029E22100FADF210019017800180078009C
:102CF0000000E00001003D000000EB0001022000A8
:102D00000180B900811F7800110009004208D80035
:102D1000CF007800804078003A4078008144070076
:102D20000884E8008984E800E0252100800F540031
:102D3000EDFF3A00D4DEAB00160032008040EB001D
:102D4000B85EE20004003A0011C0B3001000200099
:102D5000D65EE200010032000000EB008000FD00C2
:102D6000D6FEB7008000FD000004E0000300320042
:102D70008040EB00D0C1B3006A440700B85EE200B7
:102D800004003200B87EEF0001C2B300D0C1B3002E
:102D900064440700D51EAB004B003200B0938000A6
:102DA000F40F500042003C00A193800090938000FB
:102DB000422E070022002000110009000200D80066
:102DC0008000FD00067D200006804000F3F9200011
:102DD000C9012000830F5000200036000577210034
:102DE00005804000B9012000830F50001B00360011
:102DF0000471220004804000A9012000830F5000CC
:102E000016003600006B230000814000990120006D
:102E1000830F51001100360089012000F0D52600F3
:102E2000800F51000D003E0006805000EC844400ED
:102E3000830F500009003600058050008904E80027
:102E4000830F50000500360004805000F901200077
:102E5000830F5000010036008084EB00B0938000A7
:102E60000000E00001003D000000EA00800040009A
:102E7000800220000104500001003B000004EB0030
:102E80000900E0000800350040F680000000E00086
:102E9000020035008040EB002244070088407800A3
:102EA000094078001F44070049F6880006003700F3
:102EB00040F680000000E000020035008040EB009A
:102EC00018440700C8BEEF00D53EAB002400320016
:102ED000C75EEC00C7FEB700EA4F500020003A0082
:102EE000C77EEF00C193800050092000808F500002
:102EF00005003C008040EB0060C2B30009440700BD
:102F000001C2B3001400370080112000808F5000F0
:102F10000500340001C2B3006E40400001440700C8
:102F20008040EB000C003700A8F62F00088440001A
:102F30004544DD0022082000110009000204D800E9
:102F4000000478008840780060C2B300F5430700B1
:102F500001C2B30088C0500070C2B300F143070043
:102F6000D55EAB000100320067230700D57EAB00C1
:102F700001003200073D07003400F9004F057800DA
:102F80004F04BE004F03BE004F02BE004F01BE0003
:102F90004F00BE003600F900004006006D610000E1
:102FA000746800002E720000616E00006400000072
:102FB000666900006C6C0000206100007272000005
:102FC000617900002077000069740000682000002B
:102FD000726100006E6400006F6D000020760000DA
:102FE000616C0000756500007300000064650000FE
:102FF0007374000000000000CE970000D897000016
:10300000FFFF0000F6970000000000000000000035
:103010006D610000746800002E6E00007A7300007D
:10302000657100000077000072690000746500009F
:10303000207400006F2000006465000073740000BD
:103040002074000068650000206D000069640000C5
:10305000646C000065200000696E0000646500007B
:10306000782000006F660000207400006865000092
:10307000206C00006172000067650000737400003E
:103080002073000065710000756500006E6300002C
:10309000652000006F660000206E00006F6E00006B
:1030A0002D7A0000657200006F200000656C000042
:1030B000656D0000656E00007473000020660000FE
:1030C000726F00006D20000073720000632C00001E
:1030D000202D00003120000069660000206E0000F5
:1030E0006F740000206600006F7500006E640000C1
:1030F000206F00007220000069660000207300004D
:103100006D6100006C6C00006572000020740000AE
:10311000686100006E2000006D6900006E4C0000C8
:10312000656E0000677400006800000073720000A4
:10313000630000006D6900006E4C0000656E0000C9
:1031400067740000680000000898000013980000F1
:1031500001000000F6970000FFFF000096980000B5
:10316000010000009A98000000000000000000002C
:103170006D610000746800002E7300007172000021
:103180007400000070650000726600006F7200003D
:103190006D7300002064000065730000742000005F
:1031A0003D20000073710000727400002878000058
:1031B00029200000656C0000656D0000656E000050
:1031C0007420000062790000206500006C6500003A
:1031D0006D6500006E7400000078000000000000C3
:1031E000B8980000C2980000FFFF0000F6970000AA
:1031F000FFFF0000ED98000000000000000000004C
:103200006D610000746800002E7200006F74000091
:1032100032000000726F00007461000074650000ED
:1032200073200000762000006F660000206100001F
:103230006E6700006C6500002061000020740000D3
:103240006F200000646500007374000000760000C9
:103250000061000000000000009900000A990000D1
:1032600002000000F697000002000000279900000D
:10327000010000002999000000000000000000008B
:103280006D610000746800002E6300006F73000021
:103290000070000065720000666F0000726D000033
:1032A000732000006465000073740000203D00007E
:1032B000206300006F7300002878000029200000C0
:1032C000656C0000656D0000656E000074200000F4
:1032D00062790000206500006C6500006D650000EB
:1032E0006E74000000000000409900004999000041
:1032F000FFFF0000F6970000FFFF0000ED980000C0
:1033000000000000000000006D6100007468000013
:103310002E730000696E00000070000065720000EE
:10332000666F0000726D000073200000646500008D
:1033300073740000203D000020730000696E0000DF
:103340002878000029200000656C0000656D0000F1
:10335000656E0000742000006279000020650000A6
:103360006C6500006D6500006E74000000000000D8
:10337000849900008D990000FFFF0000F69700007F
:10338000FFFF0000ED9800000000000000000000BA
:103390006D610000746800002E610000746100001F
:1033A0006E3200000070000065720000666F000061
:1033B000726D0000732000006465000073740000EB
:1033C000203D000020610000746100006E320000AA
:1033D000287900002C78000029200000656C00008E
:1033E000656D0000656E00007420000062790000C9
:1033F000206500006C6500006D6500006E740000C3
:103400000079000000000000C8990000D399000076
:10341000FFFF0000F6970000FFFF0000019A000088
:10342000FFFF0000ED980000000000000000000019
:103430006D610000746800002E6D0000756C000066
:10344000646900007600000070650000726600008C
:103450006F7200006D73000020640000657300004F
:10346000742000003D200000286100002A62000056
:10347000292F000063200000696E00002033000047
:1034800032200000626900007473000020650000B3
:103490006C6500006D6500006E7400002062000025
:1034A00079200000656C0000656D0000656E00000D
:1034B000740000006200000063000000189A000021
:1034C000249A0000FFFF0000F6970000FFFF0000B5
:1034D00029990000FFFF00005A9A0000FFFF00003A
:1034E0005C9A000000000000000000006D61000018
:1034F000746800002E7300006F72000074000000FA
:10350000736F00007274000020610000727200008E
:1035100061790000206900006E200000706C0000DE
:1035200061630000650000006172000072610000CC
:1035300079000000769A0000809A0000FFFF0000EA
:10354000949A000000000000000000006D6100007F
:10355000746800002E61000072670000626F000056
:10356000756E000064730000006700006574000061
:103570002074000068650000206900006E6400008F
:10358000696300006573000020280000617200007C
:10359000676D0000696E00002C2000006172000061
:1035A000676D000061780000292000006F66000050
:1035B0002074000068650000206C0000696D000048
:1035C0006974000020760000616C000075650000E1
:1035D000732000006F66000020730000726300001B
:1035E00000610000726700006D6900006E0000005D
:1035F00061720000676D000061780000000000004B
:10360000A69A0000B59A0000FFFF000096980000FF
:1036100001000000F19A000001000000F89A00008B
:1036200000000000000000006D61000074680000F0
:103630002E730000746100007400000070650000CB
:10364000726600006F7200006D730000207300004E
:103650007461000074690000737400006963000005
:10366000732000006F6E0000207300007263000082
:10367000006D0000696E0000006D000061780000C0
:10368000006D0000656100006E000000149B0000EA
:103690001E9B0000FFFF0000969800000100000044
:1036A000399B0000010000003D9B0000010000006C
:1036B000419B000000000000000000006D61000060
:1036C000746800002E6400006F7400000077000032
:1036D00072690000746500007320000074680000C7
:1036E00065200000646F000074200000707200000C
:1036F0006F64000075630000742000006F660000B6
:10370000207300007263000031200000616E000031
:103710006420000073720000633200002074000017
:103720006F20000064650000737400002C2000000E
:1037300061660000746500007220000061200000D6
:103740007368000069660000740000007372000076
:10375000633100000073000072630000320000005B
:103760007368000069660000740000005E9B000042
:10377000679B000001000000F6970000FFFF0000BB
:10378000A69B0000FFFF0000AB9B000001000000B3
:10379000B09B000000000000000000006D61000010
:1037A000746800002E6D0000617800000077000052
:1037B00072690000746500007320000074680000E6
:1037C000652000006D610000786900006D750000E3
:1037D0006D2000006F66000020730000726300001F
:1037E00031200000616E0000642000007372000050
:1037F00063320000207400006F2000006465000048
:10380000737400002C200000656C0000656D0000E2
:10381000656E0000742000006279000020650000E1
:103820006C6500006D6500006E7400000000000013
:10383000CE9B0000D79B0000FFFF0000F697000022
:10384000FFFF0000A69B0000FFFF0000AB9B0000F5
:1038500000000000000000006D61000074680000BE
:103860002E6D0000696E0000007700007269000094
:10387000746500007320000074680000652000007B
:103880006D6900006E6900006D7500006D2000001C
:103890006F6600002073000072630000312000009A
:1038A000616E00006420000073720000633200004B
:1038B000207400006F200000646500007374000035
:1038C0002C200000656C0000656D0000656E000036
:1038D0007420000062790000206500006C65000023
:1038E0006D6500006E740000000000002C9C00005C
:1038F000359C0000FFFF0000F6970000FFFF00006E
:10390000A69B0000FFFF0000AB9B00000000000032
:10391000000000006D610000746800002E6400006B
:1039200069760000006400006976000069640000A8
:1039300065730000207300007263000031200000F6
:1039400062790000207300007263000032200000E2
:10395000746F00002064000065730000742C000088
:10396000206500006C6500006D6500006E7400004D
:103970002062000079200000656C0000656D000089
:10398000656E0000740000008A9C0000939C00009B
:10399000FFFF0000F6970000FFFF0000A69B00005D
:1039A000FFFF0000AB9B00000000000000000000D3
:1039B0006D610000746800002E6D0000756C0000E1
:1039C000006D0000756C000074690000706C0000F0
:1039D000696500007320000073720000633100000D
:1039E000206100006E64000020730000726300001C
:1039F00032200000746F0000206400006573000036
:103A0000742C0000206500006C6500006D650000EE
:103A10006E7400002062000079200000656C0000D8
:103A2000656D0000656E000074000000D89C000009
:103A3000E19C0000FFFF0000F6970000FFFF000080
:103A4000A69B0000FFFF0000AB9B000000000000F1
:103A5000000000006D610000746800002E7300001B
:103A6000756200000073000075620000737400004E
:103A70007261000063740000732000007372000024
:103A80006332000020660000726F00006D200000AD
:103A90007372000063310000207400006F2000008A
:103AA00064650000737400002C200000656C000049
:103AB000656D0000656E00007420000062790000F2
:103AC000206500006C6500006D6500006E740000EC
:103AD000000000002A9D0000339D0000FFFF000051
:103AE000F6970000FFFF0000A69B0000FFFF00000C
:103AF000AB9B000000000000000000006D610000B2
:103B0000746800002E610000646400000061000021
:103B100064640000732000007372000063310000D1
:103B2000206100006E6400002073000072630000DA
:103B300032200000746F00002064000065730000F4
:103B4000742C0000206500006C6500006D650000AD
:103B50006E7400002062000079200000656C000097
:103B6000656D0000656E0000740000007E9D000021
:103B7000879D0000FFFF0000F6970000FFFF000098
:103B8000A69B0000FFFF0000AB9B000000000000B0
:103B9000000000006D610000746800002E610000EC
:103BA0006464000073630000616C000061720000D7
:103BB0000061000064640000207300006361000085
:103BC0006C61000072200000746F0000206500002E
:103BD0006163000068200000656C0000656D0000F6
:103BE000656E0000742000006F6600002073000006
:103BF00072630000206100006E640000207300000A
:103C0000746F000072650000207200006573000090
:103C1000756C000074200000746F000020640000C8
:103C2000657300007400000073630000616C0000A5
:103C30006172000000000000CA9D0000D99D0000D4
:103C4000FFFF0000F6970000FFFF000096980000BD
:103C500001000000149E00000000000000000000B1
:103C60006D610000746800002E660000696C000041
:103C70006C000000666900006C6C0000732000009E
:103C80006465000073740000207700006974000010
:103C900068200000636F00006E7300007461000014
:103CA0006E74000020760000616C000075650000F5
:103CB00000760000616C00007565000000000000E7
:103CC000309E00003A9E0000FFFF0000F6970000C3
:103CD00001000000599E00000000000000000000EC
:103CE0006D610000746800002E6300006F700000BA
:103CF00079000000636F00007069000065730000C8
:103D00002073000072630000207400006F20000028
:103D10006465000073740000206500006C6500009D
:103D20006D6500006E7400002062000079200000C4
:103D3000656C0000656D0000656E00007400000099
:103D4000709E00007A9E0000FFFF0000F6970000C2
:103D5000FFFF000096980000000000000000000037
:103D6000000000009301000024030000B7040000DD
:103D700048060000DA0700006B090000FC0A00009A
:103D80008C0C00001C0E0000AB0F00003B1100006B
:103D9000C812000056140000E31500006E17000062
:103DA000F9180000831A00000C1C0000941D00008C
:103DB0001A1F0000A020000024220000A7230000FA
:103DC00029250000A826000027280000A4290000BB
:103DD000202B0000992C0000122E0000872F0000DD
:103DE000FC3000006F320000DF3300004E35000071
:103DF000BA360000253800008D390000F33A000083
:103E0000573C0000B93D0000173F0000744000001F
:103E1000CE410000264300007B440000CD45000059
:103E20001D4700006A480000B4490000FC4A000039
:103E3000404C0000824D0000C04E0000FC4F0000CE
:103E400034510000695200009B530000CA54000026
:103E5000F65500001E57000043580000645900004A
:103E6000835A00009D5B0000B45C0000C85D000048
:103E7000D75E0000E45F0000EC600000F16100002C
:103E8000F2620000EF630000E9640000DE650000FC
:103E9000D0660000BD670000A76800008C690000C4
:103EA0006E6A00004B6B0000246C0000F96C00008F
:103EB000CA6D0000976E00005F6F00002370000065
:103EC000E37000009E71000055720000087300004E
:103ED000B67300006074000005750000A575000051
:103EE00042760000D97600006C770000FB77000076
:103EF00084780000097900008A790000067A0000C1
:103F00007D7A0000EF7A00005D7B0000C67B000038
:103F10002A7C0000897C0000E47C0000397D0000E0
:103F20008A7D0000D77D00001D7E0000607E0000BD
:103F30009D7E0000D67E0000097F0000397F0000D2
:103F4000627F0000877F0000A77F0000C27F000023
:103F5000D87F0000EA7F0000F67F0000FE7F0000AF
:103F6000FF7F00008C020000DF0200003003000031
:103F700080030000D103000022040000730400004D
:103F8000C204000014050000B30500005406000040
:103F9000F10600008F0700002D080000CA0800008D
:103FA00063090000FC090000340B00005C0C0000F9
:103FB000820D0000A40E0000BD0F0000D310000011
:103FC000E2110000E7120000EF140000CC16000020
:103FD00092180000401A0000D61B0000531D00007C
:103FE000B51E00000B200000792200008D24000087
:103FF0006F2600001428000090290000E02A00002D
:10400000112C0000252D0000052F00008930000034
:10401000D3310000EC320000DD330000AE3400008C
:10402000673500000D36000020370000FB37000028
:10403000B23800004A390000CC3900003B3A000099
:104040009B3A0000F33A0000833B0000F43B000081
:10405000513C00009F3C0000E13C00001A3D000084
:104060004B3D0000783D0000C03D0000F93D0000E0
:10407000283E00004F3E0000703E00008D3E0000D4
:10408000A53E0000BC3E0000E03E0000FD3E0000FA
:10409000143F0000283F0000383F0000473F000069
:1040A000533F00005E3F0000703F00007F3F000074
:1040B0008A3F0000943F00009C3F0000A43F0000A6
:1040C000AA3F0000AF3F0000B83F0000C03F000023
:1040D000C53F0000CB3F0000CE3F0000D23F0000B4
:1040E000D53F0000D83F0000DC3F0000E03F00006B
:1040F000E33F0000E53F0000E83F0000E93F00002B
:10410000EB3F0000EC3F0000EE3F0000F13F0000FD
:10411000F13F0000F33F0000F43F0000F53F0000D6
:10412000F53F0000F73F0000F73F0000F93F0000B7
:10413000F83F0000FA3F0000FA3F0000FA3F00009D
:10414000FB3F0000FB3F0000FC3F0000FC3F000085
:10415000FC3F0000FE3F0000FD3F0000FD3F00006F
:10416000FD3F0000FE3F0000FE3F0000FE3F00005C
:10417000FE3F0000FE3F0000FE3F00000040000048
:10418000FF3F0000FF3F0000FF3F0000FF3F000037
:10419000FF3F0000FF3F0000FF3F0000FF3F000027
:1041A000FF3F0000FF3F0000FF3F00000040000015
:1041B00000400000004000000040000000400000FF
:1041C00000400000004000000040000000400000EF
:1041D00000400000004000000040000000400000DF
:1041E000004000000040000074680000796D00008D
:1041F000696F00002D490000490000005F69000060
:104200006400000065760000656E0000742E0000FA
:10421000736F0000757200006365000000650000A8
:10422000766500006E7400002E6100007267000069
:10423000730000005F660000777600006572000082
:10424000736900006F6E0000005F00007072000074
:104250006F64000075630000744900006400000092
:1042600062750000747400006F6E0000732E000011
:104270005F7200006177000000620000757400004A
:10428000746F00006E2E000062610000636B00001E
:104290007761000072640000006200007574000025
:1042A000746F00006E2E00006C65000066740000E4
:1042B0000062000075740000746F00006E2E000034
:1042C000636500006E74000065720000006200000B
:1042D00075740000746F00006E2E0000666F0000A1
:1042E00072770000617200006400000062750000D7
:1042F000747400006F6E00002E7200006967000089
:10430000687400000062000075740000746F0000A3
:104310006E7300002E5F00006D650000616E00008E
:104320000062000075740000746F00006E7300007E
:104330002E5F00006E6F00006973000065000000D2
:10434000707200006F7800002E6800006F7200002D
:10435000697A00006F6E0000746100006C0000005C
:10436000707200006F7800002E670000726F00000E
:10437000756E0000642E0000616D0000626900002F
:10438000616E000074000000707200006F78000021
:104390002E670000726F0000756E0000642E000032
:1043A00072650000666C00006563000074650000C3
:1043B00064000000707200006F7800002E6700003B
:1043C000726F0000756E0000642E000064650000CE
:1043D0006C740000610000006D6F0000746F0000DD
:1043E000722E00006C650000667400002E740000E0
:1043F0006172000067650000740000006D6F0000CE
:10440000746F0000722E000072690000676800007F
:10441000742E000074610000726700006574000073
:10442000005F00007662000061740000005F000021
:10443000696D00006F740000006D00006F74000073
:104440006F7200002E6C000065660000742E000084
:104450007370000065650000640000006D6F00006F
:10446000746F0000722E000072690000676800001F
:10447000742E000073700000656500006400000089
:104480006D6F0000746F0000722E00006C650000FC
:10449000667400002E700000776D0000006D000053
:1044A0006F7400006F7200002E72000069670000D8
:1044B000687400002E700000776D0000006100003D
:1044C0006363000000740000656D0000706500000B
:1044D00072610000747500007265000000720000D7
:1044E000633500002E610000646400007265000006
:1044F0007373000000720000633500002E6300003B
:104500006F6D00006D6100006E640000006D0000C2
:10451000696300002E6900006E740000656E000083
:104520007369000074790000006D00006963000089
:104530002E7400006872000065730000686F000050
:104540006C640000006D0000696300002E5F0000D5
:104550006D650000616E000000740000696D000070
:10456000657200002E70000065720000696F000027
:104570006400000061630000632E00005F740000AF
:104580006170000000000000F4A0000001000000C5
:10459000FEA000000100000002A1000020000000B9
:1045A0000FA10000020000001AA10000010000009D
:1045B00025A100000500000030A10000010000005E
:1045C0003DA10000010000004DA10000010000001D
:1045D00059A100000100000067A1000001000000D7
:1045E00076A100000500000083A100000500000086
:1045F00091A1000007000000A0A10000020000003F
:10460000B0A1000002000000C4A1000002000000F0
:10461000DAA1000001000000ECA100000100000090
:10462000FEA100000200000011A200000200000034
:1046300017A20000010000001DA200000100000000
:104640002EA200000100000040A2000001000000B6
:104650004FA20000030000005FA200000100000064
:1046600063A20000010000006FA200000100000032
:104670007BA200000100000087A2000001000000F2
:1046800095A2000001000000A3A2000002000000AB
:10469000ADA2000001000000BAA20000000000006E
:1046A00000000000DE000000AD000000CA000000B5
:1046B000FE000000BE000000EF000000040000004B
:1046C000020000005F730000797300007465000051
:1046D0006D2E00007365000074740000696E0000A8
:1046E000677300002E6600006C61000073680000B4
:1046F000005700007269000074650000207400001B
:104700006865000020730000657400007469000093
:104710006E67000073200000696E0000746F000077
:10472000206600006C61000073680000005F0000FC
:104730007379000073740000656D00002E73000033
:1047400065740000746900006E670000732E00003D
:104750007772000069740000650000005772000065
:10476000697400006520000061200000736500008E
:1047700074740000696E000067000000616400004E
:104780006472000065730000730000007661000031
:104790006C750000650000005F7300007973000015
:1047A000746500006D2E00007365000074740000D5
:1047B000696E0000677300002E72000065610000E2
:1047C0006400000052650000616400002061000088
:1047D0002073000065740000746900006E670000BB
:1047E000005F00007379000073740000656D0000C5
:1047F0002E720000656200006F6F00007400000000
:1048000052650000626F00006F74000020740000A9
:1048100068650000206D000069630000726F000091
:10482000636F00006E740000726F00006C6C00001B
:104830006572000000420000616300006B770000B9
:104840006172000064200000627500007474000052
:104850006F6E00002073000074610000747500002A
:104860007320000063680000616E0000676500004F
:10487000640000004C6500006674000020620000C7
:1048800075740000746F00006E20000073740000E7
:10489000617400007573000020630000686100000F
:1048A0006E6700006564000000430000656E000054
:1048B00074650000722000006275000074740000CE
:1048C0006F6E0000207300007461000074750000BA
:1048D0007320000063680000616E000067650000DF
:1048E00064000000466F00007277000061720000F3
:1048F0006420000062750000747400006F6E000098
:1049000020730000746100007475000073200000C3
:1049100063680000616E00006765000064000000CD
:104920005269000067680000742000006275000092
:10493000747400006F6E000020730000746100004A
:10494000747500007320000063680000616E000051
:104950006765000064000000627500007474000068
:104960006F6E000073000000427500007474000058
:104970006F6E000073200000766100006C7500000F
:104980006573000020750000706400006174000011
:104990006564000000700000726F00007800000085
:1049A000507200006F780000696D000069740000AB
:1049B00079200000766100006C75000065730000CE
:1049C00020750000706400006174000065640000E0
:1049D00000740000617000000041000020740000BD
:1049E0006170000020690000732000006465000011
:1049F00074650000637400006564000000410000FD
:104A000063630000656C0000657200006F6D00005C
:104A1000657400006572000020760000616C000083
:104A2000756500007320000075700000646100006F
:104A300074650000640000006D6900006300000000
:104A4000466900007265000064200000776800007D
:104A5000656E0000206D000069630000726F000049
:104A6000706800006F6E000065200000696E000035
:104A7000746500006E730000697400007920000006
:104A80006973000020610000626F0000766500001D
:104A9000207400006872000065730000686F0000F9
:104AA0006C640000007300006F7500006E6400000D
:104AB0002E660000696E00006973000068650000E2
:104AC0006400000046690000726500006420000078
:104AD00077680000656E00002074000068650000C3
:104AE000207000006C6100007962000061630000CA
:104AF0006B2000006F660000206100002075000040
:104B00007365000072200000696E00006974000087
:104B1000696100007465000064200000736F00008C
:104B2000756E0000642000006973000020660000BC
:104B3000696E000069730000686500006400000091
:104B4000546500006D700000657200006174000023
:104B50007572000065200000766100006C75000031
:104B6000652000007570000064610000746500003D
:104B70006400000072630000350000005243000032
:104B8000352000006D650000737300006167000050
:104B90006520000072650000636500006976000012
:104BA00065640000006D00006F7400006F7200000B
:104BB000004D00006F7400006F7200002074000050
:104BC000696D00006572000000740000696D0000EE
:104BD0006572000030000000546900006D6500003F
:104BE0007220000030000000746900006D65000054
:104BF0007231000000540000696D00006572000011
:104C000020310000000000003DA100001BA40000B6
:104C10004DA100003AA4000059A1000055A40000D5
:104C200067A1000072A4000076A1000090A400001B
:104C3000ACA40000B4A40000CBA40000D0A40000E9
:104C4000E9A40000EDA400005FA20000FFA40000A2
:104C50001CA5000020A5000053A5000062A50000CF
:104C600063A20000A0A50000BAA50000BEA5000038
:104C7000D3A50000D9A50000E5A50000ECA5000023
:104C8000F4A50000FBA500000000000000000000EB
:104C9000416400006472000065730000732000002E
:104CA0006F750000742000006F6600002073000024
:104CB00065740000746900006E67000073000000F6
:104CC000536C000065650000702000006D6F0000EF
:104CD00064650000206E00006F7400002073000007
:104CE00075700000706F0000727400006564000051
:104CF00000450000727200006F7200003A20000050
:104D00006D6900006E2000003D3D00002030000075
:104D10007846000046460000464600004646000031
:104D2000462000002100000045720000726F000064
:104D3000723A0000205500006E610000626C0000B5
:104D400065200000746F0000206600006C610000A8
:104D50007368000020620000797400006563000041
:104D60006F64000065200000283100002920000049
:104D70002100000045720000726F0000723A0000CE
:104D8000205500006E610000626C0000652000008C
:104D9000746F0000206600006C6100007368000002
:104DA0002062000079740000656300006F640000F9
:104DB00065200000283200002920000021000000AA
:104DC00045720000726F0000723A0000205500002A
:104DD0006E610000626C000065200000746F0000CE
:104DE000206600006C610000736800002062000013
:104DF00079740000656300006F64000065200000A6
:104E0000283300002920000021000000466C00002B
:104E100061730000686900006E670000204F0000A9
:104E20004B000000736F0000756E0000642E0000E0
:104E30007761000076650000005300006574000093
:104E40002074000068650000207000007269000096
:104E50006D6100007279000020770000617600002B
:104E6000652000006F660000207400006865000087
:104E7000207400006F6E0000652000006765000070
:104E80006E65000072610000746F00007200000027
:104E90007761000076650000007300006F75000008
:104EA0006E6400002E660000726500007100000054
:104EB000506C0000617900002066000072650000FF
:104EC00071750000656E0000637900000048000005
:104ED0007A00000064730000006C0000656400004C
:104EE000732E0000746500006D7000006572000094
:104EF00061740000757200006500000053650000D9
:104F0000742000006E740000632000006C650000D7
:104F1000640000007265000064000000626C000024
:104F200075650000006C000065640000732E0000D1
:104F3000736F0000756E0000640000005365000090
:104F400074200000736F0000756E00006420000084
:104F50006C650000640000006C65000064000000E7
:104F60006C650000647300002E7200006300000096
:104F7000536500007420000072630000206C000084
:104F800065640000006C000065640000732E000082
:104F9000707200006F7800002E7600000053000051
:104FA00065740000207600006572000074690000DE
:104FB000636100006C200000707200006F780000D8
:104FC000696D000069740000792000006C650000C4
:104FD00064730000006C0000656400002030000075
:104FE000006C00006564000020310000006C0000CF
:104FF00065640000732E0000707200006F7800007E
:105000002E68000000530000657400002068000056
:105010006F720000697A00006F6E0000746100001A
:105020006C200000707200006F780000696D000055
:1050300069740000792000006C6500006473000052
:10504000006C00006564000020320000006C00006D
:105050006564000020330000006C000065640000FF
:1050600020340000006C0000656400002035000062
:10507000006C00006564000020360000006C000039
:105080006564000020370000006C000065640000CB
:10509000732E000062750000747400006F6E0000D3
:1050A000730000005365000074200000627500006A
:1050B000747400006F6E0000732000006C650000C7
:1050C00064730000006C000065640000732E000033
:1050D000626F0000747400006F6D00002E6C0000A1
:1050E0006566000074000000536500007420000035
:1050F0005247000042200000626F0000746F000001
:105100006D2000006C65000066740000206C0000DB
:10511000656400000067000072650000656E0000B5
:10512000006C000065640000732E0000626F0000D8
:10513000747400006F6D00002E720000696700003B
:1051400068740000005300006574000020520000E5
:1051500047420000206200006F7400006F6D000085
:10516000207200006967000068740000206C000075
:1051700065640000006C000065640000732E000090
:10518000746F000070000000536500007420000080
:105190005247000042200000746F000070200000A1
:1051A0006C650000640000006C6500006473000022
:1051B0002E63000069720000636C0000650000004F
:1051C00053650000742000006369000072630000F2
:1051D000756C00006172000020720000696E0000B2
:1051E000672000006C65000064730000007300001D
:1051F0006F7500006E6400002E730000797300006C
:10520000746500006D0000005374000061720000BE
:1052100074200000706C0000617900006261000081
:10522000636B0000206F00006620000073790000AF
:1052300073740000656D0000207300006F7500003E
:105240006E640000204E0000004E0000007300005D
:105250006F7500006E6400002E7200006570000023
:105260006C6100007900000053740000617200005E
:1052700074200000706C0000617900006261000021
:10528000636B0000206F000066200000724E00007B
:105290002E77000061760000007300006F7500003B
:1052A0006E6400002E7000006C6100007900000048
:1052B000537400006172000074200000706C0000E4
:1052C0006179000062610000636B0000206F0000E4
:1052D00066200000704E00002E770000617600000E
:1052E000007300006F7500006E6400002E720000F5
:1052F000656300006F7200006400000053740000DA
:10530000617200007420000072650000636F00008D
:1053100072640000696E0000672000006F66000084
:10532000207200004E2E0000776100007600000021
:105330005F6C000065640000732E00007365000060
:1053400074000000536500007420000074680000C1
:10535000652000006C6500006400000062720000BF
:1053600069670000687400006E65000073730000D8
:1053700000700000000000000000000000000000BD
:1053800000000000000000000000000072000000AB
:10539000000000000000000000000000000000000D
:1053A000000000000072000000000000000000008B
:1053B00000000000000000000000000000000000ED
:1053C000730000000000000000000000000000006A
:1053D00000000000000000000045000072720000A4
:1053E0006F7200003A200000736100006D700000D1
:1053F0006C650000732000006D7500007374000080
:105400002062000065200000696E0000205B000043
:105410002D310000323800002C31000032370000FE
:105420005D200000726100006E67000065000000F2
:1054300030110000070000007C150000070000008C
:10544000C819000007000000000000000000000074
:1054500030110000070000007C150000070000006C
:105460000000000000000000C81900000500000056
:10547000BE0A000004000000000000000000000060
:105480009C27000002000000AB2200000100000089
:105490009D1C000002000000FB180000020000003C
:1054A0002D32000001000000322D0000010000003C
:1054B0004628000002000000E8260000010000006D
:1054C000BF22000002000000FB18000002000000E4
:1054D000FF32000001000000C620000001000000B3
:1054E000762F0000020000002C2E000001000000BA
:1054F000CE2C000001000000FD3900000200000079
:105500000000000000000000E40C000007000000A4
:10551000301100000D000000C81900000700000055
:1055200000000000000000004C0400000700000024
:1055300098080000070000000000000000000000C4
:10554000781E00000D000000001900000700000098
:10555000EC130000070000003011000007000000FD
:10556000480D0000070000000000000000000000DF
:10557000480D00000D000000301100000700000081
:10558000EC130000070000000019000007000000F5
:10559000781E00000700000000000000000000006E
:1055A000733000002E770000617600000073000069
:1055B000322E000077610000760000007333000097
:1055C0002E7700006176000000730000342E00008A
:1055D0007761000076000000733500002E77000030
:1055E0006176000000730000362E00007761000035
:1055F00076000000733700002E770000617600000F
:1056000000000000809A0000904100008E410000E0
:105610008F800000454500004549000049490000D1
:105620008E8F000090920000924F0000994F000072
:1056300055550000599900009A9B00009C9D000060
:105640009E9F0000414900004F550000A5A50000A5
:10565000A6A70000A8A90000AAAB0000AC2100008A
:10566000AEAF0000B0B10000B2B30000B4B50000AE
:10567000B6B70000B8B90000BABB0000BCBD00005E
:10568000BEBF0000C0C10000C2C30000C4C500000E
:10569000C6C70000C8C90000CACB0000CCCD0000BE
:1056A000CECF0000D0D10000D2D30000D4D500006E
:1056B000D6D70000D8D90000DADB0000DCDD00001E
:1056C000DEDF0000E0E10000E2E30000E4E50000CE
:1056D000E6E70000E8E90000EAEB0000ECED00007E
:1056E000EEEF0000F0F10000F2F30000F4F500002E
:1056F000F6F70000F8F90000FAFB0000FCFD0000DE
:10570000FEFF0000222A00002B2C00003A3B000084
:105710003C3D00003E3F00005B5D00007C7F0000E0
:10572000000000005A3A00005C6D00006F6C000041
:105730006F6C0000655C000069320000635C000073
:105740002F690000326300005F7000007269000082
:10575000762E0000680000005A3A00005C6D0000E0
:105760006F6C00006F6C0000655C00006932000027
:10577000635C00006D6100007374000065720000DE
:105780005F700000726F0000746F0000636F0000B4
:105790006C2E0000630000005A3A00005C6D0000AF
:1057A0006F6C00006F6C0000655C000069320000E7
:1057B000635C00002F690000326300005F7000002E
:1057C00072690000762E0000680000005A3A00005E
:1057D0005C6D00006F6C00006F6C0000655C000089
:1057E00069320000635C00006D61000073740000AA
:1057F000657200002E6300000000000052490000A6
:105800004646000000000000000000005741000074
:1058100056450000666D0000742000001000000076
:10582000000000000100000001000000841E0000D4
:1058300000000000841E00000000000001000000C5
:1058400008000000646100007461000000000000B6
:10585000000000005A3A00005C6D00006F6C000010
:105860006F6C0000655C0000746900006D650000ED
:10587000725C0000746900006D650000722E00000B
:1058800063000000010000000000000008000000AC
:1058900000000000400000000000000000010000C7
:1058A000000000005F4C00004F470000445500001E
:1058B0004D5000002E23000040210000005F00003A
:1058C00054450000535400004D4F0000442E00008A
:1058D0002340000021000000564D0000434F00000F
:1058E000444500002E410000424F0000000000002F
:1058F0005A3A00005C6D00006F6C00006F6C000095
:10590000655C000069320000635C00002F690000E4
:10591000326300005F70000072690000762E0000A4
:10592000680000005A3A00005C6D00006F6C0000D7
:105930006F6C0000655C0000666C00006173000025
:10594000685C0000666C000061730000682E000057
:10595000630000005F7000006F7700006572000058
:105960006F66000066000000506F00007765000061
:10597000726F000066660000000000006D6D0000A0
:105980006137000036360000302E00006300000052
:105990000000000000000000000000000000000007
:1059A0009EC0A9008EA4EF008AA4EF00AA24EF00F5
:1059B000AC24EF00AE24EF0020002000302588004A
:1059C000A824EF008644A900F00920008024880064
:1059D000602488008804A800010021004808DE0037
:1059E000C02488000000EB008018EB008018EB005A
:1059F0000000E800EC0F5000FBFF3A009424A800E0
:105A00009624EF0094A4A9009424A900810020000A
:105A100007003700512488005C70EF006270EF00CF
:105A200063D0BF006370EF0064D0BF006470EF000C
:105A30008AC4BF000038A300F6FF3A00100020001F
:105A4000C0838800D08388007C30EF007E30EF0078
:105A50008430EF000000EB0004052100A2042100C7
:105A600080007800E506210023072100001AEB00E2
:105A70000019EB0001F07A0001F079000000E80065
:105A8000E30F5000F9FF3A00800021008082880077
:105A9000D0002000502588000003210010808800DD
:105AA00080C0B30000F0B70040C8B30001F0B700F9
:105AB0004270EF004030EF00000006007810E20076
:105AC00022003A0014002000C4838800D1838000A3
:105AD0000100E0001D003A00D483880058D0BF00C8
:105AE000E24F500006003A008082800001487800B2
:105AF00081CCB30080828000114098000000060035
:105B000058D0BF00E14F500010003A0001848800D7
:105B100083C0B30030828000034878003182800067
:105B2000020321009200980040C8B3009040980002
:105B3000048488004082800003487800418280000D
:105B40009200980000C8B300904098000000060042
:105B5000F082800083C0B300E70F50000A003E00CF
:105B6000F08280008041780010C0B3005650E200FF
:105B70000400320056D0BF00E14F500002003A004E
:105B800020C0B30056F0B7000380FB005E30B500C4
:105B900080828000034878008003210040838800D1
:105BA0005CD0BF000008A30002003200034178006F
:105BB00012003700034178008041EB0006003700F7
:105BC00040838000D1828000315878004083880073
:105BD000D18288000241E900834F5100F8FF3A006A
:105BE0000000060040838000D18280003158780098
:105BF00040838800D18288000241E9000204E0006D
:105C0000F8FF3A00000006007C30EF007E30EF0025
:105C100058D0BF00E24F500009003A0081C0B300E5
:105C2000408280000148780041828000800321008A
:105C30009000980080CCB3009040980000000600CF
:105C400036D0BF000080FB00710321009140780036
:105C5000C808DD0080807000F0828000808F5000D6
:105C60000700310061032100914078008180FB0032
:105C700037D0BF004800DD0001007000F0828800CE
:105C8000B3FF07008103210080828000110098008B
:105C900081CCB30080828000114098000000060093
:105CA0000080FB00800140000180FB00008041007B
:105CB0004300DD000200210002014000124090007C
:105CC0000074A10010419800A00421000104E0002C
:105CD000010032000005210082317800124090005E
:105CE0000064A10010419800E400410011409000C0
:105CF0000064A0009040980000000600889FBE004D
:105D00008A1F780000447800014578008184FB00F8
:105D10000938A300020032008040EB00E0FF0700DA
:105D20000928A3000300320011C0B3000840780026
:105D3000DBFF07000880FB0000004000A14A2000B4
:105D40000AF078004F0578004F04BE0000000600FE
:105D5000014178000004E0000C003A0081C0B3006B
:105D600040828000014878004182800000032100C9
:105D700090009800C0C8B3009040980041C8B3009C
:105D80008082800011409800000006008080FB00A7
:105D9000818040000280FB0080804000C308DD005D
:105DA00002002100028140001240900043C8B3006D
:105DB00003407000104198004000210080804000A6
:105DC00011409000034070009040980000000600D1
:105DD000004378000082FB00814378000104E0006A
:105DE0000300320084004200000521000200370059
:105DF00084004200A0042100E10278000500E000D8
:105E000002003A0005007800000006000682FB0050
:105E100092029800834A7800154090000044B20036
:105E2000904298001540900081C8B3000140700076
:105E3000904298000704E000030032000400420092
:105E4000010521000200370004004200A1042100E6
:105E5000010040001024A2000500780000000600A8
:105E60008040780094C4BF000058A300180032009E
:105E70000181FB000201410004052100E2017A00DA
:105E80001300BE0005042000008062000100200015
:105E90008089BE00E2017A00000420000100200099
:105EA0009319680093916800040141001224A20034
:105EB00092007800114090000044B2009040980099
:105EC00092007800114090000540680090409800D2
:105ED000000006000000EB00A02488006024880079
:105EE0000082880000000600018280000100E000BE
:105EF00011003A00A12488006124880020002000BD
:105F000030258800412588008644A900F00920003A
:105F100080248800602488009EC0A800010037000B
:105F20009404A80094C4BF000008A300FCFF320042
:105F300010002000008288000000060090F9880010
:105F4000A1F98800B2F988000000060092F98000EB
:105F5000A3F9800000A02C00A1B923003EEA37007D
:105F600090F98000A1F9800000000600B0F98000DF
:105F70000000060080C12F00561FB400813E2000A3
:105F8000810F500003003E0061F521001000200049
:105F9000910840000000060080C12F00561FB40089
:105FA000813E2000810F500003003E0061F521007A
:105FB0000080EB009108400000000600B1FA80006C
:105FC000803E2000808F500001003A000140FE001A
:105FD0000000060080017800B2F980008301E8002B
:105FE000C210DE008301E900040032000280BF001D
:105FF000FCFF32000000E900FDFF37000000060052
:106000000000000000000000000000000000000090
:106010000000000000000000000000000000000080
:106020000000000000000000000000000000000070
:106030000000000000000000000000000000000060
:109000008001EB000200370061F079008301E80085
:10901000828F5100FCFF3A00000006008001EB0047
:109020000200370001F079008301E800828F5100CF
:10903000FCFF3A0000000600889FBE008A9FBE0029
:109040008C9FBE008E1F7800000478000206BE00D0
:1090500050159000E0159000820F5500838F5D0041
:1090600034003200404090000004E0002100320053
:10907000EE022000080747001840900014C0B3001B
:109080000A01BE008E007800FA2107000000E0000F
:1090900026003A004044980078089000881090001C
:1090A00058099000E80990000000410081804900C3
:1090B000800F5500818F5D000E003100B844900094
:1090C0000A00370058089000E80890000A054000A0
:1090D0008B8548001840900014C0B3000A01BE0000
:1090E0008E007800E32107008944E900E1CF5400B5
:1090F000F4FF3E00E00F5600E08F5E000D003200EE
:10910000E1022000888040001840900014C0B300A5
:109110000C01BE009B2107000000E00003003A00A4
:109120005C1498006D1498000300370010002000B4
:10913000010037000000EB004F0778004F06BE002B
:109140004F05BE004F04BE0000000600881F7800D7
:109150000004780062025100E0825900C0089000CB
:109160003008900062005000E08058006011B800A4
:10917000800F5200818F5A00090031002841900071
:109180000281FB00030020000400BE00A4DD0700F4
:1091900038119000C8119000000141008181490000
:1091A0000200BE004F04780000000600889FBE0049
:1091B0008A9FBE00000578000204BE00E10F510046
:1091C000E08F590079003600C00890003008900008
:1091D000800F5100818F5900740031001A407800CF
:1091E000E24F50002E003200E34F500043003200A7
:1091F000E14F500070003A00820478000200D10074
:10920000000441004941DE007A0890008A10900075
:1092100002014000E08148000A00780086FF070054
:109220000000E00064003A0008007800F01FB2007F
:10923000E002B0000A0040009085FB000804E8004E
:109240004941DE007A0890008A1090000201400037
:10925000E08148000A00780077FF07000000E00086
:1092600055003A00F81FB200E0022000080040005C
:109270000A0040001080FB004800DD00808075007F
:109280000908A300020032004408DE000200370093
:10929000F0FF20000080600001002000480037003F
:1092A0004818DD004811DE0002017000C819DE0018
:1092B0007A0890008A1090000201400083814800E3
:1092C0000A0078005CFF07000000E0003A003A0066
:1092D000E20220000A0141000800440089804C009D
:1092E000F01FB20000014100124090004800DD0074
:1092F0009280FB0001007000E7FF37004918DD0095
:109300004711DE0002017000C719DE007A089000E4
:109310008A10900002014000838148000A00780012
:1093200045FF07000000E00023003A00E4022000AF
:109330000A0242004248DD00CE40DE00810070009B
:109340004240DD00F01FB2000002420034419000B4
:10935000C811DD0002002000244090008080FB0046
:109360000000200000017100818171001440900014
:109370004800DD00010020000001710081817100C2
:10938000144078000080FB00010020000001710003
:1093900081817100F0FF20000300600080037800ED
:1093A000020378000600BE00050037001000200010
:1093B00001002000020037000080EB008080EB00FD
:1093C0004F05BE004F04BE0000000600E4874700C2
:1093D000889FBE008A9FBE008C9FBE008E1F7800B3
:1093E000000578000204BE000406BE00E10F510033
:1093F000E08F59009F003600C008900030089000B0
:10940000800F5100818F59009A0031001A40780076
:10941000E24F500044003200E34F50005900320048
:109420002B002000E14F50008F003A000200D100D5
:10943000800441004949DE007A0890008A109000BB
:1094400002014000E08148000A007800FAFE0700AF
:10945000800578000000E00083003A00EE02200062
:109460000A07470009007800F01FB200000147001A
:10947000610064000100200080BF9F000000E00048
:109480000500320012427800EF4062004460DD00C7
:1094900001407000010037000C407800004978005E
:1094A0000904E80010C0B300404598004941DE00BF
:1094B0007A0890008A10900002014000E081480084
:1094C0000A007800DCFE0700800578000000E0005C
:1094D00065003A00F81FB200880147000FB89700F6
:1094E0000000E000050032004C69DD004460DE0051
:1094F00000007100C468DE000800370002CFB3002E
:1095000013416100486ADD004860DE00000072001F
:10951000C868DE006F40600000407100804978003C
:109520008005EB00500037004818DD004811DE00D0
:1095300002017000C819DE007A0890008A109000BD
:1095400002014000838148000A007800BAFE07004B
:10955000800578000000E00043003A00E0022000AF
:109560000A0040000801440089814C00F21FB2004B
:10957000020040000C487800C860DE0011409800EE
:1095800039003700491ADD004711DE000201720080
:10959000C719DE007A0890008A109000020140008E
:1095A000838148000A007800A3FE07008005780048
:1095B0000000E0002C003A00E40220000A02420011
:1095C0004248DD00CE40DE00810070004240DD00F8
:1095D000F01FB20000024200E30342000483E800EF
:1095E0008402E80017417800C811DD000200200065
:1095F000164078008080FB00000020000001710010
:10960000818171001580FB004800DD000100200011
:109610000001710081817100144078000080FB001E
:1096200001002000000171008181710000002F0005
:109630000300600001002000C000DD0000002000E9
:109640000000760081807600004A78004801DE0044
:10965000824A78004009DE0003002000024B7800B7
:109660004808DE00804B780010C0B30040459800E9
:10967000010037002B0020000B0078004F07780016
:109680004F06BE004F05BE004F04BE004F00B100A4
:10969000000006000400FA00889FBE008A9FBE00FA
:1096A0008C1F78000006780092BF9F00A3BF9F0028
:1096B000E00F5100E08F59000B003A005005900078
:1096C000E0059000E00F5500E08F5D0015003200CE
:1096D000C008900030089000800F5500818F5D0019
:1096E00010003100110037001FB99700AFB9970083
:1096F000AEFE07000001BE00E10F5000E08F5800F1
:109700004D0036003C089000CC089000800F5100BE
:10971000818F59004C0039001FBD9700AFBD9700E5
:10972000020037001A0020000B0020000A04BE00CF
:1097300061044400E0844C003C089000CC08900098
:10974000800F5400818F5C0005003900E10F550047
:10975000E08F5D003B00360028002000090020005B
:109760000801BE000C00780090FE07000001BE005A
:10977000E00F5000E08F58000A003200E10F400077
:10978000E08F480030003200E10F5000E08F5800B9
:109790002D0032008A0F54008B8F5C0029003200AC
:1097A000E3FF3700F4FF2F00F5FF20000801BE00A3
:1097B0000C00780005FF07000000E0001A003A00E6
:1097C0001FB89700AFB89700E00F5000E08F580027
:1097D000060032000802BE000001BE000C00780046
:1097E000FAFE07000000E0000F003A00580698005B
:1097F000690698007C0090008C089000E10F400002
:10980000E08F48000600320061005000E080580000
:1098100070069800010E980010C0B30050469800E2
:109820000801BE00080037000081EB008081EB00DA
:10983000E10F50000400320012002000030020005D
:10984000010037006011B8000200BE004F0678002A
:109850004F05BE004F04BE000080FA000000060065
:10986000889FBE008A1F78000004BE002104980073
:1098700030019000C0019000E10F5100E08F5900CD
:10988000480032001002780034089000C4089000AC
:10989000800F5100818F590042003100E00F5100CC
:1098A000E08F590016003A0030C0B300944F10000A
:1098B00005003A0014119000A4119000E00F51002F
:1098C000E08F59000E003A006000B8005004980084
:1098D0006104980044009000808F540031003100F2
:1098E0004448DE0014119000A411900000004100D3
:1098F000E080490070049800010C98001F003700B8
:10990000244090000080FB004405DD00100037007B
:109910001800780025FE07000001BE00E10F40009E
:10992000E08F48001D003200E10F5000E08F58002A
:109930001C00360018007800C00890003008900025
:10994000800F5100818F5900160031008A84540025
:109950008A8F5400EEFF310052049800630498008F
:1099600018007800F9FD07004449DE0002014000BC
:10997000E081480072049800030C9800E002200087
:10998000980040006F8064004500DD00808040004A
:10999000110C98000000EB000300370010002000BD
:1099A00001003700200020004F0578004F04BE0062
:1099B00000000600889FBE008A9FBE008C9FBE00EC
:1099C0008004780001047800200090000006E80080
:1099D000770032007900900089089000E00F500075
:1099E000E08F580072003200EF06660068003A000F
:1099F00061004000E0804800F0049800810C98006D
:109A00001902780059019000E9019000E00F51001F
:109A1000E08F590004003A0044009000800F560087
:109A20005B00390062003700C460DE002440900013
:109A30000080FB000000E9008080600054003A00D4
:109A400004007800D9FD07000005BE00E10F5000BA
:109A5000E08F580058003600E10F4000E08F4800CA
:109A6000570032001902780034089000C4089000B2
:109A7000800F5500818F5D003E0039000800E00036
:109A80004B00320059019000E90190000400780079
:109A900000FF07000005BE0070002000E00F550029
:109AA000E08F5D0047003200E10F5500E08F5D0060
:109AB00041003200E10F4500E08F4D0040003200D0
:109AC0006011B800190078005BFD07000000E0009D
:109AD0003B003A00E10220001980400002202000F3
:109AE0008D0078004DFD0700190478000A01BE00C2
:109AF0000800780095FD0700501498006114980044
:109B00000D0478000F00370010C0B30040429800E9
:109B10006011B8001900780047FD07000804E8004C
:109B20000000E00026003A00190178005210900071
:109B3000E210900061004000E08048005011980061
:109B4000611198001902780024409000804F540061
:109B5000EDFF39000881FB00030020005410900045
:109B6000E4109000020050008380580050129800CA
:109B700061129800DA049800EB0498000A01BE0014
:109B80001900780071FD0700F0049800810C98001E
:109B9000AC049800E102200019804000C568DD0097
:109BA00001004000900C98000000EB000500370019
:109BB0004000200003003700200020000100370093
:109BC000100020004F06BE004F05BE004F04BE002F
:109BD00000000600881F7800E8022000000444000E
:109BE0001040900014C0B30088007800E51E070004
:109BF000320020000000E0003F003A0078F89300B7
:109C00004800DD00E8F893008180FB00010070004F
:109C10002200200051A52A00810F500036003A0092
:109C200018799000C811DD0002002000087890002B
:109C30008080FB0000002000000171008181710024
:109C4000787090004800DD000100200000017100E4
:109C500081817100687090000080FB00010020008D
:109C600000017100818171000380FB008002780097
:109C7000020278000400BE0066142400470520009C
:109C8000860F5000878F58001A00320058D190007C
:109C9000C811DD000200200048D090008080FB0049
:109CA00000002000000171008181710038D0900017
:109CB0004800DD0001002000000171008181710079
:109CC00028D090000080FB000100200000017100FE
:109CD000818171000380FB0080027800020278001D
:109CE0000400BE0012002000860F5000878F58002D
:109CF00001003A000001EB00020078004F047800F8
:109D000000000600000178000000E0000C003200B6
:109D10001004E0000A00320030009000810F500073
:109D200007003A00124090008F1E0700610060009B
:109D30003100200003003A00800078000100370065
:109D4000910020000100780000000600B200200011
:109D50000004E00009003A0052FA80000200E0002E
:109D600001003200004978000100E00001003200EB
:109D70008048780051FA88000001EB00020078006A
:109D800000000600EF03B000889FBE008A9FBE005F
:109D90008C9FBE008E1F7800E0B79F0001077800FF
:109DA0000008EB007F406100C0DF9F007E4461003F
:109DB0009100FB0000FD2F0000814000E90F5100E1
:109DC00008003E009E409000A0C3B30080CF50002A
:109DD00004003A000E87E800B90020000200E0000D
:109DE000A2013A005AFA80009AA79F00C9002000F9
:109DF0000A00E0009D0132001A04E0000A0032006F
:109E00001A409000581E07000080FB000008A300C5
:109E100005003A000804E000910132000028A30088
:109E20008D013A008E0137000040EB00004D7800B4
:109E300010459800BF1D07000080FB00390020007E
:109E40000008A30089013A000804E0000200320083
:109E50000028A30080013A006011B8000A007800D1
:109E60005CFF07006011B80092B79F00A3B79F0086
:109E7000E14F50001B003A00E40220000A024200B9
:109E800024C093000004E0007701320014C993005D
:109E9000C811DD000200200004C893008080FB0090
:109EA00000002000000171008181710074C09300E6
:109EB0004800DD0001002000000171008181710077
:109EC00064C093000080FB000100200000017100CD
:109ED0008181710092B79F00A3B79F000A007800AC
:109EE0003CFF070019002000E34F50005F013200E3
:109EF0000004E0005C013A00EB0220008A85450086
:109F00002A7890004800DD009A7890008180FB005C
:109F10000100700001202000810F500052013A0022
:109F2000DAC09000C808DD004AC090000080FB0045
:109F300080807000610AB80012003A007B619000D6
:109F4000C811DD00020020006B6090008080FB00E3
:109F50000000200000017100818171005B609000B1
:109F60004800DD00010020000001710081817100C6
:109F70004B6090000080FB00010020000002710097
:109F800081827100540D9800650D9800EA78900068
:109F9000314598000140E900E14F500032013E0098
:109FA0000181FB00030020000400BE001CDA070052
:109FB000F0B79F0081BF9F00BA7B900027459800B3
:109FC0000704E000280132000780FB008000E90060
:109FD0000100600024013A000AC090004800DD0042
:109FE000FA7890008180FB0001037000460598001C
:109FF0006F0063001C013A00AAC09000C808DD0091
:10A000001AC090000080FB0080807000610AB800D8
:10A0100012003A003B619000C811DD0002002000F0
:10A020002B6090008080FB00000020000001710088
:10A03000818171001B6090004800DD00010020005C
:10A0400000017100818171000B6090000080FB00B5
:10A05000010020000002710081827100DA78900016
:10A06000C808DD004A7890000080FB000080700086
:10A07000FD0032006104B800C8B79F00D9B79F0047
:10A080007FB197008FB9970008004100898049008F
:10A090004431DE0002044000E0844800880F520092
:10A0A000898F5A00F00039000800520089805A0058
:10A0B0000781FB0003002000E7D90700E00F5000F4
:10A0C000E08F5800E800320013C0B300E3E79F00C0
:10A0D00054FF2000840F5000E08F58000700360026
:10A0E00035C0B300E5E79F00EB0F4000E08F58005C
:10A0F00002003E0022C0B300E2E79F00620640007B
:10A10000E08648003C0D98004D0D98001FB2970066
:10A11000AFB297000400440085804C0030159800D1
:10A12000411598004FB49700DFB497000400440035
:10A1300085804C00700D9800011598004A01900030
:10A14000EFE49700E3CF54001B003A000200E00068
:10A15000C5003A007B699000C811DD0002002000B4
:10A160006B6890008080FB000000200000017100FF
:10A17000818171005B6890004800DD0001002000D3
:10A1800000017100818171004B6890000080FB002C
:10A1900001002000000171008181710012159800FA
:10A1A000231598004268DD00CE60DE00810070005B
:10A1B0004260DD00170037000200E000AA00320014
:10A1C0007FB197008FB9970000004100818049005E
:10A1D0001015980021159800EFE19700E2CF51008B
:10A1E00003003A000C0046008D804E000900370045
:10A1F00032002000030020000C00BE0088D90700B8
:10A200008100D1000080D30061016600020040009F
:10A21000E0804800F01FB0000180B000C909DE00F6
:10A22000470ADD004901DE00020172005A08900071
:10A23000EA089000820F5000838F58008A0039008E
:10A240000080EB008080EB0070059800010D980005
:10A250006000B8005005980061059800EFE2970093
:10A26000E3CF520071003A000040EB0050459800E7
:10A270001B7190004811DD000B7090000080FB0006
:10A28000000171001FB49700AFB4970002014400B1
:10A29000E0814C00120D9800230D98001A409000A8
:10A2A00014C0B3008B007800361D07000000E000EA
:10A2B0005E003A007BF893004800DD00EBF8930065
:10A2C0008180FB000100700051A52A00810F500021
:10A2D00056003A003B419000C811DD00020020000A
:10A2E0002B4090008080FB000000200000017100E6
:10A2F000818171001B4090004800DD0001002000BA
:10A3000000017100818171006A6890000080FB008B
:10A3100001002000000171008181710020252500CD
:10A3200011162400800F5100818F59003F003A0020
:10A330007BE19300C811DD00020020006BE0930078
:10A340008080FB000000200000017100818171000D
:10A350005BE093004800DD00010020000001710077
:10A36000818171004BE093000080FB000100200020
:10A37000000171008181710020272700111426003F
:10A38000800F5100818F590028003A007BE993002B
:10A39000C811DD00020020006BE893008080FB0004
:10A3A0000000200000017100818171005BE89300D2
:10A3B0004800DD0001002000000171008181710072
:10A3C0004BE893000080FB000100200000017100B9
:10A3D0008181710052059800630598003BE9930064
:10A3E000C811DD00020020002BE893008080FB00F4
:10A3F0000000200000017100818171001BE89300C2
:10A400004800DD0001002000000171008181710021
:10A410000BE893000080FB000100200000017100A8
:10A420008181710072059800030D9800EFE4970098
:10A43000094D7800481FEC0040FA8800300598006C
:10A440006000B80050159800611598000040EB00BE
:10A450004045980002003700A900200003003700A3
:10A460008004EB0001003700D900200060FB2F00C2
:10A470000F004000B0AF9F000900E000CF003A009D
:10A480009E407800F0C2B30080CF5000050032003B
:10A49000C0C5B30080CF5000020032000E04780027
:10A4A000010037000E04E8006000B800C0A79F005C
:10A4B000D1A79F00F1C1B30098CF100009003E0062
:10A4C0008000EB0022FC2F000F004100E4FC07009D
:10A4D000800478000000EB00A0AF9F00B7003700B9
:10A4E0000804E80098407800F0C2B30080CF500024
:10A4F000FBFF3200C0C5B30080CF5000F8FF320030
:10A50000BFAC9700B20020000102200009007800D3
:10A51000C2FA07008041EB008002EB00850378005F
:10A5200086002000E8C07B00014178008703E80036
:10A5300000C2B30080CF5000350036006F404000AD
:10A5400080CF500032003200C0C5B30080CF500031
:10A550002F003200E0C2B30080CF50000200320072
:10A56000868F520008003900E80F530090003A002F
:10A5700080CF50008E003A00C219DD0086027800BC
:10A58000B6002000E7FF37000104E00005003D00B1
:10A590003340B3000180FB000008B10021B02A0065
:10A5A00060C178000282FB0021B82A000100370058
:10A5B0008100E800114078000004E000040032004F
:10A5C0000000FB00840F5000F9FF3A0078003700CC
:10A5D000F0CBB30000404100F94F500002003E00B4
:10A5E0000314A00007003700F0C9B3000040410089
:10A5F000F94F500003003E000304A00000CEB3005A
:10A600000041410082F27C008502E800C5FF37006E
:10A610000704440042C0B30000C2B30080CF500022
:10A620000600360004003700490020003E003700D5
:10A63000800478003C0037000041EB000500E0009A
:10A640005B00320054CEB300994F120002003A0072
:10A6500050C0B300804C7800E80F530001003A006E
:10A66000C219DD008380FB0063806000E10F5000B1
:10A6700001003A000244A0006C806000E40F50002A
:10A6800001003A000234A000B24C98008000EB00B8
:10A6900025FC2F000F80420071FC07008004780029
:10A6A0000000E00020003A000FA997009FA9970042
:10A6B0001FA0970060FA0700800478000000E00007
:10A6C00019003A00AFA897001104E000D6FF32004D
:10A6D000314890000038A3000E003A0001027800D3
:10A6E000BFA99700B2002000090078000201E9002C
:10A6F000E10F410005003200B480FB003380FB0015
:10A700000080500003003A00F8FF37000000E0002E
:10A71000C7FF32008000EB0029FC2F000F804400AF
:10A72000A4FC0700DDFF37003FA8970030489000E9
:10A730000900E00005003200E48F54001F003A00D9
:10A740000028A3001C0032001C0037000028A300D2
:10A750001A003A00AFA89700314890000048A300C3
:10A7600015003200515190004811DD004150900019
:10A770000080FB000001710003002000C011DD001B
:10A7800002002000315890004800DD00215A90005E
:10A790000482FB0004007000010020000001710031
:10A7A00081817100C2A79F00D3A79F004DFF370092
:10A7B000690020000100370059002000AFAE97006B
:10A7C0000900E00003003A000D00E00001003A003B
:10A7D000690020004FD897008080FB007C806000DB
:10A7E000A30032000900E0002E003200E48F540084
:10A7F00025003A008000EB0022FC2F000F004100F2
:10A8000017FC0700800478000000E0001E003A00FA
:10A8100023FC2F000F8441000FA997009FA99700E8
:10A820001800780004FA0700800478000000E000B7
:10A8300015003A002FA8970010407800FB4F400009
:10A84000D80032000004E000D600320011002000E1
:10A850000800780057FC0700EAFF37002FAC97008C
:10A86000020220000800BE00ECF90700BFA8970014
:10A87000B200200008007800E1F907009A00780093
:10A8800010C0B300C04098004FDA97000434A00015
:10A89000C4DF9F00AFAE97000900E000080032005F
:10A8A000D90037003D489000710060007900200019
:10A8B000D5003A00890020000128A300D2003A0008
:10A8C000CFDA97000538A3007C003200682A070021
:10A8D000E04E98004801DE00F24E98004009DE008C
:10A8E00003002000825698004808DE009056980029
:10A8F0008042EB00B54E9800C55E9800D55E98008A
:10A90000E55E9800F55E9800F58446007484460084
:10A91000FB8346007A8346001981FB004811DD0065
:10A920001880FB000001710003002000C011DD0051
:10A93000020020001780FB004800DD001682FB00AB
:10A94000040070000100200000017100818171008D
:10A95000F2AF9F0083B79F00054B7800854B7800CE
:10A96000054C7800854C780028FC2F000F0144002E
:10A970009200780010C0B300C04098007FA89700F4
:10A980008FB09700E00F5000E08F58004600320073
:10A99000120678005C119000EC119000C2AF9F008D
:10A9A000D3AF9F00E10F5000E08F58002E0036001B
:10A9B0003C089000CC0890007FAA97008FB29700C7
:10A9C000800F5200818F5A00270031000404BE001E
:10A9D0000801BE000C007800F4F907000005BE0075
:10A9E000E00F5000E08F580078003200E10F500077
:10A9F000E08F58001C003200E10F4000E08F48005B
:10AA0000800032006022B8000801BE000C0078000F
:10AA10006EFA0700800478000000E0007A003A0037
:10AA20007C0090008C089000E10F4000E08F48000F
:10AA30000600320061004000E08048007006980087
:10AA4000010E980010C0B300504698003C089000DA
:10AA5000CC089000800F5500818F5D005B003100B5
:10AA60000A04BE00DAFF3700290020006600370024
:10AA70000900E00064003A003D4890000080FB00BF
:10AA8000490020000048A3005F003A000118A3001D
:10AA900003003200790020000008A3005A003A00A9
:10AAA0000138A300050032008004EB00CFDA9700E4
:10AAB0000554A000C5DF9F00010037008004EB00B3
:10AAC0009FA2970055109000E51090006FB197007D
:10AAD00050099800610998007D099800CFD9970026
:10AAE000434198005D5190004811DD004D509000A9
:10AAF0000080FB000001710003002000C011DD0098
:10AB0000020020003D5890004800DD002D5A9000C2
:10AB10000482FB00040070000100200000017100AD
:10AB2000818171006FB2970072029800030A980049
:10AB30007D599000C811DD00020020006D58900082
:10AB40008080FB0000002000000171008181710005
:10AB50005D5890004800DD000100200000017100F8
:10AB6000818171004D5890000080FB0001002000A1
:10AB70000001710081817100520298006302980007
:10AB80006000B8003002980041029800300A980036
:10AB9000410A9800050A7800B50290001502980055
:10ABA0001900370025FC2F000F8542000FA99700E0
:10ABB0009FA997001A0078001FF907008004780009
:10ABC0000000E00030FF3A0024FF37001FA097008C
:10ABD0007FAC97008FB4970061015400E0815C0066
:10ABE00052009800630098004FA99700DFA99700D2
:10ABF00011F90700800478000000E000ABFF32008C
:10AC00000100370019002000090078004F07780084
:10AC10004F06BE004F05BE004F04BE00EF03B1005B
:10AC200000000600E6874700889FBE008A9FBE009E
:10AC30008C9FBE008E1F7800800478000207780089
:10AC400083BF9F00F1B79F008009EB009000900048
:10AC5000100078002BFC07000000E000AE003A0076
:10AC6000C9409000200020000104E000AA00350047
:10AC7000700020000108A300A70032000D0037007B
:10AC8000494090000074A000C044980020002000BB
:10AC9000A10037000174A000C144980003003700F0
:10ACA000494090000074A000C044980010002000AB
:10ACB0009900370059009000E90090003901900098
:10ACC000C901900002015000838158006170B800F2
:10ACD000820F5000838F58008C00360002077800E6
:10ACE0008A00370039029000C90290000400780001
:10ACF000F01FB2006C003A00990078004728DD0090
:10AD00004921DE0002017000C929DE0021409000C7
:10AD10000040E9008246600012003A00E00F520055
:10AD2000E08F5A0003003A007900900089089000F3
:10AD30000400370019099000A9099000010078006B
:10AD40001AF90700E10F5000E08F5800CCFF3600E1
:10AD5000E10F4000E08F4800D1FF3200900C9800D6
:10AD6000A10C98001906780019099000A909900013
:10AD70000C007800F5F807000001BE00E00F50005D
:10AD8000E08F5800BEFF32000D80FB000100200064
:10AD900002054000838548004974DE00250032002A
:10ADA000AC4090000D81FB00080041008180FB0059
:10ADB000810F500001003600028450001C409000BA
:10ADC000084278000A01BE00FFB097006D1A070024
:10ADD000C94090000000E000AEFF3A000168A30007
:10ADE0001200320039089000C90890000A01500092
:10ADF0008B8158006140B800800F5100818F59004D
:10AE00000A0031000102200089804000491ADD005B
:10AE1000C711DE00830172004911DD007FB2970087
:10AE2000020042000220200075F807004944DD00BE
:10AE30002A00370039099000C90990008A0F510093
:10AE40008B8F590016003200494090000068A30023
:10AE50000A00320001022000898040001C4090005E
:10AE600014C0B300831A0700C94090000000E0003E
:10AE700088FF3A000164A100C1449800010220004B
:10AE800089804000190078001040900014C0B30081
:10AE90000A01BE003B1A07000000E00080FF3A00F4
:10AEA000BA0C9800CB0C9800B9019000F31FB200C7
:10AEB00000202000030450008E0F540001003600D3
:10AEC0000E04780001022000898040008380400049
:10AED000080178007FB0970049F807007FB097001D
:10AEE00008004000F0B79F0039009000C9009000B2
:10AEF00008004000E0804800B0049800C1049800B9
:10AF00000FBA9700140A4400080757000E00E0002B
:10AF100074FF3A000E0078004F0778004F06BE001D
:10AF20004F05BE004F04BE006F00B10000000600D8
:10AF3000E6874700889FBE008A9FBE008C9FBE00A8
:10AF40008E1F7800000478008206780083BF9F007F
:10AF5000F1B79F008009EB0090009000100078008E
:10AF600068FB07000000E000CE003A00C8409000F7
:10AF7000200020000104E000CA003500700020001D
:10AF80000118A300C70032000D0037000174A000B3
:10AF90004144980008003700484090000074A00029
:10AFA0004044980020002000BE0037004840900038
:10AFB0000074A0004044980010002000B900370041
:10AFC00058019000E80190000D004100E080490028
:10AFD000820F5000838F5800A5003900A20037006F
:10AFE00038029000C802900004007800F01FB20000
:10AFF00081003A00980078004728DD004921DE00F2
:10B0000002017000C929DE00214090000040E900E3
:10B01000024760001E003A00E00F5200E08F5A0025
:10B020000B003A007801900088099000E00F510071
:10B03000E08F59000E003A000100780095F90700F2
:10B040000001BE0070049800010C98000500370054
:10B0500018099000A8099000010078008DF90700F8
:10B060000001BE00E00F5100E08F59008000320067
:10B07000E10F5100E08F5900C7FF3200E10F41009E
:10B08000E08F4900C9FF3200120C9800230C980091
:10B09000484090000068A3000D003200380990007D
:10B0A000C8099000180078001040900014C0B30048
:10B0B0000102200088804000EE190700C84090007F
:10B0C0000000E000B1FF3A000164A1004144980093
:10B0D0001806780018099000A80990000C00780064
:10B0E0001AF807000001BE00E00F5000E08F580082
:10B0F000A9FF32000E80FB00010020000205400085
:10B1000083854800C96CDE0025003200AC40900009
:10B110000E81FB00090041008180FB00810F50007F
:10B1200001003600828450001C40900009427800E3
:10B130000A01BE00FFB09700CE1907000000E00032
:10B140009AFF3A0038089000C80890000A015000A1
:10B150008B8158006148B800800F5100818F5900E1
:10B160000D0031004918DD00C710DE0081007000BD
:10B170004910DD007FB197008000410002202000CF
:10B1800000022000080040009DF7070048409000A2
:10B190000064A10040449800C94CDD00260037003F
:10B1A00038089000C80890008A0F50008B8F580014
:10B1B0000F00320038019000C80190005800900044
:10B1C000E8009000800F5100818F59000800310085
:10B1D0001C40900014C0B3000A01BE000102200010
:10B1E00088804000671907000000E0006FFF3A0008
:10B1F0003A0C98004B0C9800B8019000F31FB20075
:10B2000000202000830450008D8F54000100360080
:10B210008D04780000022000080040000300400078
:10B2200009017800FFB0970075F7070048409000CB
:10B230000064A000404498007FB0970009004000DF
:10B24000F0B79F0038009000C8009000090040004F
:10B25000E080480030049800410498000FB997003E
:10B2600012894400898656000D00E0005CFF3A0018
:10B2700038019000C801900058009000E80090004C
:10B28000800F5100818F590002003600520498004F
:10B2900063049800484090000054A0004044980087
:10B2A0000000EB004F0778004F06BE004F05BE00C0
:10B2B0004F04BE006F00B10000000600889FBE0072
:10B2C0008A9FBE00800478009000900010007800F3
:10B2D0008CFA0700000578000000E00082003A00C8
:10B2E000494090000080FB000058A3007D00320020
:10B2F0000068A3000D00320039099000C9099000D0
:10B300000102200089804000190078001040900060
:10B3100014C0B300571907000000E0006F003A00A6
:10B32000494090000064A100C04498005909900071
:10B33000E9099000190078003FF707000005780040
:10B340000000E00068003A00790C90006B004400B7
:10B350001054A00029489000405C980039489000A3
:10B36000505C980049489000605C980059489000F3
:10B37000705C980069489000205C980079489000C3
:10B38000305C98000950900040549800195090008B
:10B3900050549800B6270700605498004801DE001A
:10B3A000725498004009DE0003002000025C9800FF
:10B3B0004808DE00105C9800494090000054A1004D
:10B3C000C0449800190078001BC0B3004B4098009F
:10B3D000990478006011B8000900780016F707009A
:10B3E000000578000000E0003F003A0030C0B300E4
:10B3F000994F100033003A00594090000004E000DB
:10B40000300032006000B800D0149800E1149800B9
:10B41000E802200009044400022020008A0078008D
:10B4200008007800FDF6070050C5B30060FC9B00E3
:10B43000A0CAB30070FC9B0020C5B300004C78008C
:10B44000F06C980012C6B3008274980011C4B30067
:10B450009174980020C7B30040E49B0050E49B0027
:10B4600061E49B0072E49B006948900000EC9B0043
:10B470007948900010EC9B000950900020EC9B0054
:10B480001950900030EC9B002948900040EC9B0044
:10B490003948900050EC9B004948900060EC9B00BC
:10B4A0005948900070EC9B0019099000A909900080
:10B4B000194090000B42780088007800ED180700D2
:10B4C000DA449800194090000001EB008040EB0046
:10B4D000361907000000E000020032001A002000C8
:10B4E000010037000005EB000A0078004F05BE00A0
:10B4F0004F04BE0000000600881F7800000478009A
:10B500006EFF07000000E00001003A00000C780028
:10B510004F047800000006000800FA00889FBE0073
:10B520008A9FBE008C9FBE000005780082BF9F00EE
:10B5300093BF9F009000900010007800F1F9070081
:10B54000000178000000E000EC003A004A40900062
:10B55000220020000004E000E80035005A019000BD
:10B56000EA0190000FBA97009FBA9700820F52002D
:10B57000838F5A00040036000018A30002003A002E
:10B5800082BF9F0093BF9F003A019000CA019000C4
:10B590006000B80030059800410598000FB897008A
:10B5A0009FB89700E00F5000E08F58009A003200DB
:10B5B0009A0578002B4090000080FB0001002000DD
:10B5C000490ADD00C702DE00850272004902DD0083
:10B5D000E4B79F00F5B79F00E00F5100E08F5900DE
:10B5E0002400320061065100E08659000FB997002F
:10B5F0009FB9970061005100E08059000401BE002E
:10B6000095D407000004BE006FB19700FFB197000A
:10B610000C00BE0090D40700800F5400818F5C00A6
:10B62000140039006FB29700FFB29700600012005B
:10B63000E0801A000C0160000D806000800278003C
:10B64000020278000400BE00300598004105980011
:10B650000FB997009FB997000001510081815900EF
:10B6600082BF9F0093BF9F001A099000AA09900013
:10B67000120037007A0190008A099000E00F510013
:10B68000E08F59000B003A000B00780001F807002A
:10B690000001BE00E10F5000E08F58005000320062
:10B6A000E10F4000E08F48008900320070059800EB
:10B6B000010D9800120D9800230D9800E00F510025
:10B6C000E08F59002E003A00530037004A409000A6
:10B6D0000018A3000B0032001A007800EDF70700F5
:10B6E0000001BE00E00F5000E08F580008003A0053
:10B6F0006FB29700FFB2970084BF9F0095BF9F0075
:10B70000260037001A007800A8F607000001BE00E6
:10B71000E10F4100E08F49006D003200E10F510060
:10B72000E08F59002E0036001A007800C008900003
:10B7300030089000800F5100818F5900280031009F
:10B74000120D9800230D98003A009000CA00900056
:10B750006FB29700FFB29700040040008580480058
:10B7600030059800410598000FB897009FB89700E2
:10B77000040050008580580080BF9F0091BF9F004B
:10B780000FBA97009FBA97006FB09700FFB097006D
:10B79000800F5200818F5A00CCFF3E003A0090008B
:10B7A000CA0090000FBA97009FBA970004004000AB
:10B7B0008580480030059800410598000FB8970033
:10B7C000F01FB200140032001A0078005FF6070084
:10B7D0000001BE00E00F5000E08F580005003A0065
:10B7E0004A4090000074A0004045980022002000CC
:10B7F000420037000FBA97009FBA9700472BDD0031
:10B800004920DE0000007300C928DE000206400067
:10B8100083864800010037006066B8003A00900057
:10B82000F01FB200210032003A099000CA099000CE
:10B83000820F5600838F5E001C0032004A40900049
:10B840000068A3000E003200010220008A80400040
:10B850001A0078001040900014C0B30005180700CB
:10B86000CA4090000000E000030032000174A00014
:10B8700041459800190037000164A1004145980036
:10B88000010220008A8040001A00780010409000D9
:10B8900014C0B3000C01BE00BA1707000000E0009E
:10B8A0000B003A003C0D98004D0D98003A029000B4
:10B8B000CA0290005A009000EA0090000001EB00DC
:10B8C000800F5200818F5A000C00360005003700AF
:10B8D0004A4090000074A0004045980012002000EB
:10B8E0000600370054059800650598004A4090000E
:10B8F0000054A000404598000001EB0002007800D1
:10B900004F06BE004F05BE004F04BE000080FA0087
:10B9100000000600889FBE008A1F7800000578009E
:10B920008104780002047800522207000841780060
:10B93000894078000A4078005C22070008417800BE
:10B94000894078000A407800662207004F05780099
:10B950004F04BE0000000600E40F50001F0032003C
:10B9600009003E00E10F5000110032000041EB00E1
:10B970001B003900E20F500010003200E30F5000AE
:10B9800025003A0011003700E60F50001600320083
:10B9900002C2B3008040EB000A003900E70F5000FC
:10B9A00015003200E80F50001B003A001600370067
:10B9B0000041EB0001C2B300110037000041EB0071
:10B9C00001C2B300014078000E0037000041EB00D7
:10B9D0008240780000C2B3000A00370002C2B30000
:10B9E00082407800F7FF370002C2B300824078003F
:10B9F0000040EB000300370002C2B3008040EB00C0
:10BA0000024078001B22370052C0B300F1C0B300DF
:10BA100000C2B3001722070000000600881F78004C
:10BA2000000478000001EB006000B800B9FF0700D7
:10BA30008043EB0007437800874278000742780094
:10BA400087417800074178008740780007407800F8
:10BA5000E02107008040EB0000C1B3003121070066
:10BA60008040EB0010C1B3002E2107008040EB00A6
:10BA700040C1B3002B2107008040EB0050C1B30050
:10BA8000282107008040EB0020C1B30025210700DA
:10BA90008040EB0030C1B300222107008040EB0062
:10BAA00060C1B3001F2107008040EB0070C1B300EC
:10BAB0001C2107008040EB0001407800192107009D
:10BAC0008040EB0010C0B30016210700E40F5400C3
:10BAD0001400320006003E00E20F54000E00320057
:10BAE0000B003E00E10F540022003A000A0037002C
:10BAF000E60F54001B0032000C003900E70F540021
:10BB000018003200E80F54001A003A0017003700FE
:10BB1000001020006D360700400020006B36070043
:10BB20000D003700080078001100370040002000A9
:10BB30006636070000012000643607008040EB00F5
:10BB4000E0C1B300F72007008032EF00E11C2100C4
:10BB5000F0DF2F00910860005E32EF006032EF00EE
:10BB6000040037005E32EF006032EF00400020003A
:10BB7000563607004F047800000006000010200031
:10BB80004536070000202000433607000001200052
:10BB900041360700400020003F360700100020001B
:10BBA0003D360700000120003B363700881F780033
:10BBB0000004780068FF0700E40F54002200320000
:10BBC00006003E00E20F54002A00320015003E003D
:10BBD000E10F540029003A0008003700E60F540036
:10BBE000240032001A003900E70F54001F00320011
:10BBF000E80F540021003A001E0037008043EB009C
:10BC00000743780005C2B3000542780085417800FB
:10BC10000741780087407800074078006D210700D1
:10BC200014003700001020001B36070040002000E1
:10BC3000193607000041EB0082407800F0C0B300E5
:10BC40008C2107000D003700080078000A0037003B
:10BC50004000200010360700000120000E360700CB
:10BC6000A00F20000094880004003700F62FEF009A
:10BC7000F42FEF0040002000073607004F04780043
:10BC80000000060000417800FF4F500002003E0017
:10BC90008000FB00070037008000EB00F0C3B3001A
:10BCA000804F510003003E000040E8000240500079
:10BCB0008000FB000100780000000600C27F8000C9
:10BCC000010040000100370069005000E80F5000FB
:10BCD000FDFF3C0001003700690040000000E0006B
:10BCE000FDFF3500E40F5000F5FF3200E80F500073
:10BCF000F3FF32000000E00002003A000200E00022
:10BD0000EFFF320000000600EC874700889FBE006E
:10BD10008A9FBE008C9FBE008E1F7800F14FEC0002
:10BD200080407800F1EFB70040C6B30080CF5000EC
:10BD30001C0036000040E800F1EFB700B1CFBF00B3
:10BD40000400320010C0B30011002000B45EE20015
:10BD5000010032008000EB00B4FEB7000104E000F7
:10BD600010003200D07F80002CFF0700917F800000
:10BD70000100E00012003200D07F8000808F500070
:10BD800004003A000000EB0088FF0700FA2FEF00E4
:10BD9000040037000100780084FF0700917F8000D5
:10BDA000D17F8800AF340700D17F80008001780008
:10BDB0000000E000060032000100780017FF0700D5
:10BDC00000402000C13507006CFF07005005370018
:10BDD000E38F5000B001320004003E00E18F5000BC
:10BDE00044003200E5003E0007003700E68F5000B7
:10BDF000BA033200E78F500068043200E58F50002C
:10BE000043053A00B7023700AFCFBF00040032004D
:10BE100010C0B30011002000B35EE2000100320048
:10BE20008000EB00B3FEB7000104E0000400320024
:10BE3000907F80008080EB00A0FF0700907F88004B
:10BE4000B0CFBF000400320010C0B30011002000CA
:10BE5000B25EE200010032008000EB00B2FEB700EB
:10BE60000104E00004003200907F80008080EB003D
:10BE700092FF0700907F8800B2CFBF00040032001D
:10BE800010C0B30011002000B15EE20001003200DA
:10BE90008000EB00B1FEB7000104E00004003200B6
:10BEA000907F80001100200084FF0700907F8800B1
:10BEB000B3CFBF000400320010C0B3001100200057
:10BEC000B05EE200010032008000EB00B0FEB7007F
:10BED0000104E00004003200907F80001100200087
:10BEE00076FF0700907F8800907F80009AFE070011
:10BEF00007053700289280000100780062242100A5
:10BF000092007800888F500002003400010478000D
:10BF1000800178000000E8000281E800E50F500091
:10BF2000F7FF3A0055F880006280110024002000DD
:10BF300000017800110009008402D8000001FD0012
:10BF40000280B90000057800C0DA20008000EB0014
:10BF5000800F540004003400080050001100090054
:10BF60000400D8008000FD0000FA2000800F54007B
:10BF7000020034008500EA000D00370070BB20008D
:10BF8000800F540007003C0080C12F0000004400D7
:10BF900072002000110009000200D800C112200028
:10BFA00080805000F07C2000800F5400020034009C
:10BFB000858F500001003400850078008504EA0078
:10BFC000898F50000100350081047800301F200067
:10BFD000800F540003003C005E32EF006032EF003F
:10BFE0000400370009004500009388000A805400CF
:10BFF000F0928800F04FEC008000FB00F0EFB700FB
:10C000000004E000090034000001EB000000EB0038
:10C0100040FE070080C2B300F04FE3000B00340085
:10C0200000C8B300F0EFB700080037008100EA0055
:10C0300042002000110009008200D8008000FD00AD
:10C040000001EB000000EB0032FE0700B2CFBF00A2
:10C050000400320010C0B30011002000AF5EE20007
:10C06000010032008000EB00AFFEB7000104E000E9
:10C070000700320050F880002003B00050F888001C
:10C08000411F2000810F50000100340051F888004A
:10C09000AFCFBF000400320010C0B3001100200079
:10C0A000AE5EE200010032008000EB00AEFEB700A1
:10C0B0000104E00007003200E0FC2F000A1FB4007A
:10C0C00050F8880041ED2F00810F500001003D0025
:10C0D00051F888008040EB00401F2000800F540082
:10C0E0000400340011C0B30010002000AD5EE20077
:10C0F000010032000000EB008000FD00ADFEB70043
:10C100008000FD000004E00002003200600020001A
:10C11000742C07000A00E0000C003A000900E0005F
:10C1200077043A00EF4FE20075043A00401F200008
:10C13000800F54007204340010C0B300EFEFB7005A
:10C1400070002000672C0700C8003700EF6FEF0079
:10C15000C6003700E0928000810F5000C700340015
:10C160008040EB0080C0B3006E1F07008040EB00F2
:10C17000B0C0B3006B1F070065043700788157001B
:10C1800084CC2A0007000900345978008200B100ED
:10C19000ED4FEC0080407800EDEFB7004240A90081
:10C1A00008003400034178003220070080C2B30049
:10C1B000ED4FE3000B00340000CCB300EDEFB7000F
:10C1C000080037000000FB000000EA002200200009
:10C1D000110009000200D800034178008040780077
:10C1E00024200700EECFEC0080417800EEEFB7008E
:10C1F0000080FB004500DE0002C2B300F8005000E2
:10C2000082F07F008000E900E7806000FFC16100EC
:10C2100003415100F880500082F07F000000E800E8
:10C22000670060007800500003F07F00FFEB97008C
:10C230002FE997009FE897006FEB9700DFEA9700E0
:10C240004FEA9700BFE997000FE89700E11F07004A
:10C25000B2CFBF000400320010C0B30011002000B4
:10C26000AC5EE200010032008000EB00ACFEB700E3
:10C270000104E0000700320040F880002003B00015
:10C2800040F88800411F2000810F50000100340059
:10C2900041F88800AFCFBF000400320010C0B300E7
:10C2A00011002000AB5EE200010032008000EB00D4
:10C2B000ABFEB7000104E00007003200E0FC2F00F5
:10C2C000081FB40040F8880041ED2F00810F500096
:10C2D00001003D0041F888004EF880000E00E000AB
:10C2E0005100350028928000349280006145B900E9
:10C2F00004004200CF80DE000A0540008B85480024
:10C30000409280006300B900CF80DE000A05400043
:10C310008B8548005292800002004100CF80DE00F1
:10C320000A0540008B854800669280006130B900A4
:10C330000A0540008B854800C0FF2F0000C4B900EB
:10C34000CFC4DE00D0FF2F0000A2B900CFA2DE00D4
:10C350000804420089844A006311B900CF91DE00CD
:10C3600008044100898449004233DD00CFB3DE0078
:10C370000804430089844B000A0044008B804C0071
:10C380006176B9000C01BE0025D10700027D2000B6
:10C39000811F7800110009004208D800CF00780002
:10C3A0000000570080BF9F00F092880008055500EC
:10C3B00089855D000C01BE000A00BE0018D107008F
:10C3C000047D2000811F7800110009004408D80076
:10C3D000CF007800000057000093880081DA2F001A
:10C3E0000FB89700810F500001003D00F1928800C6
:10C3F00000938000810F500001003D0001938800F0
:10C4000081252000F0928000810F5000010034004F
:10C41000F192880000938000810F500013003400D7
:10C420000193880011003700809280000E80B900CF
:10C4300042ED2F00811F7800110009004208D8004A
:10C44000CF00780000004700F092880070928000D2
:10C450000E80B900811F7800110009004208D80041
:10C46000CF007800000047000093880011082000EA
:10C47000D0928000810F500036FF3C005E32EF000A
:10C480006032EF0001C2B30080C0B300A51E0700F8
:10C4900001C2B30036FF370030F880008000400052
:10C4A00080804000909380000000E00001003D008B
:10C4B0000000EA0080804000A09380000000E000BF
:10C4C00001003D000000EA0080804000B093800041
:10C4D0000000E00001003D000000EA000080400094
:10C4E0004200DE0030F8880083007800ED0F500035
:10C4F00001003E0011002000810478008340780094
:10C50000EE0F50000400360011C0B30013002000ED
:10C51000AA5EE200010032008001EB000100780019
:10C52000AAFEB7000304E000040032000041EB0063
:10C5300082407800F0C0B3004E1F070030F8800042
:10C54000ED0F50000F003E00EA0FEC00507F880016
:10C55000E50F500007003400EA0F500001003A00D8
:10C56000EA2FEF000041EB008240780000C2B300E8
:10C57000190037000041EB0082407800024078004B
:10C5800015003700EC4FEC008001FB00ECEFB7002A
:10C590000004E0000A0034000001EB008000EB0022
:10C5A00003007800DBFC070080C2B300EC4FE3001F
:10C5B0000A00340000CCB300ECEFB70007003700EE
:10C5C0000300EA0022002000110009000200D80048
:10C5D0000041EB0082407800261F07008812E2002D
:10C5E000030032008832EF00500020003D2B07008E
:10C5F00037928000813E2000818F53001700340065
:10C6000040928000810F500014003400509280004E
:10C61000810F50001100340070928000810F500093
:10C6200003003C0080928000810F50000B0034001A
:10C6300021082000D0928000810F500007003400B4
:10C64000E0928000810F5000040034005E32EF0061
:10C650006032EF0019002000580037002892800057
:10C66000823E2000820F54000B003C00828F53005A
:10C6700009003C0040928000820F500006003C0000
:10C6800050928000820F500003003C0060928000B6
:10C69000820F5000380034005400200011000900BF
:10C6A0000404D800000378004200200011000900B3
:10C6B0008203D8000003430040928000110009006B
:10C6C0000200D80000034300509280006592800071
:10C6D000801F7800110009000200D80000017800D6
:10C6E0004F007800801F7800110009008402D800F4
:10C6F000800078004F0078000101410002034300F0
:10C7000062002000801F7800110009000204D80098
:10C71000800078004F00780080017800811F780049
:10C72000110009008403D8008001FD00CF007800CB
:10C7300083804000811F7800110009000400D800A8
:10C74000CF007800809FBE00110009008202D8004F
:10C75000800278004F00BE0005004000808050003D
:10C76000010043000000EA00F0928800868050003B
:10C77000019388001100370071928000828F500071
:10C7800003003C0080928000820F500009003400BA
:10C7900042002000110009008200D800F0928800B9
:10C7A00080928000110009000200D80000938800E8
:10C7B000020037005E32EF006032EF001108200007
:10C7C000D0928000810F500003003400E09280007E
:10C7D000810F50000A003C005E32EF006032EF0033
:10C7E0000041EB008240780000C2B300AF1E07009A
:10C7F0000041EB008240780000C2B3000700370020
:10C800000041EB008240780002407800A71E07003C
:10C810000041EB008240780002407800B11E070022
:10C8200081DA2F00F0928000810F500001003D005E
:10C83000F192880000938000810F500001003D00BC
:10C840000193880081252000F0928000810F500024
:10C8500001003400F192880000938000810F5000A5
:10C8600001003400019388008040EB000900E000E3
:10C870000400320011C0B30010002000A95EE200E5
:10C88000010032000000EB008000FD00A9FEB700AF
:10C890008000FD000004E0000200320040002000A3
:10C8A000922A07008040EB000900E00004003A00F3
:10C8B00011C0B30010002000A85EE20001003200A9
:10C8C0000000EB008000FD00A8FEB7008000FD0026
:10C8D0000004E0008E0232000080EB00812A070095
:10C8E0008B023700E11C2100708E80000098A300AD
:10C8F00040003200F0DF2F009108600077FE20003A
:10C90000974378000704E0000C003A000700780025
:10C91000E8EFB70010C0B300E7EFB70007437800B7
:10C920008742780007427800874178000741780005
:10C93000874078007F40400014003700E1CF53006B
:10C9400014003A0081FE200091407800E2CF5000B0
:10C9500028003400FDCF500026003C0020C0B3006A
:10C96000E7EFB7000140E800E3EFB700FFC3430083
:10C970000043EB008642780006427800864178004A
:10C98000064178008740780007407800111E0700B4
:10C9900018003700E2CF530016003A0081FE200055
:10C9A0009140780001407800E34FE30011003D0022
:10C9B00070C2B30080CF50000E003C0030C0B30006
:10C9C000E7EFB700FEC34300074378008042EB0067
:10C9D000054278008541780007417800874078005B
:10C9E00007407800FB1D0700700020003D2A07006B
:10C9F000E96FEF0081FE20009140780030C6B3005F
:10CA000080CF500002003C000140E800E8EFB70092
:10CA100020C3B300E84FE3000A003400E76FEF00E3
:10CA20008043EB0007437800874278000742780094
:10CA300087417800074178008740780007407800F8
:10CA4000E41D070081FE200091407800E5CF5000F2
:10CA500019003A00E4CFBF00E14F50000A003A004D
:10CA600070FE200011C0B30090CF100032003A00D9
:10CA700020C0B300E4EFB70000052000F09288006A
:10CA800000FB2F000A003700E24F50002A003A0056
:10CA900070FE200012C0B300904F110026003A0033
:10CAA00002407800E4EFB70000052000F092880013
:10CAB0000093880020003700FECF50000F003A009E
:10CAC00070FE2000E44FE20005003A0024C0B300ED
:10CAD000904F120018003A0010C0B300F1FF370069
:10CAE00021C0B30090CF100013003A00E46FEF00B4
:10CAF0005E32EF006032EF000F00370080C2B300FB
:10CB000080CF50000C003A0070FE200032C0B3000D
:10CB1000904F110008003A0011C0B30001007800E6
:10CB2000E4EFB70000052000F09288006032EF00CB
:10CB300001007800E6EFB70011082000D0928000D5
:10CB4000810F500003003400E0928000810F5000FC
:10CB50000A003C005E32EF006032EF000041EB0063
:10CB60008240780000C2B300D01D07000041EB00F6
:10CB70008240780000C2B300070037000041EB009C
:10CB80008240780002407800C81D07000041EB0099
:10CB90008240780002407800D21D0700E64FE20094
:10CBA00036003200E54FEC00E5EFB70001C6B300F8
:10CBB000814F500001003400E56FEF00E5CFBF006A
:10CBC00004C2B3008444400081CF54000100360009
:10CBD00081C4540002C4B30002444000814F540099
:10CBE000010036000144540026FC0700004578008F
:10CBF0000940780023FC0700804478000840780052
:10CC000020FC07000044780000417800894078004B
:10CC10000A407800971D0700094178008A40780093
:10CC200008407800AF1D07000A417800884078006E
:10CC3000094078009D1D0700E94FEC008040780016
:10CC4000E9EFB700F0C7B30080CF5000B0013A0061
:10CC5000E66FEF00E96FEF000041EB0082407800E3
:10CC6000024078009F1D07000041EB0082407800E1
:10CC7000024078008D1D0700A5013700E94FEC0048
:10CC800000417800E9EFB7004240A90009003400F4
:10CC90008040EB0001407800761D070080C2B300A1
:10CCA000E94FE3009A01340000C8B300E9EFB70090
:10CCB000970137000001FB000201EA004300200059
:10CCC000110009000301D800000178008040EB004A
:10CCD00001407800671D07008D013700E24FEC002E
:10CCE00000417800E2EFB7004240A900090034009B
:10CCF00080407800034078005E1D070080C2B300CA
:10CD0000E24FE3000C00340000CCB300E2EFB700C8
:10CD1000090037008000FB008100EA0022002000AB
:10CD2000110009008200D8008000FD000141780058
:10CD3000034078004F1D0700AF4FE20009003200AA
:10CD4000B24FE20007003200E09280005A12B400B5
:10CD500022002000110009000200D8006009B00084
:10CD600020F88800B04FE2000F003200B34FE2001D
:10CD70000D003200E09280005A12B4002200200020
:10CD8000110009000200D80010F8880051092000A5
:10CD9000810F500002003E00800C200010F8880037
:10CDA000A0F62F00023FB400D092800022F880004D
:10CDB000820F500001003100E06FEF0011F8800099
:10CDC000810F50000200360010C0B300E0EFB70042
:10CDD000E0928000820F500001003100E16FEF000F
:10CDE000810F50000200360010C0B300E1EFB70021
:10CDF00001FE2000914078000104E00002003200B2
:10CE0000E1CF500005003A00E14FE20003003A0094
:10CE100001007800DFEFB7001300370010FE20009C
:10CE200012C0B300904F110004003A000104E0006A
:10CE300002003A00DFEFEF000B003700DFCFBF004A
:10CE40004240A9000200340020C0B30005003700B2
:10CE50000004E00002003D00E0CFB3000100370015
:10CE6000A0C0B300DFEFB700F7FD200097437800C4
:10CE70000704E0000B003A00C0122000F092880086
:10CE800000938800074378008742780004C2B3000B
:10CE90008741780007417800874078000440780097
:10CEA00036003700E1CF53000B003A00C0122000DB
:10CEB000F09288006032EF008043EB000743780077
:10CEC000874278000742780003C2B3000741780028
:10CED0008340780028003700E1CF43000A003A0081
:10CEE0005E32EF00C01220000093880007C2B3003A
:10CEF0000043EB00874278000642780086417800C4
:10CF0000064178001B003700E2CF43000D003A00D5
:10CF100040ED2F00F0928800C0122000009388009E
:10CF20008043EB0006C2B3008742780007427800D6
:10CF300087417800074178008740780007407800F3
:10CF40000E003700E2CF53000E003A00C01220005E
:10CF5000F092880040ED2F00009388008043EB00A2
:10CF600007437800874278000742780087417800BD
:10CF700002C2B3008640780006407800951C070086
:10CF8000E3003700EACF5300E1003A00C01220006E
:10CF9000F092880040ED2F00D7003700DE4FEC0004
:10CFA00000417800DEEFB7004240A90008003400DD
:10CFB00083407800AF1C070080C2B300DE4FE3005F
:10CFC0000B00340000CCB300DEEFB70008003700E0
:10CFD0000000FB000000EA00220020001100090010
:10CFE0000200D8000041780083407800A11C0700AF
:10CFF00005FB200095427800054078000504E0001C
:10D000000400320010C0B30011002000A75EE2004F
:10D01000010032008000EB00A7FEB7000104E00031
:10D020000200320080F32F00A07F880034FB200034
:10D0300014427800044078000404E0000400320048
:10D0400010C0B30011002000A65EE2000100320013
:10D050008000EB00A6FEB7000104E00002003200F1
:10D06000800C2000A07F8800F3FA20009341780014
:10D07000034078000304E0000400320010C0B30055
:10D0800011002000A55EE200010032008000EB00EC
:10D09000A5FEB7000104E00006003200F40FE20034
:10D0A00002003200F42FEF000200370080F32F005F
:10D0B000F62FB40021FB2000914078000140780059
:10D0C0000104E0000400320010C0B3001200200090
:10D0D000A45EE200010032000001EB00A4FEB700F4
:10D0E0000204E00006003200F40FE2000200320009
:10D0F000F42FEF0002003700800C2000F62FB40060
:10D100000304E00003003200100020000104E000EE
:10D1100001003A000000EB00804078000004E000CD
:10D120000300320010002000A35EE2000100320084
:10D130000000EB008000FD00A3FEB7008000FD00B2
:10D140000004E00001003200F62FEF000404E000CC
:10D1500003003200100020000504E00001003A0046
:10D160000000EB00804078000004E0000300320083
:10D1700010002000A25EE200010032000000EB007F
:10D180008000FD00A2FEB7008000FD000004E0006A
:10D1900001003200F42FEF00E19380000100E00075
:10D1A0003E003200F18F50002D00320010003C0094
:10D1B000E68F50003300320006003C00E48F500040
:10D1C0002700320032003C00E28F500032003A006B
:10D1D0001F003700ED8F50002D003200F08F5000FF
:10D1E00028003200E88F50002B003A001E00370064
:10D1F00010052000808F50001B0032000A003C0008
:10D2000010022000808F500017003200000520001F
:10D21000808F50000E00320000022000808F5000EE
:10D220001D003A000A00370060052000808F500082
:10D23000140032000000E800808F5000140032001B
:10D240000080E900808F500013003A00040037008E
:10D25000800C2000F40FE2000800320005003700C7
:10D2600080F32F000800370080F32F00F40FE20056
:10D2700002003200F42FEF0007003700F62FB40051
:10D2800005003700800C2000A07F880002003700D6
:10D29000F42FEF00F62FEF007C32EF008225200004
:10D2A000B07F8000820F500001003400B27F880000
:10D2B00081DA2F00B07F8000810F500001003D0017
:10D2C000B17F8800A07F8000820F500001003400F1
:10D2D000A27F8800A07F8000810F500001003D00E8
:10D2E000A17F8800B07F8000A27F80008200400084
:10D2F000F19288000200500000938800040037007B
:10D30000301F2000800F540090FB340057FC370082
:10D310004F0778004F06BE004F05BE004F04BE0009
:10D32000CF00B10000000600C07F88000000EB00C5
:10D330001EFA0700F80FE20002003200F22FEF00A1
:10D340000300370010002000907F880082F907005A
:10D35000B046200050303700004020005730070012
:10D360008080EB000000E00001003200D17F8000EF
:10D370000100780000000600E80F500002003400B1
:10D380000000400071005000000006008000EB002B
:10D39000E80F500001003400110020000100780067
:10D3A000000006000200FA00F0BF9F00E30F5000EB
:10D3B0001700320006003C00E10F50000E00320062
:10D3C00010003C000000E0000800320016003700AA
:10D3D000E90F50000B003200EA0F50000F0032003E
:10D3E000E40F500010003A000C0037009460A900D0
:10D3F0008460A9001100370094E0A90084E0A9002E
:10D400000E0037009500A9008500A9000B00370029
:10D410009760A9008760A900080037009780A900DD
:10D420008780A900050037008F81E90042102000A5
:10D43000913F2000A0C22A000B3107000080FA00B3
:10D44000000006000400FA00E0BF9F00F1BF9F004B
:10D45000E18F5000040036008F81E9006210200047
:10D46000912220003E0037006FB89700E30F500074
:10D470002800320006003C00E10F5000140032008A
:10D480001B003C000000E0000800320031003700C3
:10D49000E90F50000D003200EA0F50001C0032006E
:10D4A000E40F50002B003A0022003700E1C060007A
:10D4B00081C0400004C1BF000014A1000140700001
:10D4C00004E1B70005A1A9002700370013A1A900B6
:10D4D000E1C0600081C0400010C1BF000014A10085
:10D4E0000140700010E1B70011A1A9001E00370033
:10D4F000E1C0600081C0400012C1BF000014A10063
:10D500000140700012E1B70013A1A9001600370016
:10D5100021A1A900E1C0600081C040001EC1BF0080
:10D520000014A100014070001EE1B7001FA1A90076
:10D530000D003700E1C0600081C0400020C1BF0085
:10D540000014A1000140700020E1B70021A1A90052
:10D5500005003700E481570042102000112620000A
:10D56000A0C22A00C03007000080FA0000000600B8
:10D570000200FA00F0BF9F00E30F500023003200CA
:10D5800006003C00E10F50001200320018003C0081
:10D590000000E000080032002A003700E90F5000C8
:10D5A0000C003200EA0F500018003200E40F500067
:10D5B00024003A001C003700E1C06000C608DD000E
:10D5C00004C1BF000064A1000140700004E1B70085
:10D5D00021003700E1C06000C608DD0010C1BF00B7
:10D5E0000064A1000140700010E1B7001A0037008C
:10D5F000E1C06000C608DD0012C1BF000064A100E8
:10D600000140700012E1B70013003700E1C0600074
:10D61000C608DD001EC1BF000064A100014070000B
:10D620001EE1B7000C003700E1C06000C608DD0055
:10D6300020C1BF000064A1000140700020E1B700DC
:10D64000050037008F81E9004210200041292000A9
:10D65000A0C22A00843007000080FA000000060003
:10D660000200FA00F0BF9F0001417800EA0F50006D
:10D670001A003E0010002000FFB897008100DD0076
:10D68000010078006020B20006003A0080412000CE
:10D69000008060000A003A000108A30014003A006C
:10D6A0000E003700E1406100C308DD0010C1BF007B
:10D6B0000034A1000140700010E1B7000C003700F9
:10D6C000E1406100C308DD001EC1BF000034A100BD
:10D6D000014070001EE1B700050037008F81E900AE
:10D6E00042102000A1462000A0C22A005E300700A0
:10D6F0000080FA00000006000200FA00F0BF9F0060
:10D70000E30F50002C00320006003C00E10F5000F7
:10D71000150032001E003C000000E000080032004E
:10D7200039003700E90F50000F003200EA0F5000B7
:10D7300021003200E40F500033003A002800370087
:10D7400063C060004400DD0041102000914078007B
:10D75000F2CCB30082C0600080C07000010078008D
:10D7600004E1B7002D00370063C060004400DD0015
:10D770000111200091407800F2CCB30082C060001B
:10D7800080C070000100780010E1B700230037006E
:10D7900063C060004400DD0021112000914078004A
:10D7A000F2CCB30082C0600080C07000010078003D
:10D7B00012E1B7001900370063C060004400DD00CB
:10D7C000E111200091407800F2CCB30082C06000EB
:10D7D00080C07000010078001EE1B7000F00370024
:10D7E00063C060004400DD00011220009140780019
:10D7F000F2CCB30082C0600080C0700001007800ED
:10D8000020E1B700050037008F81E90042102000B9
:10D81000214A2000A0C22A00133007000080FA002D
:10D82000000006000200FA00F0BF9F00E30F500066
:10D830001600320006003C00E10F50000E003200DE
:10D840000F003C000000E000080032001300370029
:10D85000E90F500007003200EA0F50000A003200C2
:10D86000E40F50000D003A000A003700020888005B
:10D870000F00370043088800320888000C0037008A
:10D88000520888000A003700B3088800A208880000
:10D8900007003700C2088800050037008F81E900C3
:10D8A00042102000D11E2000A0C22A00EE2F070047
:10D8B0000080FA00000006000200FA00F0BF9F009E
:10D8C000E30F50001800320006003C00E10F50004A
:10D8D0000D00320012003C000000E00008003200A1
:10D8E0001E003700E90F50000A003200EA0F500016
:10D8F0000F003200E40F500018003A001500370006
:10D90000000880000100370030088000010020007E
:10D9100017003700320880004008800006003700FA
:10D9200050088000F9FF3700A0088000F7FF37009B
:10D93000A2088000B0088000030020000100200041
:10D94000C000DD0000002000000071008180710037
:10D9500007003700C0088000ECFF37008F81E90026
:10D960004210200051212000A0C22A00BE2F070033
:10D970000080FA00000006000200FA00F0BF9F00DD
:10D98000E30F50001F00320006003C00E10F500082
:10D990001100320016003C000000E00008003200D8
:10D9A00024003700E90F500011003200EA0F500048
:10D9B0001A003200E40F50001E003A001700370032
:10D9C00094C0BF004300DE00610060009460A800C6
:10D9D0008460A8001C00370094C0BF000080FB00DA
:10D9E0004700DE0094E0A80084E0A800160037009D
:10D9F00095C0BF00610060009500A8008500A800E8
:10DA00001100370097C0BF004300DE0061006000D6
:10DA10009760A8008760A8000B00370097C0BF0080
:10DA20004400DE00610060009780A8008780A800A5
:10DA3000050037008F81E90042102000F1332000FB
:10DA4000A0C22A00882F07000080FA00000006000C
:10DA50000200FA00F0BF9F00E30F500016003200F2
:10DA600006003C00E10F50000D00320010003C00A9
:10DA70000000E0000800320016003700E90F5000F7
:10DA80000B003200EA0F50000E003200E40F50008D
:10DA900010003A000B00370084C0BF0007003700B9
:10DAA00084C0BF000080FB004700DE000E0037008E
:10DAB00085C0BF000500370087C0BF004300DE00FF
:10DAC0000200370087C0BF004400DE006100600034
:10DAD000050037008F81E900421020001137200037
:10DAE000A0C22A00602F07000080FA000000060094
:10DAF0000200FA00F0BF9F00E30F50002700320041
:10DB000006003C00E10F5000130032001B003C00F7
:10DB10000000E0000800320032003700E90F50003A
:10DB200016003200EA0F500024003200E40F5000CB
:10DB30002C003A002100370084C0BF004300DE0003
:10DB400061016000E1C06000C308DD0084C0BF0067
:10DB50000034A1000600370084C0BF000080FB0035
:10DB60004701DE00C708DD0084C0BF000074A100CB
:10DB70000140700084E0B7001F00370085C0BF007F
:10DB800061016000E1C0600085C0BF000004A10029
:10DB90000140700085E0B7001700370087C0BF0064
:10DBA0004300DE0061016000E1C06000C308DD00E9
:10DBB00087C0BF000034A1000700370087C0BF0046
:10DBC0004400DE0061016000E1C06000C408DD00C7
:10DBD00087C0BF000044A1000140700087E0B7008B
:10DBE000050037008F81E90042102000613B2000D2
:10DBF000A0C22A001C2F0700020078000080FA0053
:10DC0000000006000200FA00F0BF9F00E30F500082
:10DC10001400320006003C00E10F50000D003200FD
:10DC20000E003C000000E000080032001100370048
:10DC3000E90F500007003200EA0F500009003200DF
:10DC4000E40F50000B003A000800370004C1BF0089
:10DC50000D00370010C1BF000B00370012C1BF001C
:10DC6000090037001EC1BF000700370020C1BF00F8
:10DC7000050037008F81E90042102000914220000A
:10DC8000A0C22A00F82E07004400DE0063006000F6
:10DC9000E10F50000900320006003900E20F500089
:10DCA00008003200E30F500007003A000010200087
:10DCB000050037001000200003003700800020001E
:10DCC00001003700000420000080FA000000060078
:10DCD000EF02B000889FBE008A9FBE008C9FBE00EE
:10DCE0008E1F780080B79F0092B79F00A3B79F0058
:10DCF000B1B79F006000B8006011B800C0A79F00D6
:10DD0000D1A79F00E2A79F00F3A79F0061FC2F000F
:10DD10008F8040006A80400022C42A00070009006A
:10DD2000321878000001B1008FB69700EC8F5600D2
:10DD300004003600FA81400042102000211020002B
:10DD40000F003700E88F560002003C000D007800FD
:10DD5000020037000D804600710050004200DD00D7
:10DD600081E22100608078000018A30006003A00DC
:10DD700000FE2F008F0140003210200061102000B3
:10DD8000A0C22A00B82E07003FB697000C00E000A2
:10DD900012003200E30F560010003200E60F56006A
:10DDA0000E003200E90F56000C003200E10F460071
:10DDB0000A003200E20F460008003200E30F46007E
:10DDC00006003200E40F460004003200FA815700DA
:10DDD00052102000B1102000E9FF37000C00E000D5
:10DDE000150035001FB49700AFB497006055B80018
:10DDF0000007EB0009003700A40020000500200008
:10DE00006033B8000800BE000A01BE00B1CA0700B6
:10DE10000205BE000004BE000E07E80069001600FF
:10DE2000800F5700F4FF3500C8A79F00D9A79F00B7
:10DE3000EAA79F00FBA79F00E88F560083003C00E5
:10DE40008040EB000D00780005FE07003FB0970012
:10DE50000000E000510035004FA49700DFA49700B8
:10DE60006FA59700FFA5970038E007006011B80084
:10DE70000040E10001C8E10002D0E10003D8E10068
:10DE8000130039004FA49700DFA497006FA59700F7
:10DE9000FFA597002DE007006011B80004F02F00E7
:10DEA000F50F20006033B8008ACA07000040E10087
:10DEB00001C8E10002D0E10003D8E10004003E0007
:10DEC0000006EB0001FD2F008F86400006003700A2
:10DED00082FC2F008F01410012102000D111200080
:10DEE000A7FF37000C06E8004FA49700DFA49700B7
:10DEF0006FA59700FFA5970014E007003D01BE0045
:10DF0000C2B79F00D3B79F008001EB00E3B79F002B
:10DF1000F3B79F000001EB004FB29700DFB297000C
:10DF20006FB39700FFB397006ACA0700F4FF2F0092
:10DF3000050020006033B80066CA07000040E10019
:10DF400001C8E10002D0E10003D8E100E5FF3E0096
:10DF50004FA49700DFA497006FA59700FFA5970037
:10DF6000FADF07006011B8004FB29700DFB29700E8
:10DF70006FB39700FFB3970056CA07000203BE00B5
:10DF80000002BE000800BE000A01BE00F9CA070078
:10DF90000205BE000004BE000B0037000086EA0048
:10DFA0001FB09700AFB09700E10F4000E08F58001E
:10DFB00004003600FE81570012102000711220006C
:10DFC0006FFF37000004BE000FB097008C00780090
:10DFD000C9FD07000FB09700B0A79F00E20F5000E7
:10DFE0000F00320005003C000000E0000800320095
:10DFF000E10F500010003A0007003700E30F500017
:10E0000009003200E40F50000B003A00080037000E
:10E010001808880079003700680888007700370002
:10E020007808880075003700D8088800730037002A
:10E03000E80888007100370063FC2F008F814100E1
:10E0400042102000014D20004DFF370011C0B300E9
:10E050000D00780082FD07003FB097000000E0004F
:10E060004D0035004FA49700DFA497006FA59700DF
:10E07000FFA59700B5DF07006011B8000040E10080
:10E0800001C8E10002D0E10003D8E1001500390029
:10E090004FA49700DFA497006FA59700FFA59700F6
:10E0A000AADF07006011B80004F02F00F5FF2F0071
:10E0B000F60F20000700200006CA07000040E1001C
:10E0C00001C8E10002D0E10003D8E10005003E00F4
:10E0D0000007EB0000FD2F000F00400080BF9F00F5
:10E0E0000600370081FC2F008F81400012102000B5
:10E0F000A113200022FF37000E07E8004FA497006D
:10E10000DFA497006FA59700FFA597008FDF07009A
:10E110000FB997003206BE0082BF9F000C01BE00FF
:10E12000BFC907000002BE006033B8000800BE008F
:10E130000A01BE008FCA0700F4FF2F00F5FF2F0071
:10E140006033B8000400E1000588E1000690E100BA
:10E150000798E100E8FF3E004FA49700DFA4970076
:10E160006FA59700FFA5970078DF07000002BE00AB
:10E170006033B8000800BE000A01BE007DCA070077
:10E180000C02BE006033B8007ACA07000205BE0068
:10E190000004BE00030037000087EA001FB49700A8
:10E1A000AFB497000FB097008E00780052FD0700C3
:10E1B0000800BE000FB19700B2A79F00E90F510001
:10E1C00003003200EA0F510007003A000300370055
:10E1D000680888007108880008003700D80888009F
:10E1E000E10888000500370063FC2F008F814100A3
:10E1F00042102000A14F2000E1FE37000FB0970031
:10E200006011B80087FD07004F0778004F06BE0079
:10E210004F05BE004F04BE00EF02B1000000060033
:10E22000E80F500002003400000040007100500070
:10E23000C200DD0080E22100610078006100600022
:10E24000000006000200FA00F0BF9F000001BE00BF
:10E25000EC0F5000040036008F81E90042102000CE
:10E26000E11920000C003700E80F500002003400D4
:10E2700000004000710050004200DD0081E22100FA
:10E28000608078000018A30005003A008F81E90043
:10E2900032102000211A2000A0C22A00722D07008F
:10E2A000E30F51002000320006003C00E10F510056
:10E2B0001100320016003C000200E00008003200AD
:10E2C00025003700E90F51000B003200EA0F510022
:10E2D00015003200E40F51001F003A00180037000B
:10E2E000C718DD0005C1BF000074A1000140700027
:10E2F00005E1B7001C003700C718DD0011C1BF00E1
:10E300000074A1000140700011E1B7001600370051
:10E31000C718DD0013C1BF000074A10001407000E8
:10E3200013E1B70010003700C718DD001FC1BF00A0
:10E330000074A100014070001FE1B7000A0037001F
:10E34000C718DD0021C1BF000074A10001407000AA
:10E3500021E1B700040037008F81E900421020005E
:10E36000511C2000CCFF37000080FA00000006009E
:10E370008000EB00B3FF370011002000B1FF370031
:10E380000400FA00E0BF9F0001027800F2BF9F0086
:10E3900000017800EC0F500004003600E4815700C3
:10E3A00042102000812A200007003700FFB99700A3
:10E3B0000300E900E60F5000050036008F81E900F8
:10E3C00022002000912A2000A0C22A00262D07004A
:10E3D000E80F510002003C00020078000200370004
:10E3E0000200410071005000C200DD0060E2210027
:10E3F00084307800E30F51003100320006003C0009
:10E40000E10F51001700320022003C000200E00042
:10E410000800320041003700E90F51001D003200B2
:10E42000EA0F510032003200E40F51003B003A0085
:10E430002F00370067C061004400DD00510A200052
:10E4400091407800F2C8B30082C0600080C07000C4
:10E4500001007800A5E0B7008460A9009460A800DE
:10E460003200370067C061004400DD00710A2000FF
:10E4700091407800F2C8B30082C0600080C0700094
:10E4800001007800A7E0B70084E0A90094E0A800AC
:10E490002600370067C06100810A200091407800A3
:10E4A00082CFB30082C0600080C07000010078009D
:10E4B000A8E0B7008500A9009500A8001B00370060
:10E4C00067C061004400DD00110B2000914078001E
:10E4D000F2C8B30082C0600080C070000100780004
:10E4E000B1E0B7008760A9009760A8000F0037006F
:10E4F00067C06100210B20009140780082CFB300FB
:10E5000082C0600080C0700001007800B2E0B700F7
:10E510008780A9009780A80004003700E481570095
:10E5200042102000D12E2000A7FF37000080FA0003
:10E53000000006000200FA00889FBE008A1F7800D3
:10E54000C0BF9F000204BE000105780000017800F2
:10E55000EC0F500004003600E88157004210200004
:10E56000210C20000C003700E80F5000020034009E
:10E5700000004000710050004200DD0081E22100F7
:10E58000608078000008A30005003A00E881570089
:10E5900022102000610C2000A0C22A00B22C07002B
:10E5A000E80F510002003C00020078000200370032
:10E5B0000200410071005000C201DD000380E8004C
:10E5C00064E22100840040001110A0001100A100AD
:10E5D000E80F51000500340066804100040040004F
:10E5E0001000A1001120A000010037001120A1009F
:10E5F000020078006BFB07008A0078000801BE006B
:10E600004FB89700B2FD07008000EB004FB89700AD
:10E610008CFB07008000EB004FB89700D4FB07008D
:10E620004F0578004F04BE000080FA00000006008D
:10E630000200FA00F0BF9F0080007800EC0F50004D
:10E64000050036008F81E90042102000E11520000E
:10E65000A0C22A00842C0700E80F500002003400FA
:10E6600000004000710050004201DD000280E8001F
:10E6700063E22100030040001010A1001000A00080
:10E68000E88F5000030034006600410003004000A2
:10E690001000A0000080FA00000006009008900022
:10E6A000E001900001814000628179008100E90071
:10E6B0001108980002007800000006000200FA002D
:10E6C000889FBE0080047800010478000000E0000C
:10E6D00005003A00000028000100E000620035005B
:10E6E0000900780060003700010378000100E000B5
:10E6F00001003D000103EA00090078000900E00084
:10E7000001003D000900EA00010024000800E000CB
:10E7100050003200CF80DE0066815700811F7800F4
:10E72000110009004688D80001097800CF00780060
:10E73000DFB89700610AB800C021DD0002002000A8
:10E74000809FBE00110009004699D80000017800A2
:10E750004F00BE00020278008002780040A8DE0070
:10E76000CF80DE008080CF000100E0000300320097
:10E770000002200001015000040037000281CF0098
:10E780000200E0000100320070011100EC015100B4
:10E790000A003B00C2282000030020000400BE0045
:10E7A0001FC80700440BDD004C00DE0000007300B2
:10E7B000CC88DE00800078002200370010002000A6
:10E7C00001002000020378000603E9000300330083
:10E7D0000000400081804800FBFF3700000052002D
:10E7E00081805A00680151000201E90003003300F2
:10E7F0008180D1000080D300FBFF37007F036000E1
:10E800004319DD004580DE000001410002014100A6
:10E8100021FB29006282780003022000068051005B
:10E8200000A2B9000281E800628078000680B90089
:10E83000040240008582480011000900432AD800E4
:10E84000800078000800E00002003D000000280081
:10E85000810050000900E00002003400010078004F
:10E86000010037000100EA004F04BE000080FA00FA
:10E8700000000600800078000000E0000C003D0071
:10E8800002002C00820F500003003D000000280011
:10E89000008040000400370010002800828F5000E4
:10E8A000200034000100EA001700200008003700B3
:10E8B00000002400808F500002003C00010078001E
:10E8C0000200370000002800010050008003EB0028
:10E8D0004781DE0000027800F407B2000201410027
:10E8E00006EB29000008200004005000E2017B0034
:10E8F0000380B9000281E80062017B0002A2B90036
:10E900000000420081804A004909DD004700DE0026
:10E9100000007100C788DE000700E000010032003F
:10E920000000EA0000000600010024000100400091
:10E93000D0FF37000100240001003700C288DE004C
:10E94000808F5000FDFF3C00800178000000EB004C
:10E9500007003700010140000080D100828F510084
:10E96000020035008281510001004000C288DE00B3
:10E970000100E000F7FF3A0000000600889FBE009B
:10E980008A1F780080047800010478000102780072
:10E990008003EB005A002000190037006420B80003
:10E9A000809FBE00110009004A88D800000278004C
:10E9B0004F00BE00890078000400420080814400BE
:10E9C000840278008003EB000B003700110378000D
:10E9D00013017800020053004240A90003003400F4
:10E9E0008208780086097800170020008502E80078
:10E9F0008180E8008381E800888F5200F3FF3900AE
:10EA0000E10F5200E5FF3E000700E000E9FF3A0099
:10EA10004F0578004F04BE0000000600889FBE002E
:10EA20008A1F7800000578001CFF0700800478002A
:10EA30000A00780019FF0700000478000A00780037
:10EA400016FF070000027800098144008800440096
:10EA50008001EB00050037004A009000613178002A
:10EA60008301E8000281E8008180E800848F510082
:10EA7000F9FF39004F0578004F04BE000000060082
:10EA8000889FBE008A1F78000005780003FF0700FA
:10EA9000800478000A00780000FF07000004780076
:10EAA0000A007800FDFE0700800178000804440099
:10EAB000898044000001EB00040037004A00900008
:10EAC000E83078000201E8008180E800830F5100FF
:10EAD000FAFF39004F0578004F04BE000000060021
:10EAE000889FBE008A9FBE0080057800EBFE07006D
:10EAF000800478000B007800E8FE0700000478002E
:10EB00000B007800E5FE0700000578000B00780098
:10EB1000E2FE0700800278004B0090008A0045006A
:10EB20006102780089844400080144008001EB0000
:10EB300007003700CB0090006280780000004200A0
:10EB400080B478008301E8008984E8000281E8004D
:10EB5000858F5100F7FF39004F05BE004F04BE00FE
:10EB600000000600889FBE008A9FBE0080057800D6
:10EB7000CAFE0700000578000B007800C7FE0700FA
:10EB8000800478000B007800C4FE070000047800C1
:10EB90000B007800C1FE0700000278000A0545005E
:10EBA00089844400080444008001EB000900370018
:10EBB0004B009000E90078006801780082804000F6
:10EBC000013578008301E8000A85E8008984E800BF
:10EBD0000884E800848F5100F5FF39004F05BE001E
:10EBE0004F04BE0000000600889FBE008A9FBE0042
:10EBF00080057800A9FE0700000578000B0078006A
:10EC0000A6FE0700800478000B007800A3FE070032
:10EC1000000478000B007800A0FE070000027800D6
:10EC20000A05450089844400080444008001EB0083
:10EC3000090037004B009000E90078006801780077
:10EC400082805000013578008301E8000A85E800E1
:10EC50008984E8000884E800848F5100F5FF3900BA
:10EC60004F05BE004F04BE0000000600889FBE0096
:10EC70008A9FBE008C1F78008005780087FE070001
:10EC8000000578000B00780084FE070080047800FF
:10EC90000B00780081FE0700000478000B0078006C
:10ECA0007EFE0700000678000A03450089824400C2
:10ECB000080244008003EB00090037004B0090007D
:10ECC00065017800E40078000191B9000233780012
:10ECD0008703E8000683E8008582E8000482E800F4
:10ECE0008C8F5300F5FF39004F0678004F05BE00AA
:10ECF0004F04BE0000000600889FBE008A9FBE0031
:10ED00008C9FBE008E1F78008005780063FE070090
:10ED1000000578000B00780060FE07008004780092
:10ED20000B0078005DFE0700000478000B007800FF
:10ED30005AFE0700000778000A06450009854400CE
:10ED4000880444008006EB00160037004B04900056
:10ED50006A007C006102B90069007C006101B900B1
:10ED60000A85E8008984E8000000E000060032001F
:10ED70000400BE00C8C6070000367C008D06E8000F
:10ED80000C86E8000700370023002000F3059800F8
:10ED900070814500710029000B0078009C1B070062
:10EDA000020037008E8F5600E8FF39004F077800C9
:10EDB0004F06BE004F05BE004F04BE000000060017
:10EDC000889FBE008A9FBE008005780033FE070042
:10EDD000000578000B00780030FE07008004780002
:10EDE0000B0078002DFE0700000478000B0078006F
:10EDF0002AFE070009834400880244000A024500F5
:10EE00008003EB000B0037004B019000E601790016
:10EE1000E5007900838F5000010034008300780002
:10EE2000013279008703E8000683E8008582E80064
:10EE30000482E800808F5300F3FF39004F05BE00C5
:10EE40004F04BE0000000600889FBE008A9FBE00DF
:10EE50008005780011FE0700000578000B0078009F
:10EE60000EFE0700800478000B0078000BFE070000
:10EE7000000478000B00780008FE070009834400B6
:10EE8000880244000A0245008003EB000B003700B3
:10EE90004B019000E6017900E5007900838F500076
:10EEA00001003D0083007800013279008703E8000B
:10EEB0000683E8008582E8000482E800808F530022
:10EEC000F3FF39004F05BE004F04BE0000000600EE
:10EED000889FBE008A9FBE008C9FBE008004780081
:10EEE000EEFD07000005780009007800EBFD070043
:10EEF0000006780009007800E8FD0700800578002A
:10EF00004904900009007800E4FD0700000040007B
:10EF100060047C0009007800E0FD070080067800AE
:10EF200000022000800F540005003C000B834500C8
:10EF30008C0146006022B8008003EB000D00370012
:10EF4000C90090000A004500010040000008EB00E5
:10EF50001200370063807800668178000280B90073
:10EF600004024000858248008703E8000683E80029
:10EF70008381E800C90090008D8F5300F5FF3900B0
:10EF80000A0045000804E900030033008582D1002F
:10EF90000482D300FBFF370004B078004F06BE00A8
:10EFA0004F05BE004F04BE0000000600889FBE0053
:10EFB0008A9FBE008C1F780000047800B7FD070010
:10EFC0008004780008007800B4FD07008005780010
:10EFD00008007800B1FD07000005780008007800FF
:10EFE000AEFD07000006780008007800ABFD0700C2
:10EFF000000378000000E00024003200C800900008
:10F0000009804400608078006102B9008B8545006A
:10F0100080B578000A05450000B578000900E800D1
:10F020008001400017002000010178000F00370028
:10F03000E30079000B004100908F500001003D007B
:10F04000010878004800900000004500908F5000B3
:10F0500001003400010878006108B9000402400092
:10F06000858248008703E8008381E800868F53008B
:10F07000EFFF39000C044600020444006131B8007F
:10F080000400BE0004C60700000C78004F0678009C
:10F090004F05BE004F04BE0000000600889FBE0062
:10F0A0008A9FBE00800478007CFD07008005780000
:10F0B0000900780079FD0700000578000900780054
:10F0C00076FD0700000478000900780073FD070052
:10F0D000000278000000E0001600320088034400BF
:10F0E0008A0245000B814500F8FF27000600280032
:10F0F0008001EB000D00370049009000E20078002D
:10F10000888F500002003D008332780001047800AF
:10F11000868F50000300340049009000833378004C
:10F12000010378008301E8000281E800848F510028
:10F13000F1FF39004F05BE004F04BE00000006007D
:10F14000889FBE000004780054FD0700800478000A
:10F150000800780051FD0700800078000981440014
:10F16000480090000000410004FE07004F04BE006C
:10F1700000000600E8874700889FBE008A9FBE0007
:10F180008C9FBE008E1F78000006780043FD0700AC
:10F19000800578000C00780040FD0700000578002D
:10F1A0000C0078003DFD0700800478000C0078001A
:10F1B0003AFD0700000478000C00780037FD0700D6
:10F1C00080BF9F008B854500EBB79F000A07450075
:10F1D00089864400880444000000EB00F0B79F00DB
:10F1E0001F0037004C0490006E007C006102B900E3
:10F1F0006D007C006101B90069007C006105B90007
:10F200000E87E8008D86E8008984E8000000E000B1
:10F210000C0032000400BE0081C507000A01BE00D8
:10F220009DC507006FB1970000317C007FB097004B
:10F230000000E800F0B79F000281E800E2B79F00FD
:10F240000700370023002000730698007001460075
:10F25000710029000C0078006D1A070004003700C7
:10F26000FFB097000FB99700828F5000DDFF390083
:10F270004F0778004F06BE004F05BE004F04BE008A
:10F280008F00B10000000600889FBE008A9FBE006C
:10F290008C9FBE008E1F780000067800FFFC0700E0
:10F2A000000578000C007800FCFC07008004780062
:10F2B0000C007800F9FC0700000478000C007800CE
:10F2C000F6FC0700000778008985440088044400A4
:10F2D0000A0545008006EB00090037004C04900049
:10F2E000E9007C006B007C00F4FC070000357C002A
:10F2F0008D06E8008B85E8008984E8000A85E8002F
:10F300008E8F5600F5FF39004F0778004F06BE007C
:10F310004F05BE004F04BE0000000600889FBE00DF
:10F320008A9FBE008C9FBE0080057800DBFC070032
:10F33000800478000B007800D8FC070000047800F7
:10F340000B007800D5FC0700800678000805440013
:10F35000898444000006EB00070037004B0490004E
:10F360006A007C0043FD070080347C000C06E80046
:10F370000A85E8008984E8008D0F5600F7FF390000
:10F380004F06BE004F05BE004F04BE000000060041
:10F39000889FBE008A9FBE008C9FBE0080057800BB
:10F3A000BEFC0700800478000B007800BBFC07005F
:10F3B000000478000B007800B8FC07008006780095
:10F3C00008054400898444000006EB00070037006C
:10F3D0004B0490006A007C0053FD070080347C00E1
:10F3E0000C06E8000A85E8008984E8008D0F5600C5
:10F3F000F7FF39004F06BE004F05BE004F04BE00A8
:10F40000000006000C00FA00889FBE008A9FBE0024
:10F410008C9FBE0000047800A0FC070080057800E7
:10F42000080078009DFC0700800478000800780040
:10F430009AFC0700480590008984440000004000C1
:10F4400060047D000800780037FD07006101B90005
:10F4500082BF9F0093BF9F0069007D006101B900DA
:10F46000E2B79F00F3B79F000800780001FD070096
:10F470006101B900C2B79F00D3B79F0009004500E2
:10F48000100090006106B9008B8545006FB19700B0
:10F49000FFB197000FB897009FB89700E0C407002E
:10F4A0000004BE000C01BE004FB09700DFB0970013
:10F4B000DBC407000004540081845C00C149DD0006
:10F4C0004F44DE0008847100CFCCDE0088357D001B
:10F4D0000B0545000C01BE000FB897009FB89700C0
:10F4E000CFC407000004BE006FB19700FFB19700C2
:10F4F0004FB09700DFB09700C9C407000804400070
:10F50000898448004148DD004F44DE000804700053
:10F51000CFCCDE00180598004F06BE004F05BE0098
:10F520004F04BE000080FA0000000600889FBE0065
:10F530008A9FBE008C9FBE008005780057FC0700A4
:10F54000800478000B00780054FC07000004780069
:10F550000B00780051FC0700800678000805440085
:10F56000898444000006EB00070037004B0490003C
:10F570006A007C00EFFC070080347C000C06E80089
:10F580000A85E8008984E8008D0F5600F7FF3900EE
:10F590004F06BE004F05BE004F04BE00000006002F
:10F5A000889FBE008A9FBE008C9FBE00000478002A
:10F5B0003AFC0700000578000800780037FC0700D7
:10F5C000800578000800780034FC0700800478008B
:10F5D0000800780031FC070000027800C8029000A3
:10F5E00009804400E0847A000B80450000804200DE
:10F5F0008000EB00040037008100E8000080E80094
:10F60000848F500048003E001000E000FAFF3A00EE
:10F610000180450000004000008042000080E800BA
:10F62000810378008703E800848F530009003600C7
:10F630000100E000400032000100E9000A0145003D
:10F64000890F5000400039000000D10000B17A005D
:10F65000430037003000E000F2FF32000003EB000F
:10F6600006047800860678002C002000868143007E
:10F6700006017800040037000201E8008301E80079
:10F68000840F510008003100110009008481D80066
:10F690008000FD000B00400000004000050040001D
:10F6A0001000E000F4FF3A0086005100888F5000FF
:10F6B0000700340006004100811F78001100090096
:10F6C0000C00D80080067800CF0078000104780094
:10F6D000840F510010003100828143000400370084
:10F6E0000201E8008301E800840F51000A003100A4
:10F6F000110009008481D8008000FD000B0040004B
:10F7000000004000050040001000E000F4FF32005F
:10F7100002037800D5FF37000A014500890F540025
:10F720000B003D00080037000A00450005004000BE
:10F730000008EB000A0037000A0045000500400001
:10F740000088EB000600370005004100FCFF370091
:10F750000D804300110009000480D80001B17A0037
:10F760004F06BE004F05BE004F04BE00000006005D
:10F77000A0FA880000000600A2FA800050252600AA
:10F780000091B9009061230002004000A0FA8800B7
:10F7900000000600889FBE0080047800BFFB0700C1
:10F7A0000004780009007800BCFB07000002780024
:10F7B000A0FA8000080444008001EB0056252600D2
:10F7C00095612300060037000680B90000804200E2
:10F7D00049019000003479008301E8000884E800C2
:10F7E000848F5100F8FF3900A0FA88004F04BE0052
:10F7F000000006000080FB00C300DE00B27F240092
:10F8000002814000C308DD0001005000110020000B
:10F810008008DD0012C9700000000600F0F98000C9
:10F8200001FA800061014000E0814800F2F988009F
:10F8300003FA880000302A0021002000800F5100C8
:10F84000818F590007003A003E3FEF00403FEF0034
:10F85000A17F240011407800E14F400001003200F8
:10F860008048E800000006000001EB0011022100C2
:10F87000000120004427070061012000807E240051
:10F880005227070073270700F03F8A000000060098
:10F8900020C0B300D7FF370011FA80008100E800D4
:10F8A00011FA880000A62E00808F500027003A0031
:10F8B000423FEF00403F8200E10F40000200320073
:10F8C0000000E800403F8A00A3F607000000E000C7
:10F8D00006003D00917F240011407800E14F400078
:10F8E000090032008048E80007003700E8004000C7
:10F8F000807E24000080400010417800E14F4100EC
:10F90000010032000248E80084C4BF000038A300B0
:10F910000E003200D32507000000E0000600320090
:10F92000503F8200E10F4000080032000000E80074
:10F93000503F8A0000000600603F8200E10F400057
:10F94000020032000000E800603F8A00000006006C
:10F950008000780060042000808F50000B00390088
:10F960000000E800808F5000040036007000400066
:10F97000808F500005003A000200370070C0B300CD
:10F980009CFF370000C1B3009AFF0700000006008B
:10F990008000780020052000808F50000E003E007F
:10F9A0000080E900808F50001A003100A002200082
:10F9B000808F50001F00390064004000808F50008D
:10F9C0001000360070FC2F0000804000EC0F50004B
:10F9D00018003E000D00370050052000808F5000B9
:10F9E00004003E000000E900808F50000D0031004F
:10F9F0000A00370060052000808F50000D003A009B
:10FA00000A003700F0C0B3000700370080C0B30021
:10FA100005003700E0C0B3000300370090C0B3001A
:10FA20000100370010C1B30072FF370000C1B300FE
:10FA300070FF070000000600889FBE008A1F780044
:10FA40000005EB00180020002900200011D58000DF
:10FA500000D58000910F100031003600950037006E
:10FA6000E9007800E0FF2F000100500001002000B5
:10FA7000EF0F5000E08F580021003E0000600100B1
:10FA80000F0037000E0037000D0037000C00370064
:10FA90000B0037000A0037000B0037000C0037005E
:10FAA0000B0037000C00370015003700100037003E
:10FAB0000B0037000C0037000F0037000E00370036
:10FAC000F0C0B3000D00370080C0B3000B0037005A
:10FAD000E0C0B3000900370000C1B30007003700E1
:10FAE00010C1B3000500370070C0B3000300370039
:10FAF00040C1B3000100370050C1B3003DFF070013
:10FB000009007800A21AB400100090008A0F50007B
:10FB100001003600000578000884E800E484440011
:10FB200010D58000900F5400CDFF39005E003700E3
:10FB300014D580008801440063017A004C10DE0077
:10FB400001002000ED0F5000E08F580055003E00EE
:10FB5000006001000D003700520037001D00370023
:10FB60000D00370010003700130037001600370073
:10FB70004C0037004B0037001800370015003700E5
:10FB80001A003700240037001D0037008A0F540088
:10FB90004800310043003700F0FF20000000610002
:10FBA0007BFF07003F003700F0FF200000006100EE
:10FBB00067FF07003B003700F0FF200000006100F6
:10FBC00073FF070003003700F0FF20000000610012
:10FBD0005FFF07000884E800330037004410DD00B1
:10FBE0004480DE00000044000700370003004200AC
:10FBF0001000900066FF0700630444002A003700ED
:10FC0000F0FF2000000061008A0F50002500360040
:10FC10000005780023003700F0FF2000000061009D
:10FC2000010020007A005000E0805800ED0F5000E5
:10FC3000E08F58001B003E00006001000D003700FF
:10FC40000C0037000B0037000C0037000D003700A8
:10FC50000C0037000B003700060037000B003700A0
:10FC60000C0037000B0037000C0037000B0037008A
:10FC70000A003700A0C0B30009003700D0C0B300AD
:10FC800007003700C0C0B3000500370020C1B30033
:10FC900003003700B0C0B3000100370030C1B3002B
:10FCA000D4FE07000804E80000D58000800F54004F
:10FCB0009FFF39004F0578004F04BE00000006008A
:10FCC000F17E240011407800E14F40000100320035
:10FCD0008048E80058FF3700889FBE008A9FBE001A
:10FCE0000004BE0000402000010020000805400084
:10FCF000898548000B0037000800BE00001307008C
:10FD0000F2FF2F00F30F2000820F5000838F580066
:10FD10000200320010002000060037006204440098
:10FD2000E0844C008A0F54008B8F5C00F2FF390096
:10FD30000000EB004F05BE004F04BE0000000600AF
:10FD40004A00FA00881F78008A9FBE008C9FBE0080
:10FD500055FC2F000F8242000006BE0092BF9F009C
:10FD6000A3BF9F00E00F5100E08F590005003A004B
:10FD7000D20220008000EB00040078004AC4070093
:10FD8000DC00370084017800D20220001FB8970001
:10FD9000AFB89700F01207004FE897000040E80066
:10FDA000C0EF9F001FB89700AFB897007E054000D6
:10FDB000E0854800C600370001FB2F000F8440009B
:10FDC00088017800520120000A00BE00E2120700FC
:10FDD0001FE89700EF7097000140700090EF9F00C0
:10FDE0002FE89700FF70970001407000A0EF9F0080
:10FDF0003FE897008F78970001407000B0EF9F00B8
:10FE0000FFE097008180FB000FE897004800DD00CD
:10FE100001007000BFC097008180FB00010040001E
:10FE2000F0E79F004800DE0080EF9F00DFE09700D2
:10FE30008180FB006FE097004800DD00010070004A
:10FE4000AFC097008180FB0001004000D0E79F0019
:10FE50004800DE00E0E79F00BFE097008180FB00E4
:10FE60004FE097004800DD00010070009FC0970040
:10FE70008180FB0001004000B0E79F004800DE00E9
:10FE8000C0E79F009FE097008180FB002FE0970074
:10FE90004800DD00010070008FC097008180FB00EA
:10FEA0000100400090E79F004800DE00A0E79F00AF
:10FEB000FFD897008180FB000FE097004800DD002D
:10FEC00001007000FF7897008180FB000100400076
:10FED000F0DF9F004800DE0080E79F00DFD897003A
:10FEE0008180FB006FD897004800DD0001007000A2
:10FEF000EF7897008180FB0001004000D0DF9F0079
:10FF00004800DE00E0DF9F00BFD897008180FB0043
:10FF10004FD897004800DD0001007000DF7897009F
:10FF20008180FB0001004000B0DF9F004800DE0040
:10FF3000C0DF9F009FD897008180FB002FD89700DB
:10FF40004800DD0001007000CF7897008180FB0041
:10FF50000100400090DF9F004800DE00A0DF9F000E
:10FF6000FFD097008180FB000FD897004800DD008C
:10FF700001007000BF7897008180FB000100400005
:10FF8000F0D79F004800DE0080DF9F00DFD09700A1
:10FF90008180FB006FD097004800DD0001007000F9
:10FFA000AF7897008180FB0001004000D0D79F0010
:10FFB0004800DE00E0D79F009FD097008180FB00C3
:10FFC0002FD097004800DD0001017000BFD09700DE
:10FFD0008180FB004FD097004800DD008101700058
:10FFE0002800900000004100E080490090D79F0069
:10FFF0004801DE00A2D79F00B1D79F004808DE006D
:020000040001F9
:10000000C0D79F00DFC897008180FB006FC89700B2
:100010004800DD0001017000FFC897008180FB00EF
:100020000FD097004800DD00810170001F989700F5
:1000300000004100E0804900D0CF9F004801DE0071
:10004000E2CF9F00F1CF9F004808DE0080D79F00DD
:100050009FC897008180FB002FC897004800DD00F3
:1000600001017000BFC897008180FB004FC8970056
:100070004800DD0081017000180078000000410098
:10008000E080490090CF9F004801DE00A2CF9F0092
:10009000B1CF9F004808DE00C0CF9F00FFC097008F
:1000A0008180FB000FC897004800DD000100700050
:1000B0009F7897008180FB0001004000F0C79F00FF
:1000C0004800DE0080CF9F006E054500E0854D00B2
:1000D00000402000010020001FB99700AFB9970031
:1000E0000200400083804800800F5500818F5D0032
:1000F00031FF390053FC2F000F8441008042EB0098
:1001000062CC7200E5C79F000C00BE00F2FE070043
:100110000000E000100032000C00BE006112070079
:100120000D003700C1FA2F008F80400008007800D2
:10013000B0587800B0587800904878006F919700D8
:10014000FF9197000C00BE006D120700620646008A
:10015000E0864E00630444006E805700800F540018
:10016000F0FF3A004F06BE004F05BE004F04780076
:100170000080FA00000006002E00FA0023FD2F0088
:100180008F814100D2022000F31107009FA8970041
:100190000110A2000100EA00010070004F00DE0023
:1001A000610010000080FA00000006001600FA004E
:1001B000889FBE008A9FBE000005BE007E044000EE
:1001C000E084480009003700FE81570052012000FA
:1001D0000800BE00E01107000FE897000008A30028
:1001E0000A003A006E044400E0844C000040200005
:1001F000010020000A0040008B804800800F54005E
:10020000818F5C00F0FF39006044B8000800BE0038
:100210004F05BE004F04BE000080FA00000006003B
:10022000817E2400F20F200011486100914090006F
:1002300011409800A37E24009300610021409800A3
:100240009341900033409800C17E24001101610069
:10025000424098009140900051409800B17F2400A6
:100260009140780061409800C17F2400914078005F
:1002700071409800D17F2400914078000148980097
:10028000E17E24009140780011489800F17E24001E
:100290009140780021489800017F24009140780027
:1002A00031489800117F240091407800414898001F
:1002B000217F24009140780051489800317F24002C
:1002C0009140780061489800617F24009140780057
:1002D00071489800717F2400914078000150980087
:1002E000517F24009140780011509800917F2400A4
:1002F0009140780021509800A17F2400914078001F
:1003000031509800000006001A00FA00881F78009B
:100310008A9FBE000001EB001102210000012000B5
:100320009924070061012000807E2400A724070093
:10033000C8240700E17F2400910F50000400320020
:10034000820120008000EB00807E2400D6C20700DE
:1003500040C7BF000018A3000300320010C0B30064
:1003600024FD07004027A900A07F24001004E0001E
:1003700004003A00817E2400005A2000910F1000F2
:10038000650036006232EF000004EB006212E2000A
:1003900006003A00100020000ED707000804E8000D
:1003A00000712200800F5400F8FF3A001193800082
:1003B000F0282000808F50005700340000C0230038
:1003C000110020006CFF07000000E00007003A0069
:1003D000000024001100200067FF07006011B80032
:1003E0000000E0001E0032001400370000C02300AF
:1003F000110020006DFF07000005BE00E00F500057
:10040000E08F58001B003A0000002400110020007B
:1004100059FF07000000E00008003A0002C0230076
:1004200013002000000024001100200044FE0700FB
:10043000EA0124001B0020000E0037000000240009
:100440001100200059FF07000005BE00E00F50001A
:10045000E08F580007003A0002002400130020003B
:1004600000C023001100200035FE0700EAC1230070
:100470001B0020007C8457000800780068FF0700FC
:100480000D00370001FE2F008F804000080078002B
:10049000B0587800B0587800904878000FB19700B5
:1004A0009FB197000A00BE00951107006205450044
:1004B000E0854D006304440067805700800F5400BE
:1004C000F0FF3A000200240013002000820F5500C4
:1004D000838F5D0004003A0002C023001300200057
:1004E0000A00BE0007003700004024001100200071
:1004F000800F5500818F5D0003003A0000C023008B
:10050000110020000EFE0700820120008000EB0099
:10051000807E240064C20700E17E24001140780040
:10052000E14F4000010032008048E8004F05BE0066
:100530004F0478000080FA00000006001C00FA005A
:10054000889FBE008A1F7800000578005001900047
:10055000E0019000F0EB070008C023001900200024
:100560000800BE00E610070080B79F0091B79F000B
:10057000E3FD2F008F814100320020008380E800DE
:100580000A0078006AEA07007FA89700E30F50008E
:1005900024003A0062044400E0844C00004024003F
:1005A00011002000800F5400818F5C00ECFF3A00A6
:1005B0007C8457000800780019FF0700E3FD2F0036
:1005C0008F81410052012000880078000A007800E5
:1005D00057EA0700820120008000EB00807E2400A3
:1005E00031C2070000C0230011002000BAFD07003F
:1005F0000000E0000300320000C0230011002000D2
:10060000281107000000240011002000B2FD07009F
:100610000000E00003003200000024001100200070
:10062000201107004F0578004F04BE000080FA003B
:10063000000006008000EB0001089800710098009F
:1006400021189800200190000109780030019000E5
:10065000020141004000900013C2370020019000C9
:100660001203780015002000230020000900370045
:100670006482410062807900810F500003003A00DB
:100680000300410010009000000006008582E80091
:1006900084017800868F5200F5FF390000000500C4
:1006A0000400FA0080089000E1BF9F00F000900075
:1006B000F1BF9F004300200064815700A100290082
:1006C000531507000080FA0000000600889FBE0056
:1006D00000047800E1FF0700800478000000E000DB
:1006E00012003200780090000008A30005003200DC
:1006F00070014400230020008100290008007800D8
:1007000043150700090C98000080EB00100C9800BE
:10071000780090000000A000700498000018A3006A
:100720000200320008007800DDFF070009007800B1
:100730004F04BE0000000600889FBE0080047800C1
:10074000020478006119B800F10F5100E08F5900E0
:100750005B003E000260010011003700120037000C
:10076000130037001400370015003700170037005A
:100770002A0037002D0037002E0037002F003700E9
:1007800030003700330037003600370039003700BB
:100790003C0037003F00370042003700440037007C
:1007A0000809DD00490037000889DE0047003700EE
:1007B00008814000450037000881500043003700A1
:1007C0000888B90000017800400037000800E00008
:1007D0000E003A0080C427000000E0000300320051
:1007E000880078000900780029FC07002300200019
:1007F000F30498007081440071002900090078001A
:1008000003150700080178003000370011000900C7
:100810008800D800000178002C0037001100090082
:100820008800D80001017800280037000881700096
:100830002600370008816800240037000881600026
:10084000220037000001EB00888F50001F003A00A3
:100850001D0037000001EB00888F50001B003200A4
:10086000190037000001EB00888F5000170034009A
:10087000150037000001EB00888F50001300350091
:10088000110037000001EB00888F50000F003D0081
:100890000D0037000001EB00888F50000B003C007A
:1008A000090037000100E00007003A0002003700AD
:1008B0000100E000020032000800E00002003A00FF
:1008C0000001EB0001003700120020000200780058
:1008D0004F04BE00000006000600FA00889FBE001C
:1008E0000004780020029000800A900005814200F8
:1008F000E2047A004C48DE0001002000EE0F5000B8
:10090000E08F5800F6003E00006001000E00370046
:100910001100370019003700270037003200370078
:100920003D0037004F003700730037008A00370062
:10093000990037009C003700C2003700CF00370015
:10094000D5003700DF003700780090000000A100DC
:1009500070049800E20037006801900018089000C9
:100960000000E800100C980000004000C448DD00C2
:10097000C488DE0001307900C4003700E80190002F
:10098000980890008100E800110C980081804000D8
:10099000080890002801900000004000020040007C
:1009A0001000900080B07900080890000080E800F6
:1009B000000C9800CA003700E801900098089000E9
:1009C0008100E800110C980081804000F0FF2000B9
:1009D0000080640048019000000040006001790040
:1009E00082B07900A900370018099000F0FF2000BC
:1009F000008064004802900000004000E801900080
:100A000082004100E181790003307A000201E900AF
:100A1000120C98009D003700F0FF200080816400D8
:100A200002004200100290001808900000004000F0
:100A3000E80090000101400012007800840F50008F
:100A400003003900B5BF9F00C4BF9F0013003700EB
:100A500003004000C800900000004000608978005A
:100A6000D1FF3700F0FF20008081640002004200C7
:100A700010019000E800900018089000000040006D
:100A80008080400071BA970011007800820F5000FA
:100A900011003900B5BF9F00C2BF9F00D0BF9F00AB
:100AA0002000200070049800630020006A81570035
:100AB00061002900080078005514070080C4270051
:100AC0000000E000860032008000EB0008007800A3
:100AD0006FFB07008200370003004000C800900051
:100AE0000000400004B07800180890000080E90081
:100AF000100C9800ACFF3700180890000000400070
:100B0000E80090008101400013017800090078009E
:100B1000F00FB200E10F500007003200040039006E
:100B20008000EB00E20F500009003A000700370098
:100B30008200EA0006003700820078000200E00030
:100B400003003D008200EA00010037008280EA00D5
:100B5000810978004D003700E800900018089000E7
:100B6000000040006081780080804000F1B897006C
:100B70008981FB0008007800EFFE070098089000CC
:100B80008100E900110C980068019000818040000C
:100B9000803079003D0037004448DD004480DE00AD
:100BA0000080420082FF3700E800900018089000A3
:100BB000000040006081780080804000F1B897001C
:100BC0008981FB0008007800DBFE07000002780046
:100BD000180890000080E900100C98000400E00064
:100BE000040032000988A3000A0032000998A3001B
:100BF00008003200280190000808900080004000A2
:100C000001004100900190000400E00002003A0061
:100C10000700370023002000080890000000400073
:100C2000A8009000010040001090A00002003700D2
:100C3000010041001090A1000808900000804100D0
:100C40005BFF370002004200A001900010019000FD
:100C5000020141004800900000014100F1FF200026
:100C6000818064008381410008007800E813070058
:100C700008089000630040004DFF3700F1FF20009E
:100C80008180640008007800E30A070008089000EB
:100C90000000E80046FF3700680190001808900047
:100CA0000000E800100C9800000040008808900048
:100CB0008100E80001307900F0FF2000008064002E
:100CC0003BFF37001808900068019000800040004A
:100CD00061017900020C98000000E900100C9800F6
:100CE0004F04BE000080FA00000006000000FA0079
:100CF000889FBE008A9FBE008C9FBE008005780042
:100D0000010578008F067800010078006DC00700AB
:100D10000004780063064000650040000000A10068
:100D2000808747008D04780080C427000000E00021
:100D3000030032008A0078000B007800D4FA070024
:100D400020002000F00598000B089000800C78002F
:100D5000A844980063804400080178008A00780065
:100D60005EC007008C01780009017800910029001D
:100D70000B007800A61307008D0778004F06BE0011
:100D80004F05BE004F04BE000080FA0000000600C0
:100D900080007800201A9000F40140000001EB0070
:100DA0000800370001089000B30F100004003A005B
:100DB000710090000010A000F000980010000500E5
:100DC0000201E800840F5100F6FF39000000050021
:100DD000889FBE008A1F7800000478000105780013
:100DE000700090000020A000700498008004EB00C8
:100DF0000100E00004003A000D0037000800780010
:100E0000B5FE07008904E800780090000008A30000
:100E10000C0032000028A3000A0032008A8F540020
:100E2000F6FF3A000700370008007800AAFE070026
:100E3000780090000008A300020032000028A30000
:100E4000F9FF3A00780090000020A100700498009B
:100E50004F0578004F04BE0000000600889FBE00CA
:100E60008A1F780000047800010578007000900067
:100E70000020A000700498008004EB000100E00056
:100E800008003A001B00370008007800C0FF070088
:100E90008904E8000000E0000A003A000800780039
:100EA0008DFE0700780090000008A30016003200B5
:100EB0000028A300140032008A8F5400F2FF3A0089
:100EC00011003700780090000010A0007004980016
:100ED00008007800F2FD07000E00370008007800D7
:100EE000ABFF07000000E000F6FF3A0008007800C2
:100EF00079FE0700780090000008A300020032008D
:100F00000028A300F5FF3A00780090000020A1001F
:100F1000700498004F0578004F04BE0000000600E2
:100F200000017800700090000008A3000B00320060
:100F30000018A30009003A00221890000000E00009
:100F40000300320002007800C4FF070002003700EF
:100F5000020078009EFF0700100005000000050059
:100F600080017800201990000000EB00EF0F510085
:100F700006003E00020041007400400001B079000C
:100F80000200E800A01998001000200000000600F0
:100F90000001780001037800A0199000740240005D
:100FA0000000EB008302E900140037008000E80035
:100FB000B40F130010003A002519980081804000FA
:100FC000F4804000800178000502780000004000B5
:100FD000740040000101410001005000030037008F
:100FE000123079008301E8000281E800848F51000B
:100FF000FBFF39001000050001007800830F50004E
:10100000EAFF3900000005008000EB00211898007D
:101010000000060000027800920078000100E00065
:10102000060035008DFD07008001EB000000E000A8
:101030000F003A00130020000D00370013002000BD
:10104000F0FF2900808F5000090036001201900047
:101050008001EB000000E800808F500004003200A7
:10106000940069000100EA0001007000CF01DE0079
:1010700003007800000006000400FA00881F7800D2
:10108000000478008102780000002A00808F500060
:1010900003003A00080078001113070077003700BA
:1010A00012007800980F500074003A000282E800A5
:1010B000F0FF2500F1FF2F0005004000E080480010
:1010C000EE0F5000E08F58006C003E000060010001
:1010D0000E0037001A003700210037002B003700C0
:1010E00030003700350037002B003700350037005F
:1010F0004000370043003700450037004900370003
:1011000056003700580037005A0037008381E90045
:101110001400780000014000840078000002EB0019
:101120000400370028009000113178000402E80024
:101130000281E8008180E800830F5200F9FF390046
:1011400020002000700498008080EB0008007800E8
:101150005EFD07000000E00048003A000E00370086
:10116000780090000010A10070049800080078003A
:101170004BFD070000E627000000E0003F003200C2
:1011800008007800CEFA07003C0037007800900095
:101190000010A000700498000800780040FD0700CF
:1011A00036003700780090000008A30033003200BA
:1011B00008007800C8FD0700F7FF37002000200076
:1011C000F4FF370094007800D1BF9F00080078003A
:1011D00063FF07000080FB00E0BF9F00430020008A
:1011E00066815700B10029000800780088120700C6
:1011F00022003700940078000800780064FF0700A0
:101200001E0037000000EB00201C98001B00370078
:1012100022019000940078000800780092120700E4
:10122000160037008381E9001400780000014000B7
:10123000840078000002EB000400370048009000B2
:10124000113178000402E8000281E8008180E800A2
:10125000830F5200F9FF39000800370008007800BA
:101260007509070005003700080078002609070007
:101270000200370008007800620907004F04780078
:101280000080FA00000006000080FB004013880088
:1012900060C2BF000008A300FDFF320040138000C1
:1012A0000080FB0000000600401F200070F988004D
:1012B00000C0EB00F4FF070000C0EB00F2FF0700E6
:1012C000E14F4000020032002E1FE200FAFF3A0018
:1012D0000080FB0000000600CDC2A80000C0EB00AB
:1012E000E9FF3700CDC2A900EFFF07001100200081
:1012F000E14F400002003200F7FF07008000EB00E2
:101300000100780000000600889FBE000004BE00B7
:101310004006200080F9880000C0EB00DAFF0700DB
:10132000E14F400003003A00301FE2002500320088
:10133000F9FF3700E24F400022003A00F10F200091
:101340004113880060C2BF000008A300FDFF320007
:1013500040138000004C78004113880060C2BF0039
:101360000008A300FDFF32004013800010449800E5
:101370004113880060C2BF000008A300FDFF3200D7
:1013800040138000204498004113880060C2BF00D1
:101390000008A300FDFF3200401380003044980095
:1013A00064044400E4845400E5FF3A0000C0EB000C
:1013B000B5FF070000C0EB00B3FF070010002000DE
:1013C000010037000000EB004F04BE0000000600E3
:1013D000889FBE000004780081447800B2FF0700B7
:1013E000E14F400015003A0009407800A6FF0700D1
:1013F000E3CF440013003200092020001840780099
:10140000A1FF0700184090000884E8009EFF070035
:101410008984E900F9FF3A0000C0EB009AFF070059
:1014200000C0EB0098FF070000C0EB0096FF07002C
:101430007F006000E50F5000020032000000EB006A
:1014400001003700100020004F04BE00000006001D
:10145000889FBE008A1F7800004578000204BE0005
:101460000004E00006003D000A74A1006011B8000D
:1014700070C3B300F6FF0700E14F500028003E00A4
:1014800095FF070097FF0700F10F20000000E00024
:10149000240032000A4078000064A0007AFF0700B0
:1014A0004848DE000100200077FF07004048DE00CA
:1014B0000100200074FF07004849DD004840DE00BD
:1014C00000007100C848DE006FFF07000840780088
:1014D0006DFF070050C9B3000A04E00004003200A9
:1014E0006E405000E84F55000100320010C0B300BC
:1014F00065FF0700A8C0B300EC4F550002003A009A
:1015000000C0EB0060FF070000C0EB005EFF0700BB
:101510000004E00002003D000844E900FAFF3A0040
:101520008080FB00010078004F0578004F04BE006A
:10153000000006000400FA00889FBE008A1F7800A1
:10154000110020000004E00082003A00CBC2BF007E
:101550000068A3007D003200CDC2A800C9C2A90066
:10156000B0132000101388006422EF0061E2A8008D
:1015700061E2A90062C2BF0031CEB3000140600049
:101580004041B30062E2B70062C2BF00C1CFB30006
:10159000014060000004A00062E2B70061E2A80020
:1015A000A8C0B30000C0EB0037FF07000844E90003
:1015B000FCFF3A006011B80008407800A4FF070063
:1015C00080447800E14F50004A003A00803E2000FD
:1015D00080F98800A21A20000300200080C0B30018
:1015E0009BFF0700E14F50002A003A00EA845700B1
:1015F00000C0EB0024FF0700805C78006680570085
:10160000808F5400FAFF3A000FF89700E14F500026
:1016100038003A009FF89700A0CAB30080CF50006E
:1016200034003A00301FE2000600320002002000C1
:101630000300240090CAB30085FF07000004E00007
:10164000F8FF3A00301FE2002A0032006011B800B3
:10165000A0C3B3007EFF07000004E00025003A00AD
:101660006A84570000C0EB0007FF0700005C7800A9
:10167000890F5400FBFF3A00EFF097000180FB0058
:10168000C8C0B3000068A3001B003A0048C0B30004
:10169000190037006011B80090CAB3006CFF070052
:1016A00028C0B3009ACAB300E14F500002003600D0
:1016B0000944780009457800301FE2000500320037
:1016C0006011B8000A40780061FF07000004E000E4
:1016D000F9FF3A00301FE20006003200022020002D
:1016E0000300200000C1B30059FF07000004E00020
:1016F000010032000044EB000880FB0060F9880024
:10170000F5FE07000804E0000B003200521FA9009C
:1017100061E2A90062C2BF0031CEB30001406000A7
:101720008041B30062E2B70030C0B3006262B7002C
:1017300061E2A80005003700EAFE0700E6FE0700A8
:10174000C9C2A80061E2A900521FA80052DFBF0071
:101750008080FB00010078004F0578004F04BE0038
:101760000080FA0000000600110020000004E000E4
:1017700002003A0052DFBF008080FB0001007800C9
:1017800000000600889FBE008A1F780001057800CF
:10179000844478000004E00032003A000404E000D1
:1017A0003000320052DFBF006104600030002000D2
:1017B0002D003A002C7FAB0004003A004918DD00F0
:1017C000C711DE00830170004911DD00E1CF540034
:1017D0000B003A0010C1B3001DFF07000004E00039
:1017E00019003A00012020000A007800C6FE070018
:1017F0000000E00014003200884478001300370035
:1018000020C1B30012FF07000004E0000F003A00FF
:1018100009447800012020000A007800BAFE070081
:101820000000E000030032000A20B0000844E90094
:10183000F8FF3A00884478006011B800C0C0B300D7
:1018400003FF07000100370019C0B300A2FE070024
:101850000000EB000904E00003003200100020004B
:1018600001003700400020004F0578004F04BE0003
:1018700000000600889FBE008A9FBE008C1F780073
:10188000810578000204BE00044578000004E000F1
:1018900040003A000404E0003E00320052DFBF0086
:1018A000310020000008A3003B003A0052DFBF00D7
:1018B000640660002100200037003A0060F98000D3
:1018C0000038A30004003A00C918DD00C714DE0088
:1018D000898470004914DD00E14F55000C003A0086
:1018E0000801BE0080C1B300D9FE07000004E0007B
:1018F00021003A00E1CFB3000B007800B4FE0700EE
:101900000000E0001C0032000C4578001B0037008E
:1019100066006000040032000A81FB000300200022
:1019200070C9B300CAFE07000801BE0090C1B30031
:10193000C7FE07000004E00010003A000A447800E7
:10194000C1CFB3000B007800A1FE07000000E0004B
:10195000030032000B20B0000844E900F8FF3A0011
:1019600008457800D1CFB3000000EB0098FE0700D7
:101970000000E00001003A001AC0B30056FE070064
:101980008000EB000A04E000030032001100200098
:101990000100370041002000010078004F06780068
:1019A0004F05BE004F04BE00000006001000FA0004
:1019B000889FBE008A1F780002057800480020003A
:1019C0000004E000D1003A0052DFBF00E1046000F3
:1019D00038002000CD003A00EACF5000A4003200C9
:1019E00008003E00E1CF5000160032001000390020
:1019F000E2CF50004F003200E3CF50000A003A001F
:101A00004F003700ECCF50009C0032006011B8004E
:101A100090C0B3009B003900EDCF50009E00320013
:101A2000EECF5000A900320048002000B600370079
:101A30002CFE07000000E000B000320026FE070088
:101A40001B0037006011B80090C0B30080FE070093
:101A50000004E000A9003A00010120007680570050
:101A600029FE07000000E000A4003200AFE8970064
:101A70000180FB004600DE003FF29700AFF09700C8
:101A8000E14F50000C003A000480FB004809DD00E3
:101A9000020040000000E800010020004A09DD00CB
:101AA000C600DE00810071004A00DD00008DBE002E
:101AB00009047800940037000181FB004611DE0024
:101AC0001FF097000080FB004200DD000001410094
:101AD0000FF09700630060004A00DD000001410044
:101AE0000201E80003002000FFE89700EFC060005B
:101AF0004FF097000008B2004780DE0080C0400031
:101B0000630062000000400080C0400081C0E80027
:101B10008180FB00E98050008100E9000300330070
:101B20000201410083814900FBFF3700028DBE00A6
:101B3000DFFF37000020200000097800DCFF3700BD
:101B400060F98000640460001D0032006011B8007C
:101B5000D0C8B3003EFE07000004E00067003A0072
:101B600000C0EB00C8FD070001012000768057008F
:101B7000E5FD07000000E0006000320008C3B3008C
:101B800000C0EB00C0FD07000844E900FCFF3A007C
:101B90004FF197000281FB004411DE00000120009C
:101BA000010020000201E9000300330000004000B2
:101BB00081804800FBFF3700008DBE0051003700D8
:101BC0006011B80090C0B30021FE07000004E000DF
:101BD0004A003A000101200076805700CAFD070044
:101BE0000000E000450032005FF19700CFF0970061
:101BF00060F98000620260000F003200010078008E
:101C0000F003B200000040000208B2004711DE00FD
:101C1000020040000000E8007FF197000281FB0015
:101C20004611DE000201E9000200DD000100200093
:101C3000008DBE00340037000280FB0001017800F7
:101C4000C207B2004291DE000201E800E30060003A
:101C5000C308DD004500DE00808040008100E80010
:101C60000191B900028DBE000404780026003700FF
:101C70002CDFBF00004978008DFF37006011B800ED
:101C8000A0C0B300F2FD0700010120000004E00045
:101C900016003200190037006011B800A0C3B3006D
:101CA000EBFD07000004E00014003A00090478008E
:101CB00000C0EB0074FD070000757C000804E8001C
:101CC000E40F54000F003200F9FF37006011B80034
:101CD000D0C8B300DEFD07000004E00007003A00B2
:101CE00000C0EB0068FD0700010420000A00780036
:101CF00085FD07000000E00002003A001800200007
:101D0000010037000004EB0073FD070008007800B5
:101D10004F0578004F04BE000080FA000000060066
:101D200080F980000000E000020032000000E900BD
:101D300080F9880070F980000000E00002003200A5
:101D40000000E90070F9880000000600889FBE00CE
:101D5000800478000004EB0003003700803E200080
:101D60009CD007000804E800890F5400FBFF3900ED
:101D70004F04BE00000006008040EB0050C0B300DE
:101D80006808070001C2B30000C1B300650807007E
:101D9000E0152000EDFF07008040EB0000C1B3001C
:101DA0006008070001C2B30010C1B3005D0807005E
:101DB000E0152000E5FF07008040EB0010C1B300F4
:101DC0005808070001C2B30040C1B300550807001E
:101DD000E0152000DDFF07008040EB0040C1B300AC
:101DE0005008070001C2B30050C1B3004D080700FE
:101DF000E0152000D5FF07008040EB0050C1B30084
:101E00004808070001C2B30020C1B300450807001D
:101E1000E0152000CDFF07008040EB0020C1B3009B
:101E20004008070001C2B30030C1B3003D080700FD
:101E3000E0152000C5FF07008040EB0030C1B30073
:101E40003808070001C2B300D0C1B300350807004D
:101E5000E0152000BDFF07008040EB00D0C1B300BB
:101E60003008070001C2B300E0C1B3002D0807002D
:101E7000E0152000B5FF07008040EB00E0C1B30093
:101E80002808070001C2B30050C0B30025080700AE
:101E9000E0152000ADFF07008040EB0050C0B3000C
:101EA0002008070001C2B30060C0B3001D0807008E
:101EB000E0152000A5FF07008040EB0060C0B300E4
:101EC0001808070001C2B30070C0B300150807006E
:101ED000E01520009DFF07008040EB0070C0B300BC
:101EE0001008070001C2B300C0C1B3000D0807000D
:101EF000E015200095FF07008040EB00C0C1B30053
:101F00000808070001C2B30040C2B300050807007B
:101F1000E01520008DFF07008040EB0040C2B300B9
:101F20000008070001C2B30050C2B300FD0707005C
:101F3000E015200085FF07008040EB0050C2B30091
:101F4000F807070001C2B300F0C1B300F5070700AE
:101F5000E01520007DFF07008040EB00F0C1B300DA
:101F6000F007070001C2B30080C1B300ED0707000E
:101F7000E015200075FF07008040EB0080C1B30032
:101F8000E807070001C2B30090C1B300E5070700EE
:101F9000E01520006DFF07008040EB0090C1B3000A
:101FA000E007070001C2B300A0C1B300DD070700CE
:101FB000E015200065FF07008040EB00A0C1B300E2
:101FC000D807070001C2B300B0C1B300D5070700AE
:101FD000E01520005DFF07008040EB00B0C1B300BA
:101FE000D007070001C2B30020C2B300CD0707002D
:101FF000E015200055FF07008040EB0020C2B30031
:10200000C807070001C2B30001407800C5070700F8
:10201000E01520004DFF07008040EB0000C2B30038
:10202000C007070001C2B30030C2B300BD070700FC
:10203000E015200045FF07008040EB0030C2B300F0
:10204000B807070001C2B30010C2B300B50707000C
:10205000E01520003DFF07008040EB0010C2B300F8
:10206000B007070001C2B30060C2B300AD070700AC
:10207000E015200035FF07008040EB0060C2B30090
:10208000A807070001C2B30070C2B300A50707008C
:10209000E01520002DFF07008040EB0070C2B30068
:1020A000A007070001C2B3000040EB009D07070036
:1020B000E015200025FF07008040EB00014078007C
:1020C0009807070001C2B300E0C0B30095070700FE
:1020D000E01520001DFF07008040EB00E0C0B300CA
:1020E0009007070001C2B30010C0B3008D070700BE
:1020F000E015200015FF07008040EB0010C0B30082
:102100008807070001C2B30060C1B300850707005C
:10211000E01520000DFF07008040EB0060C1B30018
:102120008007070001C2B30070C1B3007D0707003C
:10213000E015200005FF07008040EB0070C1B300F0
:102140007807070001C2B30080C0B300750707001D
:10215000E0152000FDFE07008040EB0080C0B300CA
:102160007007070001C2B30090C0B3006D070700FD
:10217000E0152000F5FE07008040EB0090C0B300A2
:102180006807070001C2B300A0C0B30065070700DD
:10219000E0152000EDFE07008040EB00A0C0B3007A
:1021A0006007070001C2B300B0C0B3005D070700BD
:1021B000E0152000E5FE07008040EB00B0C0B30052
:1021C0005807070001C2B300C0C0B300550707009D
:1021D000E0152000DDFE07008040EB00C0C0B3002A
:1021E0005007070001C2B300D0C0B3004D0707007D
:1021F000E0152000D5FE07008040EB00D0C0B30002
:102200004807070001C2B30020C0B300450707001C
:10221000E0152000CDFE07008040EB0020C0B30099
:102220004007070001C2B30030C0B3003D070700FC
:10223000E0152000C5FE07008040EB0030C0B30071
:102240003807070001C2B30040C0B30035070700DC
:10225000E0152000BDFE07008040EB0040C0B30049
:102260003007070001C2B30020C0B3002D070700EC
:1022700001C2B30000C1B3002A07070001C2B300C6
:1022800010C1B3002707070001C2B30040C1B3006B
:102290002407070001C2B30020C1B30021070700D3
:1022A00001C2B30030C1B3001E07070001C2B30072
:1022B0000040EB001B07070001C2B30010C0B300D1
:1022C0001807070001C2B300E0C1B30015070700FB
:1022D00001C2B30070C2B3001207070001C2B3000D
:1022E00080C1B3000F07070001C2B30090C1B30063
:1022F0000C07070001C2B300A0C1B3000907070023
:1023000001C2B300B0C1B3000607070001C2B300A9
:10231000C0C1B3000307070001C2B30040C2B3004D
:102320000007070001C2B30050C2B300FD0607005A
:1023300001C2B300F0C1B300FA06070001C2B30046
:10234000D0C1B300F706070001C2B30060C1B300FB
:10235000F406070001C2B30070C1B300F106070024
:1023600001C2B30080C0B300EE06070001C2B30093
:10237000D0C0B300EB06070001C2B300E0C0B30059
:10238000E806070000802000431C07001000200022
:10239000D9173700889FBE0070F32F007812B40061
:1023A000A1122000810F500004003E003A1FA80037
:1023B0008040EB0070C2B300DA0607002193800072
:1023C0001093800080804000803E20000088B9008B
:1023D000A2F82000801F7800110009004288D80070
:1023E000800078004F007800C118B1001002200072
:1023F000808F500004003E008040EB00D0C0B3004E
:10240000C80607003A3FA800B9C72F0009007800A6
:102410004412B400A8C12000880F500004003E0000
:102420008040EB0000C1B300BE0607003A5FA80081
:10243000090078004612B400880F500004003E00E6
:102440008040EB0010C1B300B60607003A7FA80039
:10245000090078004812B400880F500004003E00C4
:102460008040EB0040C1B300AE0607003A9FA800D1
:10247000090078004A12B400880F500004003E00A2
:102480008040EB0020C1B300A60607003ABFA800B9
:10249000090078004C12B400880F500004003E0080
:1024A0008040EB0030C1B3009E0607003ADFA80071
:1024B000090078004E12B400880F500004003E005E
:1024C0008040EB0001407800960607003AFFA80024
:1024D000090078005012B400880F500004003E003C
:1024E0008040EB0010C0B3008E0607003B1FA80021
:1024F000B9F92F00090078005A12B400E831200021
:10250000880F500004003E008040EB0060C1B30023
:10251000840607003B3FA800090078005C12B40065
:10252000880F500004003E008040EB0070C1B300F3
:102530007C0607003B5FA8007C12E20002003A0024
:102540007A12E200040032008040EB00D0C1B300F8
:10255000740607003B7FA800F193800080022000F2
:10256000808F50000B00340011948000800C2000FC
:10257000808F500007003400B0122000808F500080
:1025800004003C003B9FA8008040EB00E0C1B3008A
:10259000640607003BBFA8008040EB00C0C1B30049
:1025A000600607003BDFA8008040EB0050C2B3008C
:1025B0005C0607002A12E2000D0032008040EB00AA
:1025C00090C1B300570607008040EB00B0C1B300D4
:1025D000540607008040EB0040C2B30051060700DC
:1025E0008040EB00F0C1B3004E0607003BFFA8009F
:1025F0002C12E200040032008040EB0080C1B300E6
:10260000480607003C1FA8002E12E200040032001A
:102610008040EB00A0C1B300420607003C3FA80089
:10262000881A07000000E000040032008040EB0040
:10263000E0C0B3003B0607003C5FA8007212EC004C
:10264000E20F50000A003E007412EC00E20F50004E
:1026500007003E00B0938000F40F500004003400E7
:102660008040EB0080C0B3002E0607003C7FA8002E
:10267000D2F98000E3F98000F0FF2F00F100200084
:10268000800F5100818F590006003A008040EB0016
:1026900020C0B3002306070001C2B30030C0B3005E
:1026A00020060700C1F980008101E800C3F9880015
:1026B000700C2000808F510002003E000000E800F6
:1026C000F092880084F32F0004804000620C200008
:1026D000820F500001003E00F492880000E72F00B6
:1026E00000804000820F500003003E005E32EF0089
:1026F000800C20000093880080DA2F0000804000CA
:10270000820F500001003E000493880000CE2F008D
:1027100000804000E1182000810F500001003E00C1
:102720006032EF00004B2000808F510001003A0022
:10273000383FEF004F04BE000000060090089000F4
:10274000E001900001814000628179008100E90090
:10275000110898000200780000000600889FBE0063
:102760008A1F780000047800C0049000F3FF07007F
:102770000000400060857C00C804900008007800DC
:10278000EEFF070000004000E0807C00EF0F5500E6
:10279000070032000A00E00005003500700220004A
:1027A000800F550002003C000A407800DD0507005C
:1027B0004F0578004F04BE0000000600800178003D
:1027C0000003EB000271220054002000A50020004D
:1027D000811F7800110009008281D80081017800F2
:1027E000CF0078000000E00004003A000600E0009E
:1027F00002003A00E10F510003003A0006C3B300A3
:102800008658400016002000811F78001100090042
:102810000581D80000017800CF0078000402E900AB
:10282000EBFF3A00E0C2B3008048780070C7B30005
:102830009040980076405000A040980075404000BD
:10284000B0409800C4409800000006000E00FA0056
:10285000881F7800F0805700929B2A000C00090026
:10286000B2587800D100B10040049000B3FF0700D7
:102870000000400060047C0010002000131B0700D3
:10288000E41107000000EB00E10F440004003200F7
:10289000EF80570008007800C8FF070070805700DD
:1028A0002A1207004F0478000080FA00000006009A
:1028B0000E00FA00881F7800F0805700629C2A0002
:1028C0000C000900B2587800D100B100400490001B
:1028D0009AFF07000000400060047C00E10F440004
:1028E00002003A00250B0700070037001000200007
:1028F000F61A0700EF80570008007800AFFF0700C6
:1029000070805700F50A07004F0478000080FA0035
:10291000000006000E00FA00881F7800F0805700C3
:10292000329D2A000C000900B2587800D100B10095
:102930004004900081FF07000000400060047C001C
:1029400010002000E11A0700B21107000000EB00A0
:10295000E10F440004003200EF80570008007800C7
:1029600096FF070070805700F81107004F047800A9
:102970000080FA00000006000E00FA00881F7800B0
:10298000F0805700029E2A000C000900B25878001F
:10299000D100B1004004900068FF07000000400033
:1029A00060047C0010002000C81A0700991107007D
:1029B000080078004B1207000000E000050032001C
:1029C000EF805700080078007CFF070070805700F8
:1029D000DE1107004F0478000080FA0000000600B6
:1029E000E6874700889FBE008A9FBE008C9FBE007E
:1029F0008E1F780000047800C00490004FFF07008D
:102A000000004000E0847C0089BF9F00C804900063
:102A10000800780049FF070000004000E0847C00C7
:102A2000F9B79F00C80490000800780043FF070032
:102A30000000400060877C00C80490000800780017
:102A40003EFF070000004000E0867C00C8049000C4
:102A50000800780039FF07000000400060867C0015
:102A6000C80490000800780034FF07000000400010
:102A7000E0857C00C8049000080078002FFF070064
:102A80000000400060857C00C804900008007800C9
:102A90002AFF07000000400060847C000010200036
:102AA0008A1A0700884378000A4378008B4278002E
:102AB0000C4278008D4178000E417800EFE89700D5
:102AC0000FF09700C30507004F0778004F06BE00C0
:102AD0004F05BE004F04BE006F00B10000000600AD
:102AE000889FBE008A9FBE0000047800C00490004A
:102AF00012FF070000004000E0857C00C804900041
:102B0000080078000DFF07000000400060857C0091
:102B1000C80490000800780008FF0700000040008B
:102B200060817C008A4078000B407800D105070066
:102B30004F05BE004F04BE0000000600889FBE0087
:102B40008A9FBE0000047800C0049000FBFE0700CE
:102B500000004000E0857C00C80490000800780078
:102B6000F6FE07000000400060857C00C80490006D
:102B700008007800F1FE07000000400060817C0042
:102B80008A4078000B407800C80507004F05BE005A
:102B90004F04BE0000000600889FBE008A9FBE0052
:102BA00000047800C0049000E4FE0700000040002C
:102BB000E0857C00C804900008007800DFFE070074
:102BC0000000400060857C00C80490000800780088
:102BD000DAFE07000000400060817C008A40780037
:102BE0000B407800BF0507004F05BE004F04BE0034
:102BF00000000600889FBE008A9FBE008C1F7800E0
:102C000000047800C0049000CCFE070000004000E3
:102C100060867C00C804900008007800C7FE0700AA
:102C200000004000E0857C00C804900008007800A7
:102C3000C2FE07000000400060857C00C8049000D0
:102C400008007800BDFE07000000400060847C00A2
:102C5000200020001D1A07008C40780000C2B3003D
:102C6000B00407008B40780030C2B300AD04070009
:102C70008A40780010C2B300AA0407008840780098
:102C800020C2B300A70407004F0678004F05BE001E
:102C90004F04BE0000000600E6874700889FBE0084
:102CA0008A9FBE008C9FBE008E1F780000047800B3
:102CB000C0049000A1FE070000004000E0847C00FA
:102CC00089BF9F00C8049000080078009BFE0700A1
:102CD00000004000E0847C00F9B79F00C804900029
:102CE0000800780095FE07000000400060877C0027
:102CF000C80490000800780090FE07000000400023
:102D0000E0867C00C8049000080078008BFE070075
:102D10000000400060867C00C80490000800780035
:102D200086FE070000004000E0857C00C80490009B
:102D30000800780081FE07000000400060857C00EC
:102D4000C8049000080078007CFE070000004000E6
:102D500060847C0040002000DC1907008FF09700A1
:102D600000C1B3006F040700EFE8970010C1B30083
:102D70006C0407008E40780040C1B300690407006E
:102D80008D40780050C1B300660407008C40780085
:102D900020C1B300630407008B40780030C1B3004A
:102DA000600407008A4078000040EB005D040700E3
:102DB0008840780010C0B3005A0407004F0778001D
:102DC0004F06BE004F05BE004F04BE006F00B100AD
:102DD00000000600889FBE008A1F7800000478006B
:102DE000C004900055FE07000000400060857C0094
:102DF000C80490000800780050FE07000000400062
:102E000060847C0040002000B01907008A407800F0
:102E100060C1B300430407008840780070C1B3006C
:102E2000400407004F0578004F04BE000000060074
:102E3000881F78004004900040FE0700000040001A
:102E400060047C0000042000A0190700884078007E
:102E5000D0C1B300330407004F047800000006001F
:102E6000881F78004004900034FE070000004000F6
:102E700060047C000001200094190700884078005D
:102E8000E0C1B300270407004F04780000000600EB
:102E9000889FBE008A1F780000047800C00490005C
:102EA00026FE07000000400060857C00C8049000FA
:102EB0000800780021FE07000000400060847C00CC
:102EC00000202000811907008A40780060C2B3000A
:102ED000140407008840780070C2B3001104070092
:102EE0004F0578004F04BE0000000600889FBE001A
:102EF0008A1F780000047800C00490000FFE0700CD
:102F00000000400060857C00C80490000800780044
:102F10000AFE07000000400060847C0010002000D2
:102F20006A1907003B100700880078000A00780043
:102F3000FB1007004F0578004F04BE00000006009C
:102F4000889FBE008004780040049000FBFD0700CD
:102F500000004000800144000001EB0063007900A4
:102F60000008B000F10F2000810F5000040036006F
:102F7000D19E2A00090078005CF7070006003700A0
:102F80000281E800C0112000800F5100F3FF3A00D9
:102F900003007800211807004F04BE00000006005F
:102FA0005A1F000092100000000000009E1A00004E
:102FB00010010000020000000000FE00059A1F0042
:102FC0005C02D200112000005A1F00000000000027
:102FD00000000000000000000000000000000000F1
:102FE00000000000000000000000000000000000E1
:102FF00000000000000000000000000000000000D1
:10300000521B42001B321B002A1BA0009E609E0028
:103010001C9EB6009D6A9D00169DC4009C769C0077
:10302000189CB6009B469B00009B9A009A5E9A00F3
:10303000049AB800997499002C99F00098FC9700B4
:103040009E0F92000F860F007A0F6E000F460F0042
:10305000320F0A000F1E0F00820EF2000ECA0E0081
:10306000BA0EAE000EA20E00920E76000E141F00D5
:1030700000006200A379A300000000000097A300F5
:10308000AEA3010000BEA3000100C600A300000023
:103090000000CC00A3E2A3000100BE00A3010000D9
:1030A000C6A3000000000000F1A30000A40000007F
:1030B00000009E009BA29B00D29BFA009C0E750014
:1030C0004075700075B27500F4753600767C760038
:1030D000E076240077687700D6774E0078A07800F5
:1030E000BA784400798E7900C87902007A967A001D
:1030F000CA7BAE009358940026948A0094BC940036
:10310000F094700095CC95009E95760097FA950006
:103110004C96EA00961897003097480097A09700C1
:1031200012B50000C6110000C40400000000000039
:10313000AE1B0000B400000000000000FC0F000007
:103140000400000000000000EC2F0000DC00000084
:1031500000000000AE0F0000300000000000000082
:103160004C1F000002000000000000000C1F0000C7
:103170000800000002000000621C0300800F0F0026
:103180000F000000621C0000A00000000000000012
:10319000141F00000800000002000000AAACB400E8
:1031A000AC00000000000000E61E00000E00000061
:1031B00000000000143100000C00000000000000BE
:1031C0004E1F00000200000000000000981D0000DB
:1031D0003000000000000000441F00000400000058
:1031E000000000007A1E0000140000000000000033
:1031F0001C1F00000800000000000000241F000049
:103200000800000000000000B61E000010000000D2
:1032100000000000501F000002000000000000003D
:10322000000800007606000000000000F41E000008
:103230000E000000000000008A1600000C020000D2
:1032400000000000481F0000040000000000000013
:10325000521F0000020000000200000001000000F8
:103260002C1F00000600000000000000541F00009A
:103270000200000000000000961800000802000094
:10328000000000008E1E000014000000000000007E
:10329000261E0000240000000200000000000100C3
:1032A000000000000100000000010000000001001B
:1032B000000000000100000000010000000001000B
:1032C000000000000100000000010000561F000087
:1032D0000200000002000000E8030000321F0000AE
:1032E0000600000000000000581F0000020000005F
:1032F0000200000030CC00004A1E00001800000050
:1033000000000000C01100000600000002000000E4
:1033100076117A0011901100BE1100000200000029
:103320000200000032110000901100002E00000089
:10333000020000002E0354000068000079006D00B8
:10334000006900006F002D000049000049002000C6
:1033500000200000200020000020000020002000AD
:10336000002000002000200000200000200020009D
:10337000000000007A1100001600000002000000AA
:1033800016034D00006F000062007300007900001A
:1033900061002E00006F0000720067000000000056
:1033A0007611000004000000020000000403090080
:1033B0000400000032110000440000000200000080
:1033C00009024300000201000080FA000904000025
:1033D00000010200020100000524000010010400A9
:1033E000240202000524060000010500240100005B
:1033F0000107050081030800000209000401000024
:10340000020A000000000700050202004000000060
:1034100007058200024000000000000020110000AB
:103420001200000002000000120100000202000071
:1034300000081700060A0000000001000200010059
:103440001E11000002000000000000001611000024
:103450000800000000000000C81D0000300000004F
:1034600000000000621E00001800000000000000C4
:10347000021D00009600000000000000C61E0000B3
:103480001000000000000000D61E00001000000028
:1034900000000000F81D00002E00000002000000E7
:1034A000101114001213000001161700008403000D
:1034B00084038400038403008403840003840300E2
:1034C0000000000000A00F00A00FA0000FA00F0040
:1034D000A00FA0000FA00F008403840003000000D1
:1034E000A21E00001400000000000000DE0F00001B
:1034F0001E00000000000000021F00000A00000083
:1035000002000000900104000120000096002C0041
:1035100001000000381F000006000000000000004D
:10352000760E0000380100000200000012A71D0006
:10353000A78E000048A70000000000004DA758001B
:10354000A701000067A70100006AA70000000000B3
:10355000006DA7007EA70100008AA70001008E0071
:10356000A700000000009300A79EA7000100AC0088
:10357000A70000000000B000A7B8A7000100AC0041
:10358000A70000000000C300A7CFA7000100EB00C8
:10359000A7010000F1A7000000000000F7A703004A
:1035A000A8010000EBA7010000F1A7000100210025
:1035B000A801000027A80100002DA8000100330089
:1035C000A801000039A80100003FA8000000000089
:1035D0000045A80052A8010000EBA7000100F1007F
:1035E000A701000021A801000027A800000000009A
:1035F0000063A80074A80100008AA70001008B00E6
:10360000A80100008EA700000000000091A8A30000
:10361000A80100008AA70100008BA80001008E000D
:10362000A70000000000BB00A8C4A80001008A0099
:10363000A70100008BA80100008EA7000000000079
:1036400000D4A800E0A8010000EBA7000100F100F1
:10365000A701000021A801000027A80001002D00FB
:10366000A801000033A801000039A80001003F00B4
:10367000A80000000000F700A804A9000100250030
:10368000A900000000002700A934A90001002500BE
:10369000A900000000004D00A958A9000100250064
:1036A000A900000000007100A97EA900010025000A
:1036B000A900000000009800A9A2A9000100AC0028
:1036C000A7010000AEA9000000000000C830000003
:1036D0002C000000000000003E1F0000060000005B
:1036E000000000000000000090089000E001900041
:1036F00001814000628179008100E9001108980091
:103700000200780000000600B20C0700000037003D
:10371000080C07000000E000FDFF3A000000370041
:10372000970F07000000E000FDFF3A009EC0A900CF
:103730000048040001000000000006000000FE0038
:1037400000000600889FBE008004780040049000BE
:10375000E5FF07000000400060047C0009007800DD
:10376000E1FF07008000780090052000800F5400E2
:103770000400360081642A00090078005BF5070028
:1037800006003700C9019000018140008800440014
:10379000E0BA21006100780000B179004F04BE005A
:1037A00000000600889FBE0080047800400490005E
:1037B000CDFF07000000400060047C000900780095
:1037C000C9FF07008000780090052000800F54009A
:1037D0000400360081642A000900780043F50700E0
:1037E00006003700880144004901900081804000B4
:1037F000E0BA210061017900823178004F04BE00F7
:103800000000060001662A0038F5370040602A00F3
:10381000000006000000060081804000A2B52100E3
:10382000E100790001400100402C2A000000060060
:1038300040AD210000000600F0874700889FBE00D1
:103840008A9FBE008C9FBE008E1F780080BF9F00A5
:10385000588E8000698E800020009000D0B79F00B5
:1038600050C0B300E3EF07000085EB008085EB005C
:103870006066B8003E0020000800BE00200407007B
:103880008A0F50008B8F5800020031000005BE00E7
:103890000806BE000080200001002000080440004F
:1038A000898448000E07E900F3FF3A0091672A0077
:1038B000E10F4500E08F4D004600320061054500F4
:1038C000E0854D00EAB79F00FBB79F000C04BE00E7
:1038D0002A0020000800BE00720407000A05E90063
:1038E00000402000010020000804400089844800B6
:1038F0000A00E000F7FF3A000C00BE009C0407003D
:103900006FB09700FFB09700C70407008FB897000B
:1039100021009000C1BF2000EB0407001A0507003A
:103920000C00BE00F60307006FB19700FFB19700CF
:10393000800F5100818F59000200320041692A0036
:103940002400370062054600E0854E00E93F200074
:103950007A84570088017800320020000A00BE00F7
:10396000FD03070032002000DFB097000800780058
:1039700033B507000000E00013003A00DFB1970004
:10398000E3814100D3B79F0062054500E0854D000B
:103990008904E900EEFF3A00FC8157002200200074
:1039A0000A00BE00EC03070022002000DFB09700F1
:1039B0007C80570022B50700016E2A000000E0005D
:1039C00004003A0002003700A16B2A000100370012
:1039D00061702A000FB89700C4F407004F07780001
:1039E0004F06BE004F05BE004F04BE000F01B100E0
:1039F00000000600889FBE008A9FBE008C9FBE000C
:103A00003A8E80004B8E80000A04BE000006EB0058
:103A10002D352A000800BE00C20307009D0F50008C
:103A200007003A000C06E8000808B0000980B00062
:103A30008D86E800E80F560005003200F5FF3700DC
:103A40000C00E00002003200E80F560003003A00CC
:103A50000A00BE00130407000006EB004760DD000B
:103A6000CF80DE000A0040008B8048004004070041
:103A7000AEDBBF008080FB00000020008C01460010
:103A800022352A0063017900030020000200700043
:103A90008380700064040700310B2000F0BA21001D
:103AA00089040700B80407004F06BE004F05BE009A
:103AB0004F04BE0000000600889FBE008A9FBE0023
:103AC0008C9FBE003C8E80004D8E80000C04BE009A
:103AD0000005EB002B352A000800BE00910307000B
:103AE0009B0F500007003A000A05E8000808B000E4
:103AF0000980B0008B85E800E80F55000400320013
:103B0000F5FF37000080EB000A00E0000F003200F4
:103B10000A04E9004744DD00CFC4DE000C04440081
:103B20008D844C000800BE0084030700AEFBB70084
:103B300062044400E0844C00F3BA2100320B200000
:103B40000800BE00840307000000EB004F06BE0023
:103B50004F05BE004F04BE00000006000000FE003E
:103B6000FEFF37000400FA00889FBE008A9FBE0057
:103B70008C1F780010002000F0D488000200230081
:103B8000000020008000780002007800508E88003D
:103B9000618E88000040240011002000308E8800D3
:103BA000418E8800B324200062B92200B120200099
:103BB00010DE2200C50A070094C4BF000008A3005D
:103BC000020032009EC0A800010037001C1507004B
:103BD000CFC0BF0081CFB300014060005040B300B0
:103BE000CFE0B700E0A9210092F20700F0D48000F6
:103BF000908E880080002000D0908800588E800031
:103C0000698E80006055B8009ABF9F00ABBF9F00CF
:103C10003C0020000800BE00390307008A0F500056
:103C20008B8F5800030039000005BE0098BF9F002D
:103C3000A9BF9F0000802000010020000804400070
:103C4000898448000C06E900F2FF3A00E00F5500B5
:103C5000E08F5D0002003A000C0478000800370095
:103C60001FB99700AFB9970062004100E08049009A
:103C700013D58000C2BF20003703070018002000C2
:103C8000E0DA2900FA160700080078004F067800ED
:103C90004F05BE004F04BE000080FA000000060081
:103CA000CE31EF00D031EF008080EB00E0A92100A1
:103CB00086F20700670B0700813E2000E0A9210083
:103CC00097F40700E0A921008D080700320B0700D8
:103CD00069D580000900D100E105600002003A00CA
:103CE0000908A300F3FF3A00EA1C21002004200089
:103CF000010C200010C870001A04CF000A0039001F
:103D0000620545001A04CF0006003900740A070056
:103D10000000E00004003200DE2F0200000000007E
:103D2000010037007004440020042000F10120004D
:103D300010C860000800E000DEFF32000B00E00069
:103D4000020032000908A300DAFF3A008801E90006
:103D5000EF8F510005003C00100020000300DD0043
:103D60000080EA001A0D600006003700021D2100E5
:103D7000F1005400100020000100DD000080EA0086
:103D800012096000F0D48000A08E8800E1FF2F00AF
:103D900083805000C5FF37000600FA006680570098
:103DA000E1F0210004000900315878005000B10012
:103DB00063DCBF0001C8B30001406000BFF897009A
:103DC00001407000B0FF9F0020C6210021D02100DB
:103DD000E681570004000900335878005000B10014
:103DE0005300B10065004000810F5000F8FF3A0019
:103DF0000080FA0000000600889FBE008A9FBE0077
:103E00008C1F78008042780001427800834478005B
:103E10008181FB000980FB0000804100010220003D
:103E2000810F500002003C00094478000100370077
:103E300004C450008280FB00100020008105DD00DA
:103E40008880FB000585FB006519B900020045006C
:103E50002CC621000C0040000B4178008B1107009C
:103E6000894F54000500320088C054008180FB0057
:103E70000C0045000B417800841107004F067800C4
:103E80004F05BE004F04BE0000000600889FBE0024
:103E90008A9FBE008C1F7800804278000142780023
:103EA000834478008181FB000980FB000080410091
:103EB00001022000810F500002003C0009447800FC
:103EC0000100370004C450008280FB001000200075
:103ED0000100DD0080C5EA008880FB000585FB004D
:103EE0006519B900020045002CC621000C004000F5
:103EF0000B417800AA110700894F540005003200D9
:103F000088C054008180FB000C0045000B41780004
:103F1000A31107004F0678004F05BE004F04BE00F6
:103F200000000600889FBE008A9FBE000041780006
:103F30008144780070C2B300804F51004A003E00B7
:103F40000280FB00C305DE000B457800674461007A
:103F50008880FB00100020000102DD000441780091
:103F60008B81FB00E0F0210063407800804062001C
:103F7000FFCF540039003E000904E00007003A007A
:103F800020C621000104E000020032000080410050
:103F90000F00370004C1EA00050037000104E0000B
:103FA0000E003A001D00370002C1EA0020C62100C1
:103FB0000080410001022000791107002A0037002B
:103FC0000A80FB0021C62100010040000441780066
:103FD000010220002D1107002300370089417800DD
:103FE00008417800884078000B407800A7FF070060
:103FF00089404400FFCF50000200360000CEB300DD
:1040000080C0400003C2B30089C15100084178005C
:104010000B40780078FF07001300370089417800D3
:1040200008417800884078000B40780072FF070054
:1040300089404400FFCF50000200360000CEB3009C
:1040400080C0400003C2B30089C15100084178001C
:104050000A4078008DFF0700030037000104E000EC
:10406000D1FF3A00D6FF37004F05BE004F04BE0017
:1040700000000600D5A2A900EA150700803E200036
:10408000D4C707004022EF004382A9004362A90081
:104090004342A9004322A9004302A90042E2A90029
:1040A00042C2A90042A2A80042C2BF0031CEB30062
:1040B000014060008041B30042E2B70030C0B3006D
:1040C0004262B700100020002012880041E2A800E0
:1040D0000EDFBF000080FB00401288000FDFBF0032
:1040E0000080FB004012880010DFBF000080FB0052
:1040F0004012880011DFBF000080FB0040128800E2
:1041000012DFBF000080FB00401288008002200008
:10411000B0C70700D5A2A800E5F0210095427800BD
:10412000F4F021001442780003F12100934178005B
:1041300012F121001241780021F121009140780014
:1041400020C6210026D021000548780014409800A0
:10415000234098003240980041409800650040009C
:10416000860F5000F8FF3A0000000600D5A2A90013
:104170008002200097C707000EDFBF000080FB0011
:10418000401288000FDFBF000080FB004012880053
:1041900010DFBF000080FB004012880011DFBF006D
:1041A0000080FB004012880012DFBF000080FB008F
:1041B000401288008002200086C70700D5A2A80010
:1041C0001000200083C70700D5A2A90041E2A90082
:1041D00099153700889FBE008A9FBE008C9FBE0045
:1041E0008E1F7800014478008244780003457800EF
:1041F00084457800054678008646780007477800B1
:104200008040780080C1B30046FF070088407800F6
:1042100090C1B30043FF070089407800A0C1B300FC
:1042200040FF07008A407800B0C1B3003DFF07009F
:104230008B407800C0C1B3003AFF07008C40780083
:1042400040C2B30037FF07008D40780050C2B30072
:1042500034FF07008E407800F0C1B30031FF070043
:104260004F0778004F06BE004F05BE004F04BE004A
:1042700000000600889FBE00014478008244780058
:104280008040780020C0B30026FF070088407800F7
:1042900030C0B30023FF07008940780040C0B3005E
:1042A00020FF07004F04BE0000000600889FBE00EC
:1042B000014478008244780080407800B0C0B300A8
:1042C00018FF070088407800C0C0B30015FF070042
:1042D00089407800D0C0B30012FF07004F04BE0031
:1042E00000000600889FBE000144780082447800E8
:1042F0008040780080C0B3000AFF07008840780043
:1043000090C0B30007FF070089407800A0C0B30049
:1043100004FF07004F04BE000000060021E3A900CF
:1043200085A0A900004006000C00FA00F27F800082
:104330002043A90000188000A0BF9F001018800033
:10434000B0BF9F0020188000C0BF9F0030188000C1
:10435000D0BF9F0040188000E0BF9F005018800031
:10436000F0BF9F0060188000701880004063280034
:10437000E0198800E20F51001400320005003C00F3
:104380000200E00008003200E10F51001A003A007C
:1043900009003700E30F510010003200E40F510014
:1043A00015003A0011003700C802A900C822A80071
:1043B0001000200003003700C822A900C842A8004E
:1043C00020002000F07F88000B003700C842A900C1
:1043D000C862A80030002000FAFF3700C862A900B8
:1043E000C882A80040002000F6FF3700C882A9005C
:1043F000C802A800FE2FEF0010002000F17F80000F
:104400000100DD0001C6270001007000801988004E
:104410009021EF00C0C1B3009161B70021E3A80073
:10442000000000000000000000000000000000008C
:10443000000000002043A800000000000000000071
:10444000000000000000000000000000000000006C
:104450003D63A80000000000000000000000000014
:1044600000000000000000000000000090C1BF003C
:1044700081CFB300014060000024A00090E1B700AC
:10448000000000000000000000000000000000002C
:1044900000000000000000003D23A9008200780019
:1044A0006C805700421307000080FA0000000600ED
:1044B000E07F8000AEE7070021E3A90095A0A900F6
:1044C0003DE3A9000000EB00800C8800900C880000
:1044D000C802A900C822A900C842A900C862A90050
:1044E000C882A900CC140700D3143700889FBE00EF
:1044F0000004BE00CB140700E87F880021A3A900B8
:1045000021C3BF00C1CFB3000140600021E3B70069
:1045100000CEB3002063B7002043A90023C3BF002F
:104520007F40600023E3B7002343A80022C3BF00FD
:1045300031CCB300014060008041B30022E3B700FA
:104540002223A8002203A90025E3A800F0C1B3009C
:104550002563B70000382E00601988003000200065
:104560005019880010C62700801988008001EB00D0
:104570004319880095A0A80067C164004411DD00BC
:10458000AAC0BF00F1C8B300014060000240700043
:10459000AAE0B70040E32000E019880000E027000F
:1045A000F01988003DE3A800830C8800930C880074
:1045B000C0C1B3009161B70010002000B00C8800AA
:1045C000B00C80000005B000A00C88008080EB00DB
:1045D000F27F20000300200008007800D5E70700E4
:1045E000E07F80000901780041192A0064E7070094
:1045F000CC02A900CC22A900CC42A900CC62A9001F
:10460000CC82A900C802A900C822A900C842A900FA
:10461000C862A900C882A90020002000F07F88009D
:1046200021E3A800000000000000000000000000DE
:1046300000000000000000002043A800000000006F
:10464000000000000000000000000000C802A800F8
:104650003D23A90090C1BF0081CFB300014060009D
:104660000024A00090E1B700E07F800042E707004F
:104670004F04BE000000060074E7A9007AEC0700B2
:104680000000FE000000060084C4BF004300DE00FE
:10469000610060008086FB000004E000030032003F
:1046A000E0FF2F00B03B88000100370076A7EF0045
:1046B00070A7EF0072A7EF0074A7EF0078A7EF00D4
:1046C0007AA7EF0000CEB3004260B70045C7BF0035
:1046D0000044A1000046B30045E7B7000004EB002A
:1046E00008077800880478006055B8002C00200086
:1046F00040A7A8000040FE0040A7A90047EC070023
:104700000800E000020032007607A9008804A80033
:104710007007A9007647A90000E02700F01988007B
:104720000029B000E019880025E3A80000382E0019
:1047300060198800300020005019880021E3A8008B
:1047400020002000401988000002EB000102200038
:104750002023A800C842A8003C03A8004567A80081
:1047600000000000000000003C03A9002023A90075
:10477000C842A9004567A900001880000002420055
:104780008100E900F2FF3A00430F23000C00E00033
:10479000090032000C06E9000300780041112300F3
:1047A00004187800810F5000FDFF3A00000120003E
:1047B0000405B8000B0037000981440062807900CD
:1047C00000005500E0805D0004054000E0854800E1
:1047D00004B179008904E800F08F540001003A0028
:1047E0008C047800020120001100090042DDD8008D
:1047F00080007800B0122000808F500001003E0041
:10480000C112200040ED2F0000804000800F5200B8
:10481000020039000007EB00040037000E07E80033
:10482000E30F570001003A0093FF07007007A8004C
:104830007647A8000800E000100032004567A80095
:1048400084C4BF000028A30003003A0084C4BF0052
:104850000038A300FAFF32004567A90084C4BF00F6
:104860000038A300030032000D00E00003003A000E
:1048700081FF07007607A8008006EB000800EA0029
:10488000080070004F00DE006104100098FF370040
:1048900021042000914078008180FB00C508DE00E3
:1048A00092028000FF3FFC0000CEB3004260B700E0
:1048B000920288000500FC0050052000303B880073
:1048C000A00A2000303B880061E7A800000000003B
:1048D0000000000061E7AF00FEFF37009202800099
:1048E000FF3FFC00C508DD0042C0BF007F40600004
:1048F0000140700042E0B70092028800000006000C
:104900000001BE0094018000930188001080BA006D
:104910001201BA009401880080007800020078003B
:10492000000006000002BE00920180009501880090
:104930001000BA0092018800000006000002BE00CC
:1049400092018000950188001080BA0092018800D1
:104950000080FB0000000600E8874700889FBE003B
:104960008A9FBE008C9FBE008E1F78000005BE008F
:10497000F2B79F0083BF9F00405EDE000D00200065
:104980007FB097006104B80061004600E0804E00EF
:10499000C000DD00000020000A0050008B8058009D
:1049A0008100D1000080D3003200200003002000ED
:1049B0009BAF0700800F5400818F5C000100360020
:1049C0000004BE0008077800320020001100090032
:1049D0000284D800800378000103780090018000F1
:1049E000E0B79F009C0188000A02BE000FB9970043
:1049F0008001EB000A0037001400BA00004978007B
:104A00004800DE00104198009480BA0021419800CF
:104A1000630141008301E80062024200E0824A0033
:104A2000878F5100F4FF39000600E00006003200D5
:104A30001400BA0000597800E10F5300020036005C
:104A40004800DE00004978006FB0970090018800B0
:104A500032002000030020000800BE007EAF0700E7
:104A600000004000818048000A0540008B85480016
:104A70000FB897000E00400080BF9F007FB09700E6
:104A80000E005000F0B79F00BBFF3A004F077800C0
:104A90004F06BE004F05BE004F04BE008F00B100A0
:104AA000000006000400FA00881F7800D0BF9F00B5
:104AB000E1BF9F000001BE00F03FB20005003200E0
:104AC000E681570012E02000210A200020C92A00B8
:104AD00065130700980180009301880020042400DA
:104AE000003B88006110B8000008BB0068FF0700A9
:104AF000980188004F0478000080FA00000006004A
:104B00000400FA00881F7800D0BF9F00E1BF9F001B
:104B10000202BE00000178000008A3000500320078
:104B2000E681570012E02000410B200020C92A0036
:104B30004D13070098018000910188003000240087
:104B4000003B8800030020006120B8000009BB0082
:104B50004028DE00010020000089BB004CFF070058
:104B6000980188004F0478000080FA0000000600D9
:104B70000400FA00E0BF9F00F1BF9F000001BE00EB
:104B8000F007B20005003200E481570012E0200077
:104B9000610C200020C92A003313070062F288004C
:104BA00073F288004A3EEF009001800000F3880015
:104BB0009301880010002400003B88000080FA0068
